:100000000C94B20A0C94E30A0C94E30A0C94E30AED
:100010000C94E30A0C94E30A0C94E30A0C94E30AAC
:100020000C94E30A0C94E30A0C94E30A0C94E30A9C
:100030000C94E30A0C94E30A0C94E30A0C94E30A8C
:100040000C94E30A0C94145D0C94E30A0C94E30AF8
:100050000C94E30A0C94E30A0C94F2580C94676F26
:100060000C94E30A0C94AD4D0C94E30A0C94E30A4F
:100070000C94E30A0C94E30A0C94E30A0C94E30A4C
:100080000C94E30A0C94E30A0C94E30A0C94E30A3C
:100090000C94E30A0C94E30A0C94E30A0C94E30A2C
:1000A0000C94E30A0C94E30A0C94E30A0C94E30A1C
:1000B0000C94E30A0C94E30A0C94E30A0C94E30A0C
:1000C0000C94E30A0C94E30A0C94E30A0C94E30AFC
:1000D0000C94E30A0C94E30A0C94E30A0C94E30AEC
:1000E0000C94E30A375943595F59695983598F5919
:1000F000A959AB59D16ED66EDB6EE56E5E6FEF6EB1
:10010000F76EFF6E096F136F1D6F2C6F366F5E6F8A
:10011000406F4A6F546F7A707D7070707470B470F5
:10012000817085708B708F70937099709D70A170C5
:10013000B470A770AB70AF70084AD73B3BCE016E6E
:1001400084BCBFFDC12F3D6C74319ABD56833DDA2E
:100150003D00C77F11BED9E4BB4C3E916BAAAABE3D
:10016000000000803F05A84CCDB2D44EB93836A966
:10017000020C50B9918688083CA6AAAA2ABE0000A3
:1001800000803F007C3C3E5E2B3D3F2F5B5D3B2C67
:100190002A225C005072696E7465722073746F70ED
:1001A0007065642064657520746F206572726F726B
:1001B000732E2046697820746865206572726F72AC
:1001C00020616E6420757365204D39393920746F54
:1001D0002072657374617274212E202854656D70CD
:1001E00065726174757265206973207265736574D8
:1001F0002E20536574206974206265666F726520D5
:1002000072657374617274696E6729005072696EE9
:100210007465722068616C7465642E206B696C6C07
:1002200028292063616C6C6564202121006F6B00BC
:10023000526573656E643A0053657474696E6773D2
:100240002053746F726564002200556E6B6E6F7779
:100250006E20636F6D6D616E643A22007A5F6D612E
:10026000783A007A5F6D696E3A00795F6D61783A2D
:1002700000795F6D696E3A00785F6D61783A007859
:100280005F6D696E3A005A3A00593A0020436F7523
:100290006E7420583A00453A005A3A00593A0058CC
:1002A0003A004649524D574152455F4E414D453AFD
:1002B0004D61726C696E2056313B20537072696ECD
:1002C0007465722F6772626C206D6173687570203F
:1002D000666F722067656E36204649524D5741520F
:1002E000455F55524C3A687474703A2F2F77777780
:1002F0002E6D656E64656C2D70617274732E636F04
:100300006D2050524F544F434F4C5F564552534906
:100310004F4E3A312E30204D414348494E455F54AF
:100320005950453A4D656E64656C20455854525598
:100330004445525F434F554E543A310A0020423AE9
:100340000020453A00543A0020573A0020453A0030
:10035000543A0020403A00202F0020423A00202F3B
:10036000006F6B20543A00456E642066696C65200E
:100370006C69737400426567696E2066696C6520FC
:100380006C69737400446F6E65207072696E746975
:100390006E672066696C65005072696E74657220C4
:1003A00073746F707065642064657520746F206568
:1003B00072726F72732E20466978207468652065AA
:1003C00072726F7220616E6420757365204D3939C9
:1003D0003920746F2072657374617274212E202825
:1003E00054656D70657261747572652069732072F1
:1003F000657365742E205365742069742062656688
:100400006F72652072657374617274696E6729001A
:100410006F6B004E6F204C696E65204E756D626586
:1004200072207769746820636865636B73756D2CDF
:10043000204C617374204C696E653A004E6F204306
:100440006865636B73756D2077697468206C696E7D
:1004500065206E756D6265722C204C617374204C42
:10046000696E653A00636865636B73756D206D69CD
:10047000736D617463682C204C617374204C696ED9
:10048000653A004C696E65204E756D626572206933
:1004900073206E6F74204C617374204C696E6520FC
:1004A0004E756D6265722B312C204C617374204C3B
:1004B000696E653A00446F6E6520736176696E6798
:1004C0002066696C652E006F6B0020440020490097
:1004D0002020204D33303120500050494420736596
:1004E0007474696E67733A00205A00205900202006
:1004F0004D323036205800486F6D65206F66667348
:10050000657420286D6D293A00204500205A00208E
:10051000580020420020540020204D323035205316
:1005200000416476616E6365642076617269616220
:100530006C65733A20533D4D696E20666565647243
:1005400061746520286D6D2F73292C20543D4D69F1
:100550006E2074726176656C206665656472617484
:100560006520286D6D2F73292C20423D6D696E69C1
:100570006D756D207365676D656E742074696D654A
:1005800020286D73292C20583D6D6178696D756D3B
:10059000207859206A65726B20286D6D2F73292C85
:1005A00020205A3D6D6178696D756D205A206A650D
:1005B000726B20286D6D2F73290020540020204D70
:1005C000323034205300416363656C657261746935
:1005D0006F6E3A20533D616363656C657261746947
:1005E0006F6E2C20543D7265747261637420616378
:1005F00063656C65726174696F6E00204500205AF6
:100600000020590020204D3230312058004D6178B3
:10061000696D756D20416363656C65726174696FA6
:100620006E20286D6D2F7332293A00204500205A24
:100630000020590020204D3230332058004D617881
:10064000696D756D206665656472617465732028D7
:100650006D6D2F73293A00204500205A0020590063
:1006600020204D3932205800537465707320706516
:100670007220756E69743A0053746F7265642073EA
:10068000657474696E6773207265747265697665E6
:10069000643A002020506C616E6E65724275666629
:1006A000657242797465733A200020467265652050
:1006B0004D656D6F72793A2000417072203138209B
:1006C0003230313600436F6D70696C65643A2000DA
:1006D0004C756C7A426F7400207C20417574686F91
:1006E000723A2000323031322D31312D3236002035
:1006F0004C61737420557064617465643A200031F4
:100700002E302E30004D61726C696E200020536FC8
:100710006674776172652052657365740020576155
:10072000746368646F672052657365740020427259
:100730006F776E206F757420526573657400204565
:10074000787465726E616C20526573657400506FC9
:100750007765725570007374617274002200656E63
:10076000717565696E67202200FFFFFF0000A040E1
:100770000000A0400000803F00003E4300004843CE
:100780000000C8420000000000000000000000005F
:1007900000003E43000048430000C8420000000043
:1007A00000000000000000006563686F3A004572B9
:1007B000726F723A0020746F6F206C6F6E672065E5
:1007C0007874727573696F6E2070726576656E7479
:1007D00065640020636F6C6420657874727573695A
:1007E0006F6E2070726576656E746564006563680F
:1007F0006F3A006572726F722077726974696E6702
:1008000020746F2066696C65004E6F74205344201D
:100810007072696E74696E67002F005344207072A5
:10082000696E74696E67206279746520002E0044D9
:10083000656C6574696F6E206661696C65642C20F7
:1008400046696C653A200046696C652064656C6594
:100850007465643A002E006F70656E206661696C85
:1008600065642C2046696C653A200057726974698A
:100870006E6720746F2066696C653A20002E006FE9
:1008800070656E206661696C65642C2046696C65D4
:100890003A20002E006F70656E206661696C656499
:1008A0002C2046696C653A200046696C65207365AA
:1008B0006C6563746564002053697A653A00466923
:1008C0006C65206F70656E65643A002E006F706510
:1008D0006E206661696C65642C2046696C653A20FF
:1008E0000053442063617264206F6B006F70656E0B
:1008F000526F6F74206661696C656400766F6C7509
:100900006D652E696E6974206661696C656400535B
:100910004420696E6974206661696C006563686F64
:100920003A004572726F723A0054656D706572617B
:100930007475726520686561746564206265642001
:100940007377697463686564206F66662E204D4115
:100950005854454D5020747269676765726564200C
:100960002121003A2045787472756465722073778E
:10097000697463686564206F66662E204D494E5425
:10098000454D502074726967676572656420210067
:100990003A20457874727564657220737769746360
:1009A000686564206F66662E204D415854454D5051
:1009B00020747269676765726564202100202D20AC
:1009C000496E76616C6964206578747275646572CD
:1009D000206E756D626572202100202D20496E7693
:1009E000616C6964206578747275646572206E75D7
:1009F0006D6265722100504944204175746F7475B1
:100A00006E652066696E6973686564202120506C8C
:100A100061636520746865204B702C204B692061F0
:100A20006E64204B6420636F6E7374616E74732008
:100A3000696E2074686520636F6E666967757261A0
:100A400074696F6E2E6800504944204175746F744C
:100A5000756E65206661696C6564212074696D65D9
:100A60006F75740020403A006F6B20543A00504973
:100A700044204175746F74756E65206661696C659C
:100A800064212054656D706572617475726520749F
:100A90006F206869676800204B643A2000204B692A
:100AA0003A2000204B703A200020436C6173696348
:100AB0002050494420002054753A2000204B753ABC
:100AC0002000206D61783A2000206D696E3A200088
:100AD00020643A200020626961733A2000457272F6
:100AE0006F723A001000F401E0020E0120030901C8
:100AF00060030401A003FF00E003FA003004F500E6
:100B00008004F000F004EB005005E600B005E100C1
:100B10003006DC00B006D7004007D200E007CD0069
:100B20008008C8005009C300000ABE00F00AB900DE
:100B3000F00BB400100DAF00000EAA00600FA5006E
:100B4000B010A00050129B00C013960040159100F9
:100B5000C0168C00C0188700901A8200C01C7D004F
:100B6000901E7800E0207300E0226E00F0246900FF
:100B70004027640040295F00802B5A00D02D55008B
:100B8000902F5000A0314B0030334600F03441002C
:100B900060363C00C0373700F0383200103A2D0084
:100BA000003B2800F03B2300B03C1E00503D1900E4
:100BB000D03D1400203E0F00903E0A00D03E0500BC
:100BC00045313A200045303A20005A3A2000593A3F
:100BD0002000583A20004D53312C4D53322050699B
:100BE0006E730A00205A3A0020593A0020583A0001
:100BF000656E6473746F7073206869743A200024A2
:100C0000F4D43050C38E20C2A24017828B701112D0
:100C10007A910D816CD90AA861E108C7586607610D
:100C20005143061E4B5D05C145A7041A4111040935
:100C30003D9803713931034036DB0265339102D4AC
:100C4000305402802E1D02632CEE01752AC501B0BE
:100C500028A001102781018F2564012B244B01E07E
:100C6000223401AC211F018D200D01801FFC008466
:100C70001EED00971DDF00B81CD200E61BC6002049
:100C80001BBC00641AB200B219A8000A19A0006ABD
:100C9000189900D117910040178B00B516840031C8
:100CA000167E00B31579003A157300C7146F00580B
:100CB000146A00EE1366008813630025135E00C7F4
:100CC000125B006C12570015125400C111510070D4
:100CD000114F0021114B00D61049008D10470046DE
:100CE00010440002104200C00F4000800F3E00423E
:100CF0000F3C00060F3B00CB0E3800930E37005C14
:100D00000E3500270E3400F30D3200C10D31009076
:100D10000D3000600D2E00320D2D00050D2C00D978
:100D20000C2B00AE0C2900850C29005C0C2700352B
:100D30000C27000E0C2600E80B2400C40B2400A096
:100D40000B23007D0B23005A0B2100390B210018C7
:100D50000B2000F80A1F00D90A1E00BB0A1E009DC6
:100D60000A1D00800A1D00630A1C00470A1B002C94
:100D70000A1B00110A1A00F7091A00DD091900C43C
:100D8000091900AB091900920917007B09180063C3
:100D90000917004C09160036091600200916000A2A
:100DA000091500F5081500E0081400CC081400B877
:100DB000081400A4081400900813007D0812006BAA
:100DC00008130058081200460812003408110023C6
:100DD0000811001208110001081100F0071000E0CE
:100DE000071000D0071000C0071000B0070F00A1C7
:100DF00007100091070E0083070F0074070F0065AE
:100E0000070E0057070E0049070E003B070D002E86
:100E1000070E0020070D0013070D0006070D00F94F
:100E2000060C00ED060D00E0060C00D4060C00C810
:100E3000060C00BC060C00B0060C00A4060B0099C2
:100E4000060C008D060B0082060B0077060B006C6B
:100E5000060B0061060A0057060B004C060A00420A
:100E6000060A0038060A002E060A0024060A001A9E
:100E7000060A001006090007060A00FD050900F42D
:100E8000050900EB050900E2050900D9050900D0B4
:100E9000050900C7050900BE050900B5050800AD34
:100EA000050800A50509009C050800940508008CAC
:100EB000050800840508007C050800740508006C1E
:100EC000050700650508005D050700560508004E8A
:100ED00005070047050700400508003805070031F1
:100EE0000507002A050700230507001C0506001654
:100EF0000507000F0507000805060002050700FBAF
:100F0000040600F5040700EE040600E8040600E20B
:100F1000040700DB040600D5040600CF040600C960
:100F2000040600C3040600BD040600B7040600B1B1
:100F3000040500AC040600A6040600A00405009BFE
:100F400004060095040500900406008A0405008547
:100F5000040500800406007A04050075040500708D
:100F60000405006B04050066040500610405005CCF
:100F700004050057040500520405004D040500480F
:100F8000040500430405003E0404003A040500354E
:100F9000040500300404002C040500270404002389
:100FA0000405001E0404001A0404001604050011C0
:100FB0000404000D040400090405000404040000F6
:100FC000040400FC030400F8030400F4030400F02C
:100FD000030400EC030400E8030400E4030400E05D
:100FE000030400DC030400D8030400D4030400D08D
:100FF000030400CC030400C8030300C5030300245A
:10100000F404D9201BC40C5C0E9804C4095F02656B
:10101000077101F405F900FB04B30048048700C11F
:101020000369005803550003034500BE023A0084DB
:1010300002310053022A002902250004022000E4A4
:10104000011C00C8011900AF0117009801140084A9
:10105000011300710110006101100051010E0043E5
:10106000010D0036010B002B010B0020010B0015B8
:101070000109000C01090003010800FB000800F34E
:10108000000800EB000700E4000600DE000600D8C0
:10109000000600D2000600CC000500C7000500C213
:1010A000000500BD000400B9000400B5000400B153
:1010B000000400AD000400A9000400A5000300A284
:1010C0000003009F0004009B0003009800030095AC
:1010D00000020093000300900003008D0002008BCB
:1010E00000030088000200860002008400030081E3
:1010F0000002007F0002007D0002007B00020079F8
:101100000002007700010076000200740002007205
:10111000000100710002006F0002006D0001006C10
:101120000002006A00010069000200670001006619
:10113000000100650001006400020062000100611E
:10114000000100600001005F0002005D0001005C22
:101150000001005B0001005A000100590001005825
:101160000001005700010056000100550001005425
:101170000001005300000053000100520001005123
:10118000000100500001004F0001004E0000004E21
:101190000001004D0001004C0001004B0000004B1D
:1011A0000001004A00010049000100480000004819
:1011B0000001004700010046000000460001004514
:1011C000000000450001004400010043000000430E
:1011D0000001004200000042000100410000004107
:1011E000000100400001003F0000003F0001003E00
:1011F0000000003E0001003D0000003D0001003CF9
:101200000000003C0000003C0001003B0000003BEF
:101210000001003A0000003A0001003900000039E6
:1012200000010038000000380000003800010037DD
:1012300000000037000100360000003600000036D4
:1012400000010035000000350000003500010034C9
:1012500000000034000000340001003300000033BF
:1012600000000033000100320000003200000032B4
:1012700000010031000000310000003100010030A9
:1012800000000030000000300001002F0000002F9F
:101290000000002F0000002F0001002E0000002E93
:1012A0000000002E0001002D0000002D0000002D88
:1012B0000000002D0001002C0000002C0000002C7C
:1012C0000000002C0001002B0000002B0000002B70
:1012D0000000002B0001002A0000002A0000002A64
:1012E0000000002A00010029000000290000002958
:1012F000000000290000002900010028000000284B
:10130000000000280000002800000028000100273D
:101310000000002700000027000000270000002731
:101320000001002600000026000000260000002624
:101330000000002600010025000000250000002517
:101340000000002500000025000000250001002409
:1013500000000024000000240000002400000024FD
:1013600000010023000000230000002300000023F0
:1013700000000023000000230000002300010022E1
:1013800000000022000000220000002200000022D5
:1013900000000022000100210000002100000021C7
:1013A00000000021000000210000002100000021B9
:1013B00000010020000000200000002000000020AC
:1013C000000000200000002000000020000000209D
:1013D0000001001F0000001F0000001F0000001F90
:1013E0000000001F0000001F0000001F0001001E81
:1013F0000000001E0000001E0000001E000000652E
:1014000063686F3A000000090A02080B0C0D07061A
:1014100003040100000000000000000000000000C4
:1014200000000000000000000000000000000000BC
:101430000011100F0000000000000000000000007C
:101440000000000000000000000000010210202049
:101450000808102040102040800201020108040208
:10146000010102040810204080804020100804027E
:1014700001800402018040201008040201080402D7
:1014800001010204081020408001020408102040DD
:101490008005050505070508080808020202020A7A
:1014A0000A08080404040401010101010101010307
:1014B00003030303030303040707070C0C0C0C0CC2
:1014C0000C0C0C0202020206060606060606060BB5
:1014D0000B0B0B0B0B0B0B0000200023002600292D
:1014E000002C002F0032000001000003010601095A
:1014F0000100002200250028002B002E00310034BE
:101500000002010000050108010B01000021002478
:101510000027002A002D00300033000101000004E4
:101520000107010A014E414E494E495459494E4660
:10153000CDCCCC3D0AD7233C17B7D13877CC2B3252
:101540009595E6241FB14F0A000020410000C842D3
:1015500000401C4620BCBE4CCA1B0E5AAEC59D7432
:10156000B935BD3511241FBECFEFD1E2DEBFCDBFEF
:1015700000E00CBF13E0A0E0B2E0E0E5F9EF00E02E
:101580000BBF02C007900D92A83EB107D9F72FE01C
:10159000A8EEB3E001C01D92A938B207E1F715E14A
:1015A000C2E6D5E100E006C022970109FE010BBFAB
:1015B0000E946A76C036D10780E00807A9F70E942A
:1015C00073710C94977C0C940000CF93DF93EC0123
:1015D0009C012C5F3F4F41E050E060E070E0898D5E
:1015E0009A8D0E941A69882399F04D895E896F89C6
:1015F000788D452B462B472B59F44C815D816E81AC
:101600007F814D8B5E8B6F8B788F998190689983EA
:10161000DF91CF910895CF92DF92EF92FF920F93D7
:101620001F93CF93DF93EC0189899A89AB89BC8999
:10163000803E9F4FAF41B10510F080E06BC0CE01FE
:10164000C4DF8823D1F30E942E67182F8823A9F3C3
:10165000E98DFA8DCC80DD80EE80FF8032E0C31A08
:10166000D108E108F108058404C0CC0CDD1CEE1C97
:10167000FF1C0A94D2F786859785A089B189C80E88
:10168000D91EEA1EFB1E81E08093730DC092760F77
:10169000D092770FE092780FF092790F80E092E08D
:1016A000E6E7FDE0DF019C011D9221503040E1F7AB
:1016B00001E0E98DFA8D8481081790F426E73DE07A
:1016C000B701A601400F511D611D711D8091740D60
:1016D0009091750D0E94345C8823E1F00F5FE9CF93
:1016E000C12C82E0D82EE12CF12C058404C0CC0C56
:1016F000DD1CEE1CFF1C0A94D2F749895A896B89BC
:101700007C894C0D5D1D6E1D7F1D498B5A8B6B8B2B
:101710007C8B812FDF91CF911F910F91FF90EF90E4
:10172000DF90CF900895CF93DF93EC0141E06111FA
:1017300001C040E06C857D858E859F850E946E6727
:10174000882341F0888920E2829FC00111248A58B1
:10175000924F02C080E090E0DF91CF910895FB01AD
:101760002BE030E231932150E9F7DC0190E027E0F3
:101770003A2FEB2F8D9181110AC0DA013C9311961B
:10178000EC9381E0FB019081903239F525C08F32D6
:10179000A1F38E3219F0E4E8F1E008C02A30E1F05C
:1017A00098E02AE0E5CF31963817B1F03491311145
:1017B000FACF291788F03FED380F3E3568F431E055
:1017C000390FFB01E90FF11D9FE9980F9A3108F4D9
:1017D00080528083932FCCCF80E008950F931F9386
:1017E000CF93DF93EC018B018B81882311F080E094
:1017F00042C0FB018789803139F18032C1F783E033
:101800008B83F801428D538D648D758D4D8B5E8B6E
:101810006F8B788F9E012F5E3F4FC8010E94256815
:10182000882329F31A8F098F81E089831C821D8206
:101830001E821F82188619861A861B861C861D86A4
:101840001E861F86188A17C082E08B831D8A1E8A17
:101850001F8A188EFB01408D518D60E070E095E08D
:10186000440F551F661F771F9A95D1F7498B5A8BE6
:101870006B8B7C8BD7CFDF91CF911F910F91089508
:101880002F923F924F925F926F927F928F929F9290
:10189000AF92BF92CF92DF92EF92FF920F931F937E
:1018A000CF93DF93EC015B016A018B81811103C04F
:1018B0008FEF9FEFC9C0898180FFFACF49895A898C
:1018C0006B897C8988859985AA85BB852601612CD1
:1018D000712C8A019B01081B190B2A0B3B0B40162C
:1018E00051066206730618F06A01C81AD90A760111
:1018F0003E0124E0620E711CE114F10409F477C08A
:10190000488559856A857B854A0181E098222B812B
:101910001A012B01E9E05694479437942794EA95ED
:10192000D1F7898D9A8DFC01223049F4628D738D37
:10193000848D958D620D731D841D951D3DC0148190
:101940001150122181149104C9F4111117C0452BB3
:10195000462B472B49F48D899E89AF89B88D8C839E
:101960009D83AE83BF830AC04C815D816E817F8180
:1019700093010E94A667882309F49ACFE98DFA8D16
:101980006C817D818E819F816250710981099109ED
:10199000058404C0660F771F881F991F0A94D2F729
:1019A0002685378540895189620F731F841F951FD3
:1019B000610F711D811D911D20E032E02819390948
:1019C00087012E153F0508F489010115F2E01F0774
:1019D00069F52091760F3091770F4091780F5091F3
:1019E000790F621773078407950719F41FC0C601A2
:1019F0002BC09501AB01BC018091740D9091750DC8
:101A00000E94DB5B882309F453CFA00EB11E8885AA
:101A10009985AA85BB85800F911FA11DB11D88875F
:101A20009987AA87BB87E01AF10A66CF40E00E9437
:101A30006E67882309F43CCFB4016A58724FA8013D
:101A4000C5010E945F79E1CFDF91CF911F910F9186
:101A5000FF90EF90DF90CF90BF90AF909F908F90CE
:101A60007F906F905F904F903F902F900895CF930D
:101A7000DF931F92CDB7DEB741E050E0BE016F5F4C
:101A80007F4FFEDE019719F4898190E002C08FEF4D
:101A90009FEF0F90DF91CF910895CF92DF92EF9259
:101AA000FF920F931F93CF93DF936C01EB017A01A9
:101AB000FC018381823060F00085118522853385A9
:101AC0000F71112722273327012B022B032B11F033
:101AD0008FEF5CC04115510511F0F70110821DE038
:101AE00040E250E0BE01C601CBDE8032910539F004
:101AF00021E0892B09F420E0822F819547C02881BD
:101B00002223C1F0253E61F32E3251F33B853F7312
:101B10003F3061F4E114F10449F04A8D5B8D452BAF
:101B200029F42F713FEF320F323030F02B8523FD37
:101B3000D7CF2CC080E02AC030E021503109129F5D
:101B4000C001139F900D1124F701E80FF91F29819F
:101B500020832B8121832D8122832F81238329853B
:101B600024832E852583288926832A8927832C8907
:101B700020872E892187288D22872C8D23872E8DE3
:101B80002487288126FFD2CF1586D0CFDF91CF9131
:101B90001F910F91FF90EF90DF90CF9008951F93CA
:101BA000CF93DF93EC018B81823018F480E090E0DA
:101BB00023C0488559856A857B85A5E0769567951C
:101BC00057954795AA95D1F7142F1F70CE014FDF77
:101BD00097FDECCF488559856A857B85415E5F4FCF
:101BE0006F4F7F4F488759876A877B8720E2129F14
:101BF000C00111248A58924FDF91CF911F9108950F
:101C00004F925F926F927F92AF92BF92CF92DF928C
:101C1000EF92FF920F931F93CF93DF93EC016A0132
:101C20007B012B81222349F089899A89AB89BC8960
:101C300084179507A607B70710F480E06CC0223020
:101C400009F464C0C114D104E104F10449F41C8214
:101C50001D821E821F82188619861A861B865AC00C
:101C600088859985AA85BB85E98DFA8DE585F0E0A3
:101C70003996AC01BD0141505109610971090E2E1F
:101C800004C076956795579547950A94D2F79701C2
:101C90008601015011092109310904C036952795A3
:101CA00017950795EA95D2F7041715072607370702
:101CB00020F0892B8A2B8B2B49F48D899E89AF8943
:101CC000B88D8C839D83AE83BF8304C0041B150B2A
:101CD000260B370B280139015E0184E0A80EB11CE8
:101CE000411451046104710489F04C815D816E815D
:101CF0007F819501898D9A8D0E94A66791E0491A8E
:101D00005108610871088111EBCF05C0C886D986DA
:101D1000EA86FB8681E0DF91CF911F910F91FF90C2
:101D2000EF90DF90CF90BF90AF907F906F905F90DB
:101D30004F9008950F931F93CF93DF93EC018B8106
:101D40008823D9F1898187FF32C061E0CE01EBDCC5
:101D50008C01009791F1FC018081853E71F18B81AE
:101D6000823040F449895A896B897C89448F558F28
:101D7000668F778F4D895E896F89788DF801538FD3
:101D8000428F758B648BE091E803F091E903309703
:101D900059F0B8016A5E7F4FC80148961995F8015D
:101DA000808D918D938B828B89818F778983DF9151
:101DB000CF911F910F910C942E6781E0888380E072
:101DC000DF91CF911F910F910895CF93DF93EC0195
:101DD000B1DF1B82DF91CF910895FC012381211196
:101DE000F4CF08954F925F926F927F92AF92BF921D
:101DF000CF92DF92EF92FF920F931F93CF93DF93D7
:101E000000D01F92CDB7DEB75C016A017B01FC01F7
:101E100083818130E9F4818181FF1AC0F5018189D4
:101E20009289A389B48984179507A607B70780F01C
:101E3000892B8A2B8B2B09F476C0F50140845184C1
:101E400062847384B701A601C501DADE811102C084
:101E500080E06AC0F501818D928DC114D104E10446
:101E6000F10471F4458956896789708D0E94236A4F
:101E7000882371F3F501158A168A178A108E3AC0E5
:101E8000F50144815581668177819E012F5F3F4F27
:101E90000E94A6678823E1F249815A816B817C8187
:101EA000F501818D928DFC012789203139F4483F5D
:101EB000FFEF5F0761057105E8F407C0483F2FEFAA
:101EC000520762072FE07207A8F40E94236A882352
:101ED00009F4BECFF50144815581668177810FEF0A
:101EE0001FEF2FEF3FE0818D928D0E948B6888233A
:101EF00009F4AECFF501C18AD28AE38AF48A8181DE
:101F000080688183C50116DF882309F4A1CFB7015A
:101F1000A6014C145D046E047F0410F4B301A20109
:101F2000C5016EDE01C081E00F900F900F900F9001
:101F3000DF91CF911F910F91FF90EF90DF90CF90A5
:101F4000BF90AF907F906F905F904F900895FF92F9
:101F50000F931F93CF93DF93EC01F42E80E2689FE1
:101F6000F0011124EA58F24F8385817121F0842F0A
:101F7000827109F04FC08091760F9091770FA091F8
:101F8000780FB091790F8C879D87AE87BF87688B5C
:101F90004489558960E070E0BA0155274427028DD5
:101FA000138D20E030E0402B512B622B732B4D8B97
:101FB0005E8B6F8B788F8385887151F4048D158DBE
:101FC000268D378D098B1A8B2B8B3C8B81E00CC0B7
:101FD000803101F59E012F5E3F4F898D9A8D0E94C1
:101FE00025688823B9F084E08B838F2D8F708983D7
:101FF0001C821D821E821F82188619861A861B86E5
:10200000F4FE0BC040E050E0BA01CE01EBDE8111DE
:1020100004C011C01B8280E00EC0F5FE0BC04989D0
:102020005A896B897C89CE01DF91CF911F910F91E5
:10203000FF90E6CD81E0DF91CF911F910F91FF904E
:102040000895AF92BF92CF92DF92EF92FF920F93DB
:102050001F93CF93DF937C01EB016A01B22E898D30
:102060009A8DF701928F818F40E050E0BA01CE0146
:10207000C7DDA12C088519852A853B8589899A8920
:10208000AB89BC89081719072A073B07A0F585E02B
:1020900036952795179507958A95D1F70F70CE013C
:1020A0007EDD009709F482C0FC012081222311F01B
:1020B000253EB9F4A1100EC04091760F5091770FD4
:1020C0006091780F7091790FF70144875587668783
:1020D0007787008BFC018081AA24A3948111CACF49
:1020E0000AC04BE050E0BC01C6010E945279892B26
:1020F00009F0C0CF59C08B2D8274823409F056C0CC
:10210000AA2049F0F701008961E0C7010CDBEC016E
:10211000009769F44BC08B81823009F447C0CE012F
:102120007ADA882309F442C0C6E7DDE000E080E205
:10213000FE0111928A95E9F78BE0F601DE0101902C
:102140000D928A95E1F7E091E803F091E903309769
:1021500039F0BE01625F7F4FCE014096199508C0ED
:1021600081E298E2998B888B80E098E09F878E8748
:10217000888999899B8B8A8B998F888F8E859F857B
:102180009F8B8E8B0E942E67882381F04B2D602FB2
:10219000C701DF91CF911F910F91FF90EF90DF90DA
:1021A000CF90BF90AF90D3CEB7FEF0CF80E0DF915D
:1021B000CF911F910F91FF90EF90DF90CF90BF9044
:1021C000AF9008953F924F925F926F927F928F925D
:1021D0009F92AF92BF92CF92DF92EF92FF920F93B6
:1021E0001F93CF93DF93CDB7DEB7C354D1090FB69A
:1021F000F894DEBF0FBECDBF5C016B0124965FAFCC
:102200004EAF2497522E1C8E1F8E19821C82611590
:10221000710511F410E073C0FC0183818111FACFC4
:102220002496EEADFFAD249780818F3211F07601B8
:102230001DC02496EEADFFAD249780818F3231F41E
:1022400031962496FFAFEEAF2497F3CFF60183814A
:102250008250823060F3F601618D728DCE0101965D
:10226000BDDA8823B9F2CE0101967C018E01045EAD
:102270001F4F3801FE0131964F01402E312E19C0FB
:102280008823A9F121E0AE01495C5F4FB701C80185
:10229000D8DE882309F4BECFEC14FD0411F0C70189
:1022A00094DD0615170501F1942D832D7801092F72
:1022B000182FAE014E5B5F4FBE01695C7F4F2496C5
:1022C0008EAD9FAD24974BDA882309F4A3CF2496D3
:1022D000EEADFFAD249780818F3291F63196249632
:1022E000FFAFEEAF2497F3CF982D892DDFCF252DAB
:1022F000AE01495C5F4FB701C501A3DE182FCE01C7
:1023000001966BDDCE014C9668DD812FCD5BDF4FF2
:102310000FB6F894DEBF0FBECDBFDF91CF911F91F6
:102320000F91FF90EF90DF90CF90BF90AF909F9074
:102330008F907F906F905F904F903F900895CF93D4
:10234000DF93EC0140E050E0BA014CDD882369F0F6
:1023500061E0CE01E8D9009741F025EEFC01208331
:102360001B82DF91CF910C942E6780E0DF91CF919B
:1023700008951F93CF93DF93CDB7DEB76B970FB65A
:10238000F894DEBF0FBECDBFAB0119821C8222E0E4
:10239000BC01CE01019616DF182F882321F0CE0153
:1023A0000196CDDF182FCE01019617DD812F6B9698
:1023B0000FB6F894DEBF0FBECDBFDF91CF911F9156
:1023C00008952F923F924F925F926F927F928F92D9
:1023D0009F92AF92BF92CF92DF92EF92FF920F93B4
:1023E0001F93CF93DF9300D01F921F92CDB7DEB71C
:1023F0008C015B013A01DC0113968C9113978130BB
:10240000C1F411968C9181FF14C082FF18C0F801AD
:10241000418952896389748980859185A285B385B4
:1024200084179507A607B70751F0C801E9DB8111AA
:1024300006C081E0F80180838FEF9FEF3AC163010E
:1024400083C0D80159968D919C915A97FC01F481D3
:10245000F1501A012B0169E0569447943794279460
:102460006A95D1F7F221FD834A0121E09222FF23F0
:1024700009F476C080E092E08819990976018C15FC
:102480009D0508F47C01D8015996ED91FC915A976D
:1024900014962D903D904D905C901797B2E02B1ABA
:1024A000310841085108058404C0220C331C441C27
:1024B000551C0A94D2F786859785A089B189280E84
:1024C000391E4A1E5B1EED812E0E311C411C511C13
:1024D000E114F2E0FF0609F08AC08091760F909136
:1024E000770FA091780FB091790F82159305A4050D
:1024F000B50569F41092730D8FEF9FEFDC018093A7
:10250000760F9093770FA093780FB093790F950182
:10251000B201A1018091740D9091750D0E94345CFF
:10252000882309F486CFF80180859185A285B3853B
:102530008E0D9F1DA11DB11D80879187A287B38736
:10254000AE0CBF1CCE18DF08D80118964D915D91D6
:102550006D917C911B97C114D10409F072CF7DC09D
:102560008114910409F086CF14964D915D916D917F
:102570007C911797411551056105710559F45596E0
:102580008D919D910D90BC91A02D0097A105B10555
:1025900041F521C09E012F5F3F4F0E94A66788230F
:1025A00009F447CF89819A81AB81BC81F801218DE3
:1025B000328DF9012789203139F4883FFFEF9F07D9
:1025C000A105B10540F40DC0883F2FEF9207A20787
:1025D0002FE0B20730F0C8010E94E50A81114ACF0E
:1025E00028CFF80184839583A683B78343CF8114D2
:1025F000910419F5D80118964D915D916D917C91DA
:102600001B9751968D919D910D90BC91A02D4817CF
:1026100059076A077B0788F00E942E67882309F410
:1026200008CF81E08093730D2092760F3092770F60
:102630004092780F5092790F08C041E0C201B10179
:102640000E946E67882309F4F4CEA701B501C40186
:102650008A58924F0E945F7966CF51968D919D91D5
:102660000D90BC91A02DF801218184179507A60734
:10267000B70738F4418B528B638B748B20682183AE
:102680000CC08091E8039091E903892B31F061142B
:10269000710419F02068F8012183D80111968C91FA
:1026A00083FD02C0C30105C0C80144DB8111FACF1C
:1026B000C0CE0F900F900F900F900F90DF91CF91A1
:1026C0001F910F91FF90EF90DF90CF90BF90AF9050
:1026D0009F908F907F906F905F904F903F902F9042
:1026E0000895FC01659175918591949108957F926B
:1026F0008F929F92AF92BF92CF92DF92EF92FF9212
:102700000F931F93CF93DF93EC018C01000F111FE8
:10271000000F111FF801E952FA4F10821182128244
:10272000138223EE35E04FED55E06BED75E087ED5C
:1027300095E00E949C44C8018858984FD2DF9E01C2
:102740002759384F5901F90174904E01880C991C92
:10275000880C991C840103551A4F20E030E040ECAE
:102760005FE30E942E756B017C01672D772767FD63
:102770007095872F972F0E94FB729B01AC01C701B8
:10278000B6010E942E75F801608371838283938362
:10279000F401E75EFD4F60817181828193816093D6
:1027A000040270930502809306029093070220E0D2
:1027B00030E040E752E40E9460723EEBC32E35E009
:1027C000D32E7B018C0129EB35E045EB55E061EB25
:1027D00075E08DEA95E00E94253B0E945164F4016A
:1027E000E952FA4F108211821282138223EE35E0F1
:1027F0004FED55E06BED75E087ED95E00E949C4450
:1028000094012459384F4901C9016BDFF501249126
:102810008E01000F111F000F111F03551A4F6B017E
:102820007C01F7FAF094F7F8F094622F772767FDB0
:102830007095872F972F0E94FB729B01AC01C701F7
:10284000B6010E942E75F8016083718382839383A1
:1028500020E030E040E752E460910402709105020C
:1028600080910602909107020E9460725EEBC52E75
:1028700055E0D52E7B018C0129EB35E045EB55E089
:1028800061EB75E08DEA95E00E94253B0E94516462
:10289000C40127DFF5011491CC0FDD1FCC0FDD1F24
:1028A0009E0123553A4F59019B01AC010E94807152
:1028B0006B017C01612F772767FD7095872F972F1C
:1028C0000E94FB729B01AC01C701B6010E942E75EC
:1028D000F5016083718382839383FE01E75EFD4F80
:1028E00020E030E040E05FE360817181828193818C
:1028F0000E942E7560930402709305028093060275
:102900009093070220E030E040E752E40E946072BA
:10291000FEEBCF2EF5E0DF2E7B018C0129EB35E0BD
:1029200045EB55E061EB75E08DEA95E00E94253BB3
:102930000E945164CE018C57984FD3DE9E012952DC
:102940003A4F79018E0105531A4FF80120813181E8
:10295000428153810E948071F70160837183828379
:102960009383CE018456984FBCDE9E0121543A4F8A
:102970006901F80120813181428153810E94807177
:10298000F6016083718382839383CE018057984FD1
:10299000A8DEC75FDD4FF80120813181428153817C
:1029A0000E948071688379838A839B83F701808189
:1029B0009181A281B381F50180839183A283B38346
:1029C0001092040210920502109206021092070261
:1029D000DF91CF911F910F91FF90EF90DF90CF90FB
:1029E000BF90AF909F908F907F900C94045DFC01FE
:1029F0002491222341F03091C00035FFFCCF209379
:102A0000C6000196F4CF22E030E087E59CE00C940C
:102A1000D04FFC012491222341F03091C00035FFBA
:102A2000FCCF2093C6000196F4CF22E030E087E58A
:102A30009CE00C94D04FFC012491222341F0309172
:102A4000C00035FFFCCF2093C6000196F4CF2AE0EA
:102A500030E087E59CE00C94264FCF93DF93C8EAE3
:102A6000D7E0FE018491882341F09091C00095FF4A
:102A7000FCCF8093C6003196F5CFE8E6F6E084916E
:102A8000882341F09091C00095FFFCCF8093C60051
:102A90003196F5CF8091C00085FFFCCF8AE080930E
:102AA000C600FE018491E8EAF7E0882349F090919E
:102AB000C00095FFFCCF8093C60031968491F5CF7E
:102AC0004091330C5091340C6091350C7091360C60
:102AD00080E696E08CDF4091370C5091380C609185
:102AE000390C70913A0C8DE596E081DF40913B0CFA
:102AF00050913C0C60913D0C70913E0C8AE596E043
:102B000076DF40913F0C5091400C6091410C7091E8
:102B1000420C87E596E06BDF8091C00085FFFCCF1B
:102B20008AE08093C600FE018491E8EAF7E08823FA
:102B300049F09091C00095FFFCCF8093C60031967C
:102B40008491F5CFEDE3F6E08491882341F09091F4
:102B5000C00095FFFCCF8093C6003196F5CF8091E1
:102B6000C00085FFFCCF8AE08093C600FE018491FF
:102B7000E8EAF7E0882349F09091C00095FFFCCF88
:102B80008093C60031968491F5CF4091430C5091CB
:102B9000440C6091450C7091460C84E396E027DF6D
:102BA0004091470C5091480C6091490C70914A0C2F
:102BB00081E396E01CDF40914B0C50914C0C6091EE
:102BC0004D0C70914E0C8EE296E011DF40914F0C4F
:102BD0005091500C6091510C7091520C8BE296E028
:102BE00006DF8091C00085FFFCCF8AE08093C6009D
:102BF000FE018491E8EAF7E0882349F09091C00053
:102C000095FFFCCF8093C60031968491F5CFEDE01F
:102C1000F6E08491882341F09091C00095FFFCCFAD
:102C20008093C6003196F5CF8091C00085FFFCCF20
:102C30008AE08093C600FE018491E8EAF7E08823E9
:102C400049F09091C00095FFFCCF8093C60031966B
:102C50008491F5CF4091230C5091240C6091250C68
:102C60007091260C84E096E0E6DE4091270C5091AE
:102C7000280C6091290C70912A0C81E096E0DBDE33
:102C800040912B0C50912C0C60912D0C70912E0CBE
:102C90008EEF95E0D0DE40912F0C5091300C60917A
:102CA000310C7091320C8BEF95E0C5DE8091C00045
:102CB00085FFFCCF8AE08093C600FE018491E8EA9C
:102CC000F7E0882349F09091C00095FFFCCF8093F6
:102CD000C60031968491F5CFE6ECF5E08491882327
:102CE00041F09091C00095FFFCCF8093C6003196D3
:102CF000F5CF8091C00085FFFCCF8AE08093C600AD
:102D0000FE018491E8EAF7E0882349F09091C00041
:102D100095FFFCCF8093C60031968491F5CF40910A
:102D20001B0C50911C0C60911D0C70911E0C8DEBB6
:102D300095E05DDE4091170C5091180C6091190CD4
:102D400070911A0C8AEB95E052DE8091C00085FFED
:102D5000FCCF8AE08093C600FE018491E8EAF7E0A8
:102D6000882349F09091C00095FFFCCF8093C60066
:102D700031968491F5CFE1E2F5E08491882341F02A
:102D80009091C00095FFFCCF8093C6003196F5CF9F
:102D90008091C00085FFFCCF8AE08093C600FE01D1
:102DA0008491E8EAF7E0882349F09091C00095FF0C
:102DB000FCCF8093C60031968491F5CF40911F0CD3
:102DC0005091200C6091210C7091220C88E195E0CB
:102DD0000EDE4091070C5091080C6091090C709127
:102DE0000A0C85E195E003DE4091530C5091540CA0
:102DF0006091550C7091560C82E195E01CDE40917B
:102E0000130C5091140C6091150C7091160C8FE0FE
:102E100095E0EDDD40910F0C5091100C6091110C7C
:102E20007091120C8CE095E0E2DD40910B0C50911A
:102E30000C0C60910D0C70910E0C89E095E0D7DDC3
:102E40008091C00085FFFCCF8AE08093C600FE0120
:102E50008491E8EAF7E0882349F09091C00095FF5B
:102E6000FCCF8093C60031968491F5CFE7EFF4E074
:102E70008491882341F09091C00095FFFCCF80930E
:102E8000C6003196F5CF8091C00085FFFCCF8AE067
:102E90008093C600FE018491E8EAF7E0882349F0B8
:102EA0009091C00095FFFCCF8093C600319684912D
:102EB000F5CF4091CB055091CC056091CD05709137
:102EC000CE058EEE94E093DD4091CF055091D00574
:102ED0006091D1057091D2058BEE94E088DD409130
:102EE000D3055091D4056091D5057091D60588EE33
:102EF00094E07DDD8091C00085FFFCCF8AE0809367
:102F0000C600FE018491E8EAF7E0882349F0909139
:102F1000C00095FFFCCF8093C60031968491F5CF19
:102F2000EAEDF4E08491882341F09091C00095FF90
:102F3000FCCF8093C6003196F5CF8091C00085FF0D
:102F4000FCCF8AE08093C600FE01C491E8EAF7E076
:102F5000CC2349F08091C00085FFFCCFC093C60010
:102F60003196C491F5CF409146025091470260914D
:102F700048027091490280ED94E039DD2DEB37E392
:102F800046E05EE360914202709143028091440208
:102F9000909145020E946072AB01BC018DEC94E0FF
:102FA00038DD2DEB37E346E05EE360913E02709141
:102FB0003F0280914002909141020E942E75AB0128
:102FC000BC018AEC94E025DD8091C00085FFFCCF38
:102FD0008AE08093C600DF91CF910895CF93DF936D
:102FE0001F921F92CDB7DEB78091830F9091840F0F
:102FF0009E012F5F3F4F009719F429583F4002C0B0
:10300000281B390B3A83298389819A810F900F906D
:10301000DF91CF9108952091020430910304243070
:1030200031050CF06AC0409104045091050460E63B
:10303000649F9001659F300D1124BC01C901845F1C
:103040009B4F0E947E79E8EAF7E08491882341F063
:103050009091C00095FFFCCF8093C6003196F5CFCC
:10306000EEE5F7E08491882341F09091C00095FF50
:10307000FCCF8093C6003196F5CF809104049091E7
:10308000050420E6289FF001299FF00D1124E45F3C
:10309000FB4F8191882339F09091C00095FFFCCFC0
:1030A0008093C600F6CFECE5F7E08491882341F0E9
:1030B0009091C00095FFFCCF8093C6003196F5CF6C
:1030C0008091C00085FFFCCF8AE08093C60080918C
:1030D000040490910504019664E070E00E94037678
:1030E000909305048093040480910204909103045A
:1030F0000196909303048093020408958091FC0349
:103100009091FD0360E070E001960C9491768091BF
:10311000FC039091FD034AE050E060E070E001960E
:103120000C94F977682F772767FD70952091060436
:103130003091070440E6429FC001439F900D112447
:10314000845F9B4F0E9473799093FD038093FC03EF
:1031500021E0892B09F420E0822F08950E94B16FAD
:103160006093F8037093F9038093FA039093FB0341
:10317000E0910604F0910704E85FFB4F8081811124
:1031800014C0EDE2F2E08491882341F09091C000F8
:1031900095FFFCCF8093C6003196F5CF8091C0009B
:1031A00085FFFCCF8AE08093C600089587E59CE008
:1031B0000E94384EE0E3F2E08491882341F0909140
:1031C000C00095FFFCCF8093C6003196F5CF4091AB
:1031D00091055091920560919305709194054F5F10
:1031E0005F4F6F4F7F4F2AE030E087E59CE00E9401
:1031F000D74E8091C00085FFFCCF8AE08093C60047
:10320000ADCF2F923F924F925F926F927F928F92AB
:103210009F92AF92BF92CF92DF92EF92FF920F9365
:103220001F93CF93DF93CDB7DEB76E970FB6F894A9
:10323000DEBF0FBECDBF90E6992E04E010E028E976
:10324000E22E23E0F22E3AE0832E40E1C42E44E049
:10325000D42E772473948091D80C9091D90C20911E
:10326000DA0C3091DB0C821B930B8F779927892B1B
:1032700009F421C2809102049091030404970CF098
:103280001AC287E59CE00E941C4E809301042091A5
:10329000FF03309100048A3061F08D3051F08A33A1
:1032A00021F49091FE03992321F02F3531050CF480
:1032B000E1C12115310509F4FBC18091040490910D
:1032C0000504989E5001999EB00C1124F501E20F5F
:1032D000F31FE45FFB4F10822091FE032111C5C153
:1032E0001092FE03FC01E85FFB4F10829501245F02
:1032F0003B4F29016EE470E0C9010E947379009789
:1033000009F40AC19093FD038093FC038419950985
:103310008A0D9B1D4AE050E060E070E0835F9B4FA8
:103320000E94F977609395057093960580939705B1
:1033300090939805209191053091920540919305C5
:10334000509194052F5F3F4F4F4F5F4FA090040463
:10335000B0900504621773078407950709F43AC013
:103360009A9CC0019B9C900D11246EE872E0845FD2
:103370009B4F0E94A279892B69F5EEEAF7E08491D0
:10338000882341F09091C00095FFFCCF8093C60048
:103390003196F5CFE3E8F4E08491882341F09091F1
:1033A000C00095FFFCCF8093C6003196F5CF4091C9
:1033B00091055091920560919305709194052AE0D2
:1033C00030E087E59CE00E94D74E8091C00085FFE9
:1033D000FCCF8CC09A9C20019B9C500C1124C201F4
:1033E000845F9B4F5C016AE270E00E9473790097F2
:1033F00009F450C020E0612CF201E20FF11DE45FFE
:10340000FB4F30813A3219F02F5F6326F5CF90934E
:10341000FD038093FC038A199B09840D951D60E0D0
:1034200070E0835F9B4F0E9491760E94C872262DA8
:1034300030E02617370709F45EC0EEEAF7E0849122
:10344000882341F09091C00095FFFCCF8093C60087
:103450003196F5CFE5E6F4E08491882341F0909130
:10346000C00095FFFCCF8093C6003196F5CF409108
:1034700091055091920560919305709194052AE011
:1034800030E087E59CE00E94D74E8091C00085FF28
:10349000FCCF2CC0EEEAF7E08491882341F09091B4
:1034A000C00095FFFCCF8093C6003196F5CFECE3CA
:1034B000F4E08491882341F09091C00095FFFCCF07
:1034C0008093C6003196F5CF4091910550919205B9
:1034D00060919305709194052AE030E087E59CE0C7
:1034E0000E94D74E8091C00085FFFCCF8AE0809378
:1034F000C6005CDE47C08091950590919605A0912D
:103500009705B09198058093910590939205A093AB
:103510009305B09394053BC06AE270E0C2010E943B
:103520007379892BA1F1EEEAF7E08491882341F0C9
:103530009091C00095FFFCCF8093C6003196F5CFE7
:10354000E3E1F4E08491882341F09091C00095FF7D
:10355000FCCF8093C6003196F5CF409191055091F4
:10356000920560919305709194052AE030E087E51B
:103570009CE00E94D74E8091C00085FFFCCF8AE07E
:103580008093C600109200041092FF03D6C1809170
:10359000040490910504989E5001999EB00C11244A
:1035A000F501E45FFB4F2F0167E470E0CF010E945B
:1035B0007379009709F444C09093FD038093FC0352
:1035C000841995098A0D9B1D60E070E0835F9B4F15
:1035D0000E9491760E94C8726430710588F58091CE
:1035E000EA03811118C08091EE05811129C0F6010E
:1035F0008491E0E1F4E0882349F09091C00095FFC8
:10360000FCCF8093C60031968491F5CF8091C000A5
:1036100085FFFCCF13C0F7018491E8E9F3E088232C
:1036200049F09091C00095FFFCCF8093C600319681
:103630008491F5CF8091C00085FFFCCF8092C600B9
:1036400080910404909105040196B8010E940376CC
:1036500090930504809304048091020490910304E4
:103660000196909303048093020410920004109238
:10367000FF03F1CD8B3311F47092FE039091FE03A2
:103680009111E9CD4091040450910504B9016F5F97
:103690007F4F709300046093FF03949EF001959E0A
:1036A000F00D1124E20FF31FE45FFB4F8083D3CDB5
:1036B0001092FE0342C18091EF05882309F43DC1B9
:1036C0008091FF0390910004892B09F036C1A0E698
:1036D0009A2E88248394B4E02B2E312C18EEC12E20
:1036E00013E0D12EE12CF12C0CE3402E512C612C57
:1036F000712C83E9A82E82E0B82E8E010F5F1F4F38
:103700004091E4065091E5066091E6067091E70667
:103710008091DC069091DD06A091DE06B091DF0677
:10372000481759076A077B0708F007C18091020410
:103730009091030404970CF000C18091C906909108
:10374000CA06A091CB06B091CC068093E406909374
:10375000E506A093E606B093E70681EC96E00E94AA
:10376000370D482F809301048A30A1F04D3091F03D
:103770004A3321F42091FE03222361F02091FF03BC
:10378000309100042F3531052CF48F3FFFEF9F0758
:1037900009F0B5C04091E4065091E5066091E60657
:1037A0007091E7068091DC069091DD06A091DE061F
:1037B000B091DF06481759076A077B0708F46CC009
:1037C000E5E8F3E08491882341F09091C00095FFF3
:1037D000FCCF8093C6003196F5CF8091C00085FF65
:1037E000FCCFFAE0F093C6000E94B16F6093EC0347
:1037F0007093ED038093EE039093EF032091F00319
:103800003091F1034091F2035091F303621B730B6B
:10381000840B950BA70196010E941676CA01B90187
:10382000A30192010E9416767F936F933F932F938B
:10383000BF92AF921F930F930E94BC79E8EAF7E022
:1038400084910FB6F894DEBF0FBECDBF882349F038
:103850009091C00095FFFCCF8093C6003196849173
:10386000F5CFF8018191882339F09091C00095FF40
:10387000FCCF8093C600F6CF8091C00085FFFCCFBF
:103880003AE03093C6008EEE95E00E944A4D61E02A
:103890008EEE95E00E94424C2091FF03309100048F
:1038A0002115310509F404CF809104049091050499
:1038B000989EF001999EF00D1124E20FF31FE45F32
:1038C000FB4F1082FC01E85FFB4F808220910204D5
:1038D000309103042F5F3F4F309303042093020481
:1038E0000196B1010E94037690930504809304042D
:1038F0001092FE03109200041092FF0301CF4B338D
:1039000011F48092FE034091FE034111F9CE4091E3
:10391000040450910504B9016F5F7F4F7093000458
:103920006093FF03949EF001959EF00D1124E20F29
:10393000F31FE45FFB4F8083E3CE6E960FB6F894DF
:10394000DEBF0FBECDBFDF91CF911F910F91FF90D2
:10395000EF90DF90CF90BF90AF909F908F907F902F
:103960006F905F904F903F902F9008958F929F920D
:10397000AF92BF92CF92DF92EF92FF920F931F937D
:10398000CF93DF935DE7E52E53E0F52E07ED15E0CD
:10399000CDEAD5E06AEEC62E65E0D62EF70181911C
:1039A0007F01C0DB882311F1A9DB4B015C01F6012B
:1039B0008081811103C060918C0501C061E070E0DD
:1039C00080E090E00E94FB72F80120813181428109
:1039D00053810E942E759B01AC01C501B4010E9468
:1039E0008071688379838A839B8309C0F801808111
:1039F0009181A281B38188839983AA83BB830C5F61
:103A00001F4F2496FFEFCF1ADF0A81E8E81683E004
:103A1000F80621F686E486DB8823D1F06FDB6B01A4
:103A20007C0160939D0570939E0580939F05909304
:103A3000A00520E030E0A9010E945C74181644F44F
:103A4000C0920402D0920502E0920602F0920702B0
:103A5000DF91CF911F910F91FF90EF90DF90CF906A
:103A6000BF90AF909F908F90089580DF89E45ADBDC
:103A7000882351F043DB6093A1057093A2058093E6
:103A8000A3059093A40508C01092A1051092A20569
:103A90001092A3051092A4058AE444DB882351F018
:103AA0002DDB6093A5057093A6058093A7059093E1
:103AB000A80508951092A5051092A6051092A705D5
:103AC0001092A8050895CF92DF92EF92FF92CF93C4
:103AD000DF93EC01C090BF05D090C005E090C10518
:103AE000F090C205A7019601688179818A819B8146
:103AF0000E94597287FF04C0C882D982EA82FB8281
:103B0000C090C305D090C405E090C505F090C605EF
:103B1000A70196016C817D818E819F810E945972DF
:103B200087FF04C0CC82DD82EE82FF82C090C70591
:103B3000D090C805E090C905F090CA05A70196018C
:103B4000688579858A859B850E94597287FF04C0A4
:103B5000C886D986EA86FB86C0900902D0900A0200
:103B6000E0900B02F0900C02A70196016881798128
:103B70008A819B810E945C74181624F4C882D982C1
:103B8000EA82FB82C0900D02D0900E02E0900F02FC
:103B9000F0901002A70196016C817D818E819F813A
:103BA0000E945C74181624F4CC82DD82EE82FF82BF
:103BB000C0901102D0901202E0901302F090140213
:103BC000A7019601688579858A859B850E945C742A
:103BD000181624F4C886D986EA86FB86DF91CF9131
:103BE000FF90EF90DF90CF900895CF92DF92EF9209
:103BF000FF920F931F938DEA95E065DF0E94B16FEE
:103C00006093F8037093F9038093FA039093FB0396
:103C10002091AD053091AE054091AF055091B005B2
:103C20006091D7057091D8058091D9059091DA05FA
:103C30000E945972811179C02091B1053091B2056D
:103C40004091B3055091B4056091DB057091DC059E
:103C50008091DD059091DE050E945972811165C049
:103C600020E030E040E752E46091040270910502E8
:103C700080910602909107020E946072EEEBCE2EB8
:103C8000E5E0DE2E7B018C0129EB35E045EB55E0CC
:103C900061EB75E08DEA95E00E94253B8091AD05D2
:103CA0009091AE05A091AF05B091B0058093D70576
:103CB0009093D805A093D905B093DA058091B1050A
:103CC0009091B205A091B305B091B4058093DB0546
:103CD0009093DC05A093DD05B093DE058091B505DA
:103CE0009091B605A091B705B091B8058093DF0516
:103CF0009093E005A093E105B093E2058091B905AA
:103D00009091BA05A091BB05B091BC058093E305E5
:103D10009093E405A093E505B093E6051F910F91FC
:103D2000FF90EF90DF90CF9008956091170270910F
:103D30001802882777FD8095982F0E94FB722091AA
:103D400004023091050240910602509107020E9440
:103D50002E7520E030E040E752E40E94607220E0DF
:103D600030E048EC52E488CFAF92BF92CF92DF921E
:103D7000EF92FF920F931F93CF93DF93D82F209151
:103D8000A5053091A6054091A7055091A805609121
:103D9000A1057091A2058091A3059091A4050E94B0
:103DA0006974C62F172F082FF92E60911702709192
:103DB0001802882777FD8095982F0E94FB7220912A
:103DC00004023091050240910602509107020E94C0
:103DD0002E7520E030E040E752E40E94607220E05F
:103DE00030E048EC52E40E9460722091BE052F93AF
:103DF000DF93FF920F931F93CF935B016C01F2E06F
:103E0000EF2E01E020E041EA55E06DEA75E087ED34
:103E100095E00E94B46B8091AD059091AE05A091A4
:103E2000AF05B091B0058093D7059093D805A093C6
:103E3000D905B093DA058091B1059091B205A091B2
:103E4000B305B091B4058093DB059093DC05A09396
:103E5000DD05B093DE058091B5059091B605A09182
:103E6000B705B091B8058093DF059093E005A09366
:103E7000E105B093E2058091B9059091BA05A09152
:103E8000BB05B091BC058093E3059093E405A09336
:103E9000E505B093E6050E94B16F6093F803709357
:103EA000F9038093FA039093FB030F900F900F9008
:103EB0000F900F900F90DF91CF911F910F91FF9076
:103EC000EF90DF90CF90BF90AF900895F8940E944C
:103ED0006D54179A169A159A149A60E084E00E941D
:103EE000B570EEEAF7E08491882341F09091C0002C
:103EF00095FFFCCF8093C6003196F5CFECE0F2E061
:103F00008491882341F09091C00095FFFCCF80936D
:103F1000C6003196F5CF8091C00085FFFCCF8AE0C6
:103F20008093C600FFCFCF92DF92EF92FF920F9364
:103F30001F930E94B16F0091F4031091F50320913B
:103F4000F6033091F703C090F803D090F903E090A6
:103F5000FA03F090FB036C197D098E099F0906177F
:103F600017072807390728F4012B022B032B09F028
:103F7000ADDF8091000290910102A0910202B09108
:103F80000302892B8A2B8B2B09F10E94B16F0091C0
:103F9000F8031091F9032091FA033091FB03601BA1
:103FA000710B820B930B0091000210910102209182
:103FB000020230910302061717072807390730F469
:103FC0009091010780910007981741F01F910F9180
:103FD000FF90EF90DF90CF900C94DC3A179A169AEE
:103FE000159A149AF3CF0E946D548091EA038111BF
:103FF00034C081E08093EA0380919105909192050D
:10400000A0919305B091940580938D0590938E05B2
:10401000A0938F05B0939005EEEAF7E08491882392
:1040200041F09091C00095FFFCCF8093C60031967F
:10403000F5CFE4E9F1E08491882341F09091C0004C
:1040400095FFFCCF8093C6003196F5CF8091C000DC
:1040500085FFFCCF8AE08093C60008958091EA0333
:104060000895EF92FF920F931F93CF93DF938C01EC
:104070007B01C0E0D0E0F70161917F01F801808110
:1040800091819C012F5F3F4F318320830E94E07B11
:104090002196C430D10579F784E090E0DF91CF918B
:1040A0001F910F91FF90EF900895EF92FF920F9361
:1040B0001F93CF93DF938C017B01C0E0D0E0F70129
:1040C00061917F01F801808191819C012F5F3F4FB9
:1040D000318320830E94E07B2196C031D10579F79E
:1040E00080E190E0DF91CF911F910F91FF90EF90D1
:1040F0000895EF92FF920F931F93CF93DF938C015C
:104100007B01C0E0D0E0F70161917F01F80180817F
:1041100091819C012F5F3F4F318320830E94E07B80
:104120002196C430D10579F784E090E0DF91CF91FA
:104130001F910F91FF90EF9008950F931F93CF93CE
:10414000DF93EC018B01FB016081888199819C01E7
:104150002F5F3F4F398328830E94E07BF801618104
:10416000888199819C012F5F3F4F398328830E946A
:10417000E07B82E090E0DF91CF911F910F91089555
:104180000F931F93CF93DF93CDB7DEB72A970FB668
:10419000F894DEBF0FBECDBF80E390E3A0E3B0E0B4
:1041A0008D839E83AF83B88784E690E09A87898762
:1041B000BE016B5F7F4FCE01099653DF63E37CE066
:1041C000CE01099672DF63E47CE0CE0109966DDFD3
:1041D00003E21CE0F80161918F0189859A859C01B9
:1041E0002F5F3F4F3A8729870E94E07BFCE0033333
:1041F0001F0781F76BE17CE0CE0109967ADF67E16A
:104200007CE0CE01099675DF6FE17CE0CE01099676
:1042100070DF67E07CE0CE0109966BDF03E51CE010
:10422000F80161918F0189859A859C012F5F3F4F2D
:104230003A8729870E94E07BFCE007351F0781F75A
:1042400063E17CE0CE01099654DF6FE07CE0CE01B3
:1042500009964FDF6BE07CE0CE0109964ADF0BEC5C
:1042600015E0F80161918F0189859A859C012F5F86
:104270003F4F3A8729870E94E07BF5E0073D1F0703
:1042800081F769EF76E0CE01099657DF67EF76E0B8
:10429000CE01099652DF65EF76E0CE0109964DDF3B
:1042A00063EF76E0CE01099648DF61EF76E0CE015C
:1042B000099643DF6FEE76E0CE0109963EDF66E4B5
:1042C00072E0CE01099615DF62E472E0CE01099634
:1042D00010DF6EE372E0CE0109960BDF86E590E316
:1042E000A7E3B0E089839A83AB83BC8384E690E044
:1042F0009A878987BE016F5F7F4FCE010996B1DE35
:10430000E8EAF7E08491882341F09091C00095FF9E
:10431000FCCF8093C6003196F5CFE8E3F2E08491BC
:10432000882341F09091C00095FFFCCF8093C60098
:104330003196F5CF8091C00085FFFCCF8AE0809355
:10434000C6002A960FB6F894DEBF0FBECDBFDF9130
:10435000CF911F910F910895EF92FF920F931F93AA
:10436000CF93DF938C017B01C0E0D0E0F801808126
:1043700091819C012F5F3F4F318320830E94D87B26
:10438000F70181937F012196C031D10579F780E152
:1043900090E0DF91CF911F910F91FF90EF900895E2
:1043A000EF92FF920F931F93CF93DF938C017B01CA
:1043B000C0E0D0E0F801808191819C012F5F3F4FE8
:1043C000318320830E94D87BF70181937F0121965E
:1043D000C430D10579F784E090E0DF91CF911F914F
:1043E0000F91FF90EF9008950F931F93CF93DF935A
:1043F000EC018B01888199819C012F5F3F4F3983AC
:1044000028830E94D87BF8018083888199819C0150
:104410002F5F3F4F398328830E94D87BF801818327
:1044200082E090E0DF91CF911F910F910895AF92BC
:10443000BF92CF92DF92EF92FF920F931F93CF9391
:10444000DF93CDB7DEB7EC970FB6F894DEBF0FBEA3
:10445000CDBFD82E24E630E03AAF29AF46E550E391
:1044600067E370E049AB5AAB6BAB7CAB7E0185E395
:10447000E80EF11C8E01075C1F4FB70189AD9AADA4
:104480009C012F5F3F4F3AAF29AF6BAF7CAF0E94CB
:10449000D87BF70181937F016BAD7CADE017F1070D
:1044A00069F7D110AFC043E050E0CE01C1960E9441
:1044B0008579892B09F0A6C063E37CE0C8014CDF55
:1044C00063E47CE0C80148DF23E2E22E2CE0F22E18
:1044D00089AD9AAD9C012F5F3F4F3AAF29AF0E9443
:1044E000D87BF70181937F01F3E3EF16FCE0FF0631
:1044F00079F76BE17CE0C80153DF67E17CE0C8013C
:104500004FDF6FE17CE0C8014BDF67E07CE0C80172
:1045100047DF93E5E92E9CE0F92E89AD9AAD9C0129
:104520002F5F3F4F3AAF29AF0E94D87BF7018193AD
:104530007F01F7E5EF16FCE0FF0679F763E17CE029
:10454000C8012EDF6FE07CE0C8012ADF6BE07CE071
:10455000C80126DF8BECE82E85E0F82E89AD9AADF8
:104560009C012F5F3F4F3AAF29AF0E94D87BF701E4
:1045700081937F01F7EDEF16F5E0FF0679F769EF1C
:1045800076E0C80131DF67EF76E0C8012DDF65EF27
:1045900076E0C80129DF63EF76E0C80125DF61EF2F
:1045A00076E0C80121DF6FEE76E0C8011DDF66E42A
:1045B00072E0C801F5DE62E472E0C801F1DE6EE38C
:1045C00072E0C801EDDEE8EAF7E08491882341F06B
:1045D0009091C00095FFFCCF8093C6003196F5CF37
:1045E000E8E7F6E08491882341F09091C00095FFC0
:1045F000FCCF8093C6003196F5CF8091C00085FF37
:10460000FCCFE3C080E1EFE4F2E0DE01919601909F
:104610000D928A95E1F780E1EFE5F2E0DE01519637
:1046200001900D928A95E1F780E1EFE6F2E0DE017C
:10463000119601900D928A95E1F76E0181E2C80E04
:10464000D11CA3E3EA2EACE0FA2E8E010F5E1F4FC1
:1046500063E47CE0AE014F5F5F4FB3E2AB2EBCE0A2
:10466000BB2E24E030E0F60181919191A191B191AE
:104670006F01F70181939193A193B1937F01F801A9
:1046800081919191A191B1918F01FB0181939193BE
:10469000A193B193BF01FA0181919191A191B1913F
:1046A000AF01F50181939193A193B1935F012150E3
:1046B000310921153105B9F680E090E8ABE3B5E4A6
:1046C00080931B0C90931C0CA0931D0CB0931E0C9C
:1046D0008093170C9093180CA093190CB0931A0C9C
:1046E00010921F0C1092200C1092210C1092220C90
:1046F00080E29EE4A0E0B0E08093530C9093540CD1
:10470000A093550CB093560C1092070C1092080C05
:104710001092090C10920A0C80E090E0A0EAB1E43B
:104720008093130C9093140CA093150CB093160C5B
:104730008DEC9CECACECBEE380930F0C9093100CD2
:10474000A093110CB093120C80E090E0A0EAB0E4CA
:1047500080930B0C90930C0CA0930D0CB0930E0C4B
:104760001092D3051092D4051092D5051092D6055B
:104770001092CF051092D0051092D1051092D2055B
:104780001092CB051092CC051092CD051092CE055B
:10479000E8EAF7E08491882341F09091C00095FF0A
:1047A000FCCF8093C6003196F5CFE2EAF2E081912A
:1047B000882339F09091C00095FFFCCF8093C6000C
:1047C000F6CF8091C00085FFFCCF8AE08093C600C1
:1047D0000E942D15EC960FB6F894DEBF0FBECDBF2C
:1047E000DF91CF911F910F91FF90EF90DF90CF90CD
:1047F000BF90AF900895CF92DF92EF92FF920F9308
:104800001F93CF93DF9300D01F92CDB7DEB740E068
:1048100052EC61E070E087E59CE00E94E64DE6E541
:10482000F7E08491882341F09091C00095FFFCCF80
:104830008093C6003196F5CF8091C00085FFFCCFF4
:104840008AE08093C60088EA97E0FC012491222345
:1048500041F03091C00035FFFCCF2093C600319667
:10486000F5CF24B720FF14C0EEE4F7E034913323F2
:1048700041F04091C00045FFFCCF3093C600319617
:10488000F5CF3091C00035FFFCCF3AE03093C60041
:1048900021FF14C0EEE3F7E03491332341F040915F
:1048A000C00045FFFCCF3093C6003196F5CF309164
:1048B000C00035FFFCCF3AE03093C60022FF14C0A1
:1048C000EDE2F7E03491332341F04091C00045FF21
:1048D000FCCF3093C6003196F5CF3091C00035FF44
:1048E000FCCF3AE03093C60023FF14C0EDE1F7E0BF
:1048F0003491332341F04091C00045FFFCCF309309
:10490000C6003196F5CF3091C00035FFFCCF3AE0BC
:104910003093C60025FF14C0EDE0F7E02491222378
:1049200041F03091C00035FFFCCF2093C600319696
:10493000F5CF2091C00025FFFCCF2AE02093C600D0
:1049400014BEE5E0F7E02491222341F03091C0004D
:1049500035FFFCCF2093C6003196F5CFEFEFF6E0A0
:104960002491222341F03091C00035FFFCCF2093E9
:10497000C6003196F5CF2091C00025FFFCCF2AE07C
:104980002093C600FC012491E8EAF7E0222349F0D5
:104990003091C00035FFFCCF2093C60031962491A2
:1049A000F5CFEFEEF6E02491222341F03091C000E4
:1049B00035FFFCCF2093C6003196F5CFE4EEF6E04C
:1049C0002491222341F03091C00035FFFCCF209389
:1049D000C6003196F5CFE8EDF6E02491222341F0B0
:1049E0003091C00035FFFCCF2093C6003196F5CF43
:1049F000E0EDF6E02491222341F03091C00035FF34
:104A0000FCCF2093C6003196F5CF2091C00025FF42
:104A1000FCCF2AE02093C600E5ECF6E024912223A7
:104A200041F03091C00035FFFCCF2093C600319695
:104A3000F5CFE9EBF6E02491222341F03091C0005C
:104A400035FFFCCF2093C6003196F5CF2091C000F2
:104A500025FFFCCF2AE02093C600FC018491E8EA00
:104A6000F7E0882349F09091C00095FFFCCF809338
:104A7000C60031968491F5CFEAEAF6E08491882366
:104A800041F09091C00095FFFCCF8093C600319615
:104A9000F5CF0E94EE174AE050E0BC0187E59CE0AC
:104AA0000E94FA4EE3E9F6E08491882341F0909168
:104AB000C00095FFFCCF8093C6003196F5CF4AE049
:104AC00050E060ED74E087E59CE00E94FA4E809132
:104AD000C00085FFFCCF8AE08093C60010920804D6
:104AE0001092090410920A0410920B0480E09FDCDB
:104AF00033E2C32E3CE0D32E43E3E42E4CE0F42E0D
:104B000007EF1BE0F60161917191819191916F0125
:104B1000F70121913191419151917F0129833A838C
:104B20004B835C830E94F97229813A814B815C81BD
:104B30000E942E750E94CD72F8016193719381934A
:104B400091938F01F3E3CF16FCE0DF06D9F60E94C4
:104B500005540E9486390F900F900F900F90DF91AF
:104B6000CF911F910F91FF90EF90DF90CF900C9419
:104B7000F2652F923F924F925F926F927F928F9247
:104B80009F92AF92BF92CF92DF92EF92FF920F93DC
:104B90001F93CF93DF93CDB7DEB7A0970FB6F894EE
:104BA000DEBF0FBECDBF87E40E949218882309F4B0
:104BB0000BC20E947E180E94C87264307105D1F148
:104BC00044F46230710521F15CF577FF17C00C9455
:104BD00084336A35710509F4A3C134F46C3171056D
:104BE00009F469C00C9484336B35710509F49CC1D8
:104BF0006C35710509F49DC10C9484338091EA03EE
:104C0000811106C00E94B61C0E94F51D0C94163539
:104C10008091EA03811104C00E94351D81E007C024
:104C20008091EA03811106C00E94351D80E09CD866
:104C30000C94163580E50E949218882339F00E9462
:104C40007E180E94CD724B015C0103C0812C912C17
:104C5000540183E50E949218882361F00E947E1817
:104C600020E030E04AE754E40E942E750E94CD72A5
:104C70004B015C010E9451640E94B16F6B017C0189
:104C8000C80CD91CEA1CFB1C0E94B16F6093F8038E
:104C90007093F9038093FA039093FB030E94B16F22
:104CA0006C157D058E059F0510F00C9484330E94D1
:104CB000B65139D9F3CF8091040290910502A091A9
:104CC0000602B09107028093990590939A05A093EC
:104CD0009B05B0939C0580911702909118029093C8
:104CE000E9058093E80584E690E0909318028093AC
:104CF00017020E94B16F6093F8037093F9038093D9
:104D0000FA039093FB0381E00E940B5D8091D7052D
:104D10009091D805A091D905B091DA058093AD05A1
:104D20009093AE05A093AF05B093B0058091DB05DD
:104D30009091DC05A091DD05B091DE058093B10571
:104D40009093B205A093B305B093B4058091DF05AD
:104D50009091E005A091E105B091E2058093B50541
:104D60009093B605A093B705B093B8058091E3057D
:104D70009091E405A091E505B091E6058093B90511
:104D80009093BA05A093BB05B093BC0510920402A2
:104D900010920502109206021092070288E50E9406
:104DA0009218882311F090E00AC089E50E949218B9
:104DB0008111F9CF8AE50E94921891E0982790938B
:104DC000080291110C94873388E50E949218811192
:104DD0000C9487338091080281110C948D3389E5FE
:104DE0000E94921881110C948D33809108028111D8
:104DF0000C9493338AE50E94921881110C9493339A
:104E000088E50E9492188823D1F00E948718672BAA
:104E1000682B692BA1F00E947E182091CB05309160
:104E2000CC054091CD055091CE050E9480716093D4
:104E3000D7057093D8058093D9059093DA0589E555
:104E40000E9492188823D1F00E948718672B682B44
:104E5000692BA1F00E947E182091CF053091D005DA
:104E60004091D1055091D2050E9480716093DB057D
:104E70007093DC058093DD059093DE058AE50E9442
:104E800092188823D1F00E948718672B682B692B12
:104E9000A1F00E947E182091D3053091D405409155
:104EA000D5055091D6050E9480716093DF057093FF
:104EB000E0058093E1059093E20523EE35E04FEDA8
:104EC00055E06BED75E087ED95E00E949C4480E035
:104ED0000E940B5D8091990590919A05A0919B0588
:104EE000B0919C058093040290930502A093060262
:104EF000B09307028091E8059091E905909318021C
:104F0000809317020E94B16F6093F8037093F903C6
:104F10008093FA039093FB030E94045D0C94843306
:104F200010928C050C94843381E080938C050C9452
:104F3000843385E40E949218811102C00E9451645A
:104F40000DE7C02E03E0D02E8BECE82E85E0F82E86
:104F500007ED15E0B12CF60181916F010E949218C6
:104F6000882339F1F3E0BF120CC00E947E18F801CB
:104F7000608371838283938383EE95E00E94414531
:104F800018C00E947E18F70120813181428153812F
:104F90000E948071F801608371838283938323EE82
:104FA00035E04FED55E06BED75E087ED95E00E9443
:104FB0009C44B394F4E0EF0EF11C0C5F1F4F24E00F
:104FC000B212C9CF0C9484338DE40E9492188823C6
:104FD00011F40C94D7320E947E180E94C872623776
:104FE000710509F45BC60CF085C06F31710509F4D9
:104FF00009C20CF043C06731710509F459C1F4F4DA
:105000006431710509F423C154F46131710509F467
:1050100018C16231710509F46AC50C948433653195
:10502000710509F43FC16631710511F00C948433A8
:105030008EEE95E00E9459480C9484336A317105D4
:1050400009F459C17CF46831710509F444C169312E
:10505000710511F00C9484338EEE95E00E94644843
:105060000C9484336C31710509F459C10CF451C1AD
:105070006E31710509F488C10C948433653571056E
:1050800009F467C5E4F46135710509F42AC56CF4C7
:105090006A32710509F44CC26035710511F00C9447
:1050A00084339D9AA5980C9484336335710509F473
:1050B0001AC50CF01CC51092ED050C9484336936AA
:1050C000710509F4C9C254F46C35710509F457C56A
:1050D0006836710509F44AC20C9484336B36710545
:1050E00009F4FCC40CF4D3C46D36710509F486C30D
:1050F0000C9484336D3D710511F40C94DF300CF089
:1051000042C06E3B710509F422C4DCF468377105B6
:1051100009F4A0C664F46337710509F4B1C56737B3
:10512000710511F00C948433EFE7F2E0A0C6693703
:10513000710509F491C66C38710509F479C20C94B3
:1051400084336C3C710509F48EC784F4693C7105A5
:1051500009F43CC76B3C710511F00C9484330DE7E6
:1051600013E0E3E4EE2EECE0FE2E6EC76E3C71051C
:1051700009F4F7C70CF497C76C3D710511F40C9452
:10518000CD300C948433643F31E0730711F40C94F8
:10519000DB3154F56F3291E0790711F40C94C93189
:1051A00084F46D32F1E07F0711F40C94EE306E322E
:1051B000714011F00C94843381E00E945E450C94A0
:1051C00084336F3531E0730711F40C946632603923
:1051D00081E0780711F40C94D8316E35714011F0EC
:1051E0000C9484330C943032673FE1E07E0711F475
:1051F0000C94E23174F4653F21E0720711F40C94D1
:10520000DE31663F714011F00C94843381E00C94E0
:10521000DF316C3883E0780711F40C941532673E67
:1052200093E0790711F40C94C2326B38734011F09B
:105230000C9484336DE7E62E63E0F62ED12C0C94AB
:10524000E93117981698159814980C948433E5E76B
:10525000F3E08491882341F09091C00095FFFCCF4A
:105260008093C6003196F5CF8091C00085FFFCCFBA
:105270008AE08093C6008EEE95E00E943D47E7E607
:10528000F3E08491882341F09091C00095FFFCCF1A
:105290008093C6003196F5CF8091C00085FFFCCF8A
:1052A0000C9481338EEE95E00E9494470C948433E5
:1052B0000091FC031091FD030C5F1F4F6AE270E048
:1052C000C8010E947379009719F0FC013197108290
:1052D00041E0B80153C08EEE95E00E945D480E9407
:1052E000B16F6093F0037093F1038093F203909396
:1052F000F3030C9484338091F005882311F40C940B
:10530000843383E50E94921881110C9499330C9494
:1053100084338EEE95E00E94804B0C948433809110
:10532000FC039091FD036AE270E004960E94737999
:105330008C010097E1F0209106043091070440E6CB
:10534000429FC001439F900D11246EE470E0845F82
:105350009B4F0E94737960E270E00E94737901961E
:105360009093FD038093FC03F801319710826091C4
:10537000FC037091FD036C5F7F4F40E08EEE95E083
:105380000E9469480C9484338091F005882311F4BD
:105390000C9484338EEE95E00E94364D8091FC0390
:1053A0009091FD036AE270E004960E9473798C018B
:1053B0000097E1F0209106043091070440E6429FF7
:1053C000C001439F900D11246EE470E0845F9B4FF9
:1053D0000E94737960E270E00E9473790196909365
:1053E000FD038093FC03F801319710826091FC0368
:1053F0007091FD036C5F7F4F8EEE95E00E94474AEF
:105400000C9484330E94B16F6093EC037093ED03AE
:105410008093EE039093EF030091F0031091F1035A
:105420002091F2033091F303601B710B820B930BFD
:1054300028EE33E040E050E00E941676CA01B90140
:105440002CE330E040E050E00E9416767F936F93AB
:105450003F932F9383E992E09F938F93CE01019620
:105460009F938F930E94BC79E8EAF7E084910FB68E
:10547000F894DEBF0FBECDBF882349F09091C000E5
:1054800095FFFCCF8093C60031968491F5CFFE0145
:1054900031968191882339F09091C00095FFFCCF1F
:1054A0008093C600F6CF8091C00085FFFCCF8AE0D4
:1054B0008093C6008091D20B882311F40C9484331E
:1054C0001092D20B6091BE05E62FF0E0EE0FFF1FA9
:1054D000EC5DF24F808191810E94E25020912D027B
:1054E00030912E0240912F02509130020E945C7444
:1054F000181614F00C9484336091BE05062F10E04A
:1055000080E090E00E94EE4FF801EE0FFF1FEC5D8F
:10551000F24F91838083F801EE0FFF1FEE0FFF1F04
:10552000E65EF24F10821182128213820C94843351
:1055300083E50E949218882311F40C9484330E940E
:105540007E186B017C0180E50E949218882311F47B
:105550000C948433C701B6010E94C8726F3F710575
:1055600009F010F40C94AA330C9484338091BE0596
:105570008093EB0384E50E949218882379F10E94BE
:105580007E180E94CD726093EB03662339F1E8EA3E
:10559000F7E08491882341F09091C00095FFFCCF03
:1055A0008093C6003196F5CFE0ECF2E0819188233C
:1055B00039F09091C00095FFFCCF8093C600F6CFE4
:1055C00040E050E06091EB0387E59CE00E94314FA2
:1055D0008091C00085FFFCCF0C94813383E50E944D
:1055E0009218882309F1B090EB030E947E186B019A
:1055F0007C010B2D10E00E94C872DC01CB016B2DE9
:105600000E94EE4FF801EE0FFF1FEC5DF24F918309
:105610008083F801EE0FFF1FEE0FFF1FE65EF24FD3
:10562000C082D182E282F3820E946C540C94843353
:1056300083E50E949218882311F40C9484330E940D
:105640007E180E94C872CB010E9480509093230D57
:105650008093220D0C9484338091BE058093EB03DC
:1056600084E50E949218882379F10E947E180E9496
:10567000CD726093EB03662339F1E8EAF7E0849199
:10568000882341F09091C00095FFFCCF8093C60025
:105690003196F5CFE7EDF2E08191882339F09091D2
:1056A000C00095FFFCCF8093C600F6CF40E050E0ED
:1056B0006091EB0387E59CE00E94314F8091C00030
:1056C00085FFFCCF0C948133E1E6F3E084918823DD
:1056D00041F09091C00095FFFCCF8093C6003196B9
:1056E000F5CF6091EB03E62FF0E0EE0FFF1FE05ED9
:1056F000F24F808191810E94E250AB01BC0121E018
:1057000030E087E59CE00E94D04FEEE5F3E0849125
:10571000882341F09091C00095FFFCCF8093C60094
:105720003196F5CF6091EB03E62FF0E0EE0FFF1F0F
:10573000EC5DF24F808191810E94E250AB01BC018F
:1057400021E030E087E59CE00E94D04FEAE5F3E0FD
:105750008491882341F09091C00095FFFCCF809305
:10576000C6003196F5CF80911E0D90911F0D0E94BD
:105770006053AB01BC0121E030E087E59CE00E9472
:10578000D04FE7E5F3E08491882341F09091C00089
:1057900095FFFCCF8093C6003196F5CF8091220D06
:1057A0009091230D0E946053AB01BC0121E030E0D9
:1057B00087E59CE00E94D04FE3E5F3E084918823E5
:1057C00041F09091C00095FFFCCF8093C6003196C8
:1057D000F5CF8091EB0390E00E94E84F4AE050E063
:1057E000BC0187E59CE00E94FA4E8091C00085FFD5
:1057F000FCCF8AE08093C6000C9416358091BE05DC
:105800008093EB0384E50E949218882371F10E9433
:105810007E180E94CD726093EB03662331F1E8EAB3
:10582000F7E08491882341F09091C00095FFFCCF70
:105830008093C6003196F5CFEEEEF2E08191882399
:1058400039F09091C00095FFFCCF8093C600F6CF51
:1058500040E050E06091EB0387E59CE00E94314F0F
:105860008091C00085FFFCCF4CC71092D20B83E51E
:105870000E949218882309F1B090EB030E947E18D1
:105880006B017C010B2D10E00E94C872DC01CB0182
:105890006B2D0E94EE4FF801EE0FFF1FEC5DF24FF3
:1058A00091838083F801EE0FFF1FEE0FFF1FE65E6E
:1058B000F24FC082D182E282F38283E50E94921885
:1058C000882351F00E947E1860932D0270932E025F
:1058D00080932F029093300282E40E9492188823D2
:1058E00051F00E947E1860933102709332028093CF
:1058F00033029093340286E40E949218882369F060
:105900000E947E186093290270932A0280932B02D2
:1059100090932C0281E08093D20B0E946C540E94E1
:10592000B16F4B015C018091EB0390E0880F991FF0
:10593000FC01EC5DF24F00811181FC01E05EF24F51
:1059400020803180CC24CA94DC2C760179C783E591
:105950000E949218882359F00E947E180E94C872F3
:10596000CB010E9480509093230D8093220D0E94C2
:10597000B16F4B015C0105E413E091E4E92E93E083
:10598000F92E2DE3C22E23E0D22E3AE0732E209181
:10599000220D3091230D80911E0D90911F0D8217C5
:1059A000930714F00C94F2340E94B16F68197909CE
:1059B0008A099B09693E73408105910508F462C01C
:1059C0006091BE05E62FF0E0EE0FFF1FE05EF24FA4
:1059D000808191810E94E250AB01BC01F801849169
:1059E000E5E4F3E0882349F09091C00095FFFCCFF7
:1059F0008093C60031968491F5CF22E030E087E5B0
:105A00009CE00E94D04FF7018491E1E4F3E0882309
:105A100049F09091C00095FFFCCF8093C60031966D
:105A20008491F5CF6091BE0570E04AE050E087E5D3
:105A30009CE00E94FA4EF6018491EDE3F3E08823A6
:105A400049F09091C00095FFFCCF8093C60031963D
:105A50008491F5CF80911E0D90911F0D0E9460538F
:105A6000AB01BC0121E030E087E59CE00E94D04F13
:105A70008091C00085FFFCCF7092C6000E94B16F7C
:105A80004B015C010E94B6510E94931F80CF83E5B9
:105A90000E9492188823F1F00E947E1820E030E0E6
:105AA000A9010E94597287FD0FC00E947E1820E054
:105AB00030E04FE753E40E945C7418163CF00E94FB
:105AC0007E180E94CD7203C060E001C06FEF60934A
:105AD000BD051AC68FEF8093BD0516C61092BD0591
:105AE00013C69D9811C681E08093ED050DC683E530
:105AF0000E949218882399F00E947E1820E030E0DE
:105B00004AE754E40E942E750E94CD726093000211
:105B1000709301028093020290930302F5C588E519
:105B20000E949218811169C789E50E94921881111B
:105B300064C78AE50E94921881115FC785E40E94BC
:105B4000921881115AC70E945164149A0E94B86435
:105B5000DBC583E50E9492180E947E1820E030E0A9
:105B60004AE754E40E942E750E94CD726093F403BC
:105B70007093F5038093F6039093F703C5C52DE763
:105B800033E038A32F8F03E31CE0A3E48A2EACE0BC
:105B90009A2EB7EFAB2EBBE0BB2E312CEF8DF8A1C8
:105BA0008191F8A3EF8F0E949218882309F45BC0BB
:105BB000F3E03F1251C00E947E186B017C0120E08F
:105BC00030E040EA51E40E94597287FF3FC0A701CC
:105BD0009601F80160817181828193810E946072D7
:105BE0002B013C019B01AC0160910B0C70910C0CE2
:105BF00080910D0C90910E0C0E942E7560930B0CF1
:105C000070930C0C80930D0C90930E0CA3019201D9
:105C1000F40160817181828193810E942E75F4016B
:105C20006083718382839383F501608171818281B6
:105C300093810E94F972A30192010E942E750E9425
:105C4000CD72F5016083718382839383F801C082F2
:105C5000D182E282F38207C00E947E18F80160833D
:105C600071838283938333940C5F1F4FF4E08F0E14
:105C7000911C24E0A20EB11C34E033128FCF44C536
:105C8000E2EAF2E08491882309F43EC59091C000D5
:105C900095FFFCCF8093C6003196F4CFEFE9F2E098
:105CA0008491882341F09091C00095FFFCCF8093B0
:105CB000C6003196F5CF4091D7055091D805609137
:105CC000D9057091DA0522E030E087E59CE00E947A
:105CD000D04FECE9F2E08491882341F09091C0002C
:105CE00095FFFCCF8093C6003196F5CF4091DB0540
:105CF0005091DC056091DD057091DE0522E030E019
:105D000087E59CE00E94D04FE9E9F2E08491882386
:105D100041F09091C00095FFFCCF8093C600319672
:105D2000F5CF4091DF055091E0056091E10570915C
:105D3000E20522E030E087E59CE00E94D04FE6E9F2
:105D4000F2E08491882341F09091C00095FFFCCF50
:105D50008093C6003196F5CF4091E3055091E4055C
:105D60006091E5057091E60522E030E087E59CE072
:105D70000E94D04FECE8F2E08491882341F09091AA
:105D8000C00095FFFCCF8093C6003196F5CF0E94EE
:105D9000AA640E94FB722091330C3091340C409124
:105DA000350C5091360C0E946072AB01BC0122E0B0
:105DB00030E087E59CE00E94D04FE9E8F2E0849172
:105DC000882341F09091C00095FFFCCF8093C600DE
:105DD0003196F5CF81E00E94AA640E94FB72209167
:105DE000370C3091380C4091390C50913A0C0E948C
:105DF0006072AB01BC0122E030E087E59CE00E94CC
:105E0000D04FE6E8F2E08491882341F09091C00001
:105E100095FFFCCF8093C6003196F5CF82E00E94BB
:105E2000AA640E94FB7220913B0C30913C0C409183
:105E30003D0C50913E0C0E946072AB01BC0122E00F
:105E400030E087E59CE00E94D04F8091C00085FF44
:105E5000FCCF57C480E001C081E00E940B5D54C4B8
:105E60009091C00095FFFCCF8093C600319684913D
:105E70008111F6CF1E9903C0EAEBF2E009C0EDEB09
:105E8000F2E006C09091C00095FFFCCF8093C60061
:105E900081918111F7CFE8E7F2E08491882341F006
:105EA0009091C00095FFFCCF8093C6003196F5CF4E
:105EB000029903C0EAEBF2E009C0EDEBF2E006C0A4
:105EC0009091C00095FFFCCF8093C6008191811115
:105ED000F7CFE1E7F2E08491882341F09091C00090
:105EE00095FFFCCF8093C6003196F5CF1D9903C076
:105EF000EAEBF2E009C0EDEBF2E006C09091C000E1
:105F000095FFFCCF8093C60081918111F7CFEAE61F
:105F1000F2E08491882341F09091C00095FFFCCF7E
:105F20008093C6003196F5CF019903C0EAEBF2E009
:105F300009C0EDEBF2E006C09091C00095FFFCCFE8
:105F40008093C60081918111F7CFE3E6F2E084915E
:105F5000882341F09091C00095FFFCCF8093C6004C
:105F60003196F5CF1C9903C0EAEBF2E009C0EDEBE6
:105F7000F2E006C09091C00095FFFCCF8093C60070
:105F800081918111F7CFECE5F2E08491882341F013
:105F90009091C00095FFFCCF8093C6003196F5CF5D
:105FA000379903C0EAEBF2E009C0EDEBF2E006C07E
:105FB0009091C00095FFFCCF8093C6008191811124
:105FC000F7CF8091C00085FFFCCF9BC3FDE7EF2E8C
:105FD000F3E0FF2E00E010E0F70181917F010E94C5
:105FE0009218882319F10E947E1898012D5D334F75
:105FF00069010E94CD72F60160837183828393836D
:106000000E947E1898012950344F6901F801ED5C17
:10601000F34F20813181428153810E942E750E946D
:10602000CD72F60160837183828393830C5F1F4F6F
:106030000031110589F668C3F4E0EF0EF11C23E08E
:106040000138120709F460C3F80181918F010E94A1
:106050009218882389F30E947E18F7016083718368
:1060600082839383E9CF83E50E949218882351F0BD
:106070000E947E1860931B0C70931C0C80931D0C67
:1060800090931E0C84E50E949218882309F43CC367
:106090000E947E186093170C7093180C8093190C53
:1060A00090931A0C31C383E50E949218882351F013
:1060B0000E947E1860931F0C7093200C8093210C1B
:1060C0009093220C84E50E949218882351F00E943C
:1060D0007E186093070C7093080C8093090C9093C2
:1060E0000A0C82E40E949218882361F00E947E18B4
:1060F0000E94CD726093530C7093540C8093550C96
:106100009093560C88E50E949218882351F00E94C3
:106110007E186093130C7093140C8093150C90935D
:10612000160C8AE50E949218882351F00E947E186E
:1061300060930F0C7093100C8093110C9093120CC1
:1061400085E40E949218882309F4DEC20E947E181A
:1061500060930B0C70930C0C80930D0C90930E0CB1
:10616000D3C20DE713E07BECE72E75E0F72EF801C4
:1061700081918F010E949218882339F00E947E1825
:10618000F7016083718382839383F4E0EF0EF11C47
:1061900023E00038120759F7B7C283E50E9492182E
:1061A000882309F4B1C20E947E180E94C8727093BD
:1061B00018026093170281E08093E705A5C283E58A
:1061C0000E949218882309F49FC20E947E180E94A0
:1061D000C872709316026093150296C280E50E9401
:1061E0009218882351F00E947E18609346027093A3
:1061F0004702809348029093490289E40E949218D2
:10620000882381F00E947E182DEB37E346E05EE3A1
:106210000E942E7560934202709343028093440261
:106220009093450284E40E949218882381F00E9492
:106230007E182DEB37E346E05EE30E9460726093C8
:106240003E0270933F02809340029093410283E4A8
:106250000E949218882351F00E947E1860933A029F
:1062600070933B0280933C0290933D020E94D14F79
:10627000E7E0F3E08191882339F09091C00095FF29
:10628000FCCF8093C600F6CFEAE0F3E0819188234B
:1062900039F09091C00095FFFCCF8093C600F6CFF7
:1062A0004091460250914702609148027091490224
:1062B00022E030E087E59CE00E94D04FEEE0F3E082
:1062C0008191882339F09091C00095FFFCCF809395
:1062D000C600F6CF2DEB37E346E05EE36091420265
:1062E0007091430280914402909145020E94607235
:1062F000AB01BC0122E030E087E59CE00E94D04F7A
:10630000E2E1F3E08191882339F09091C00095FF9C
:10631000FCCF8093C600F6CF2DEB37E346E05EE37B
:1063200060913E0270913F02809140029091410243
:106330000E942E75AB01BC0122E030E087E59CE0B5
:106340000E94D04FE6E1F3E08191882339F09091EB
:10635000C00095FFFCCF8093C600F6CF2DEB37E34E
:1063600046E05EE360913A0270913B0280913C020C
:1063700090913D020E942E75AB01BC0122E030E0FD
:1063800087E59CE00E94D04F8091C00085FFFCCF44
:10639000B8C183E50E949218882319F00E947E18E4
:1063A00004C060E070E086E193E40E94A454ACC1B4
:1063B0000E945164A9C10E94C020A6C180E00E9431
:1063C0001722A2C10E942D159FC1D394F5E0DF16BC
:1063D00079F0F70181917F010E9492188823A9F337
:1063E0000E947E180E94C8728D2D0E94F964EDCF24
:1063F00082E40E949218882339F00E947E180E943D
:10640000C87284E00E94F96483E50E949218882390
:1064100061F0F12C0E947E180E94C8728F2D0E949C
:10642000F964F39425E0F212F5CF80E50E9492180A
:10643000882329F00E947E180E94CD72162F83E5D2
:106440000E949218882329F00E947E180E94CD7223
:10645000062F602F70E0812F90E00E94E06454C10D
:1064600083E50E949218811104C00DE713E0F12C1E
:1064700010C010E00E947E180E94CD72812F0E94F1
:106480009C651F5F1530B1F7F0CFF394F5E0FF1670
:1064900079F0F80181918F010E9492188823A9F365
:1064A0000E947E180E94CD728F2D0E949C65EDCFB8
:1064B00082E40E949218882309F461C00E947E1829
:1064C0000E94CD7284E00E949C6559C083E50E94C1
:1064D0009218882309F453C00E947E180E94C87243
:1064E0006130710541F06230710509F048C00DE777
:1064F00013E0F12C25C00DE713E0F12CF801819198
:106500008F010E949218882341F00E947E180E94F9
:10651000C8724FEF8F2D0E944B65F394F5E0FF1288
:10652000EDCF82E40E949218882349F10E947E18E0
:106530000E94C8724FEF20C0F394F5E0FF1689F077
:10654000F80181918F010E9492188823A9F30E947B
:106550007E180E94C872462F6FEF8F2D0E944B65E8
:10656000EBCF82E40E949218882349F00E947E18A3
:106570000E94C872462F6FEF84E00E944B650E9414
:106580005866C2C01092EA0380918D0590918E05E5
:10659000A0918F05B09190058093910590939205FD
:1065A000A0939305B09394050E94D618ADC084E5DE
:1065B0000E949218882309F463C00E947E180E94EA
:1065C000CD726093EB03662391F1E8EAF7E08491E2
:1065D000882341F09091C00095FFFCCF8093C600C6
:1065E0003196F5CFEAE1F3E08191882339F090917B
:1065F000C00095FFFCCF8093C600F6CF40E050E08E
:106600006091EB0387E59CE00E94314FECE1F3E001
:106610008191882339F09091C00095FFFCCF809341
:10662000C600F6CF8091C00085FFFCCF6AC01092F3
:10663000BE05E8EAF7E08491882341F09091C0001C
:1066400095FFFCCF8093C6003196F5CFEDE2F3E0E5
:106650008191882339F09091C00095FFFCCF809301
:10666000C600F6CF6091BE0570E04AE050E087E5D5
:106670009CE00E94FA4E8091C00085FFFCCF41C093
:10668000E8EAF7E08491882341F09091C00095FFFB
:10669000FCCF8093C6003196F5CFEAE4F2E0849116
:1066A000882341F09091C00095FFFCCF8093C600F5
:1066B0003196F5CF809106049091070420E6289F3B
:1066C000F001299FF00D1124E45FFB4F8191882395
:1066D00039F09091C00095FFFCCF8093C600F6CFB3
:1066E000E8E4F2E08491882341F09091C00095FFA6
:1066F000FCCF8093C6003196F5CF8091C00085FF16
:10670000FCCF8AE08093C6000E94AE188FC180E063
:1067100090E00E9477130C94EA2681E090E00E94BA
:1067200077130C94F52682E090E00E9477130C9486
:1067300000270E948718AB01BC014093E4065093E8
:10674000E5066093E6067093E70681EC96E00E940A
:10675000000EDACF0E947E180E94C87220E0E22F5D
:10676000EE0FFF0BED5BFC4F808191818617970741
:1067700059F22F5FF4CF0E94B16F4B015C01C7014A
:10678000B601605F784D8F4F9F4F681979098A096C
:106790009B0928EE33E040E050E00E941676BA01F3
:1067A000A9012AE030E087E59CE00E94264F809115
:1067B000C00085FFFCCFFAE0F093C6000E94B16FE5
:1067C0004B015C010E94B6510E94931F3FEFC3161C
:1067D000D306E306F30609F099C06091EB03E62FB8
:1067E000F0E0EE0FFF1FE05EF24F808191812016F6
:1067F00031060CF0C9C00E94E2502B013C016091AF
:10680000EB03E62FF0E0EE0FFF1FEC5DF24F80810F
:1068100091810E94E25020E030E040E85FE30E9476
:106820007F719B01AC01C301B2010E945C7487FFC0
:10683000CAC08FEFC816D806E806F80609F099C056
:106840000E94B16F681979098A099B09693E7340F2
:106850008105910508F4B6CFE0E5F3E08491882343
:1068600041F09091C00095FFFCCF8093C600319617
:10687000F5CF6091EB03E62FF0E0EE0FFF1FE05E37
:10688000F24F808191810E94E250AB01BC0121E076
:1068900030E087E59CE00E94D04FECE4F3E0849187
:1068A000882341F09091C00095FFFCCF8093C600F3
:1068B0003196F5CF6091EB0370E04AE050E087E558
:1068C0009CE00E94FA4EE8E4F3E08491882341F0D2
:1068D0009091C00095FFFCCF8093C6003196F5CF14
:1068E000F7FE49CFE5E0F3E006C09091C00095FFC8
:1068F000FCCF8093C60081918111F7CF8091C000B9
:1069000085FFFCCF2AE02093C60058CFF7FC91CF3B
:106910006091EB03E62FF0E0EE0FFF1FE05EF24F19
:10692000808191810E94E2502B013C016091EB0338
:10693000E62FF0E0EE0FFF1FEC5DF24F80819181BA
:106940000E94E2509B01AC01C301B2010E947F7121
:106950000E94C87297FF07C09095809570956195C9
:106960007F4F8F4F9F4F64307105810591055CF516
:1069700060CFF7FC2DC00E94B16F6C197D096031AA
:10698000774208F45DCF24C00E94E2502B013C0105
:106990006091EB03E62FF0E0EE0FFF1FEC5DF24F8E
:1069A000808191810E94E25020E030E040E85FE386
:1069B0000E9480719B01AC01C301B2010E94597217
:1069C00018160CF436CF0E94B16F6B017C0131CFE9
:1069D0000E94B16F6093F0037093F1038093F20310
:1069E0009093F3030E94B16F6093F8037093F903DF
:1069F0008093FA039093FB0387CE0E94516488E54D
:106A00000E9492188111179A89E50E9492188111AB
:106A1000169A8AE50E9492188111159A85E40E94BF
:106A20009218882309F470CE149A6ECEA0960FB6F1
:106A3000F894DEBF0FBECDBFDF91CF911F910F91B4
:106A4000FF90EF90DF90CF90BF90AF909F908F908E
:106A50007F906F905F904F903F902F900895CF93CD
:106A6000DF938091020490910304039714F40E9431
:106A7000011960E08EEE95E00E94424C8091020484
:106A800090910304892B09F460C08091EE0588235E
:106A900009F443C0809106049091070420E6289FE2
:106AA000E001299FD00D1124C45FDB4F6FE373E039
:106AB000CE010E94A279892BB9F4BE018EEE95E039
:106AC0000E94D34BE7ECF4E08491882341F090914D
:106AD000C00095FFFCCF8093C6003196F5CF809122
:106AE000C00085FFFCCF15C08EEE95E00E94364DAC
:106AF000E5EBF4E08491882341F09091C00095FF8C
:106B0000FCCF8093C6003196F5CF8091C00085FF01
:106B1000FCCF8AE08093C60002C00E94B925809114
:106B2000020490910304019790930304809302045C
:106B30008091060490910704019664E070E00E9441
:106B4000037690930704809306040E94B6510E9436
:106B5000931FDF91CF910C94755C2AEB33E0FC011D
:106B6000318320832781222319F004960C94E50EAB
:106B700008958EEE95E00C946B458DEB96E0EDDF7D
:106B80008BE796E0EADF8CE596E0E7DF8DE396E0C1
:106B9000E4DF8CE196E0E1CF2F923F924F925F923B
:106BA0006F927F928F929F92AF92BF92CF92DF921D
:106BB000EF92FF920F931F93CF93DF93CDB7DEB782
:106BC00068970FB6F894DEBF0FBECDBF1C012A0137
:106BD0003B0148015901DC01D8966D917D918D9161
:106BE0009C91DB970E94F9726B017C01A3019201D9
:106BF0000E942E750E9446720E94CD726D877E871C
:106C00008F87988BA5019401C701B6010E942E754C
:106C10000E9446720E94CD72698B7A8B8B8B9C8B03
:106C20002D853E854F855889283731054105510509
:106C300040F488E790E0A0E0B0E08D879E87AF87C2
:106C4000B88B29893A894B895C89283731054105F8
:106C5000510540F488E790E0A0E0B0E0898B9A8B82
:106C6000AB8BBC8B91012C5B3F4FD9018D919D91DA
:106C70000D90BC91A02D8D839E83AF83B887BC01FE
:106C8000CD010E94FB7269837A838B839C83F1011F
:106C900064AD75AD86AD97AD0E94F97269877A874C
:106CA0008B879C8720E030E0A90169817A818B8104
:106CB0009C810E945972882339F1A7019601C7016E
:106CC000B6010E942E754B015C0129853A854B85E2
:106CD0005C85CA01B9010E942E759B01AC01C501FA
:106CE000B4010E947F714B015C0129813A814B8183
:106CF0005C81CA01B9010E9480719B01AC01C50190
:106D0000B4010E94607203C060E070E0CB010E9499
:106D100046720E94C8722B013C016D817E818F8179
:106D2000988590958095709561957F4F8F4F9F4F77
:106D30000E94FB724B015C01F101E05CFF4F60813E
:106D40007181828193810E94F9726D837E838F832A
:106D5000988720E030E0A901C501B4010E94597272
:106D6000882349F12D813E814F815885CA01B9019F
:106D70000E942E756D8B7E8B8F8B988FA70196014D
:106D8000C701B6010E942E759B01AC016D897E89F9
:106D90008F89988D0E947F716B017C01A501940100
:106DA000C501B4010E9480719B01AC01C701B6010D
:106DB0000E94607203C060E070E0CB010E943673F5
:106DC000D10150968D909D90AD90BC9053977501D8
:106DD0006401C418D508E608F7080E94C872C61AEC
:106DE000D70AE80AF90AF7FE6BC020E030E0A901F3
:106DF00069817A818B819C810E945972882309F470
:106E000047C029813A814B815C81CA01B9010E9446
:106E100080716B017C01C501B4010E94F9729B0174
:106E2000AC01C701B6010E942E756B017C0129855A
:106E30003A854B855C85CA01B9010E942E759B017C
:106E4000AC01C701B6010E947F716B017C012D81ED
:106E50003E814F815885CA01B9010E942E759B0160
:106E6000AC01C701B6010E9480716B017C0120E07A
:106E700030E040E850E469817A818B819C810E94F6
:106E80002E759B01AC01C701B6010E94607203C060
:106E900060E070E0CB010E9446720E94C8722B0134
:106EA0003C0197FF03C0412C512C32014814590476
:106EB0006A047B0410F024013501C12CD12C760129
:106EC0008FB7F894F101E45BFF4F9081911121C0DD
:106ED000F101448A558A668A778AC40CD51CE61C5F
:106EE000F71CD101C08ED18EE28EF38E2D853E85AA
:106EF0004F85588924AF35AF46AF57AFA05CBF4F21
:106F000029893A894B895C892D933D934D935C93F4
:106F100013978FBF68960FB6F894DEBF0FBECDBF34
:106F2000DF91CF911F910F91FF90EF90DF90CF9065
:106F3000BF90AF909F908F907F906F905F904F9099
:106F40003F902F9008954F925F926F927F92AF92F1
:106F5000BF92CF92DF92EF92FF920F931F93CF9346
:106F6000DF93EB017A01209709F458C041155105D0
:106F700009F454C0AAA4BBA40CA51DA59501A801A1
:106F80006EA17FA188A599A50E945972882309F452
:106F900045C08FA981113AC0F70146A057A060A44F
:106FA00071A4A3019201B501C8010E945C74181676
:106FB0006CF5A3019201C301B2010E942E756B0111
:106FC0007C018AA99BA9ACA9BDA9BC01CD0190589F
:106FD0009B01AC010E9480712EA53FA548A959A92B
:106FE0000E942E759B01AC01C701B6010E947F7102
:106FF0000E949B756B017C019B01AC01B501C8012E
:107000000E94597287FD02C056018701A501B8018F
:107010004EA35FA368A779A781E08EABDF91CF91E4
:107020001F910F91FF90EF90DF90CF90BF90AF90A6
:107030007F906F905F904F900895DF92EF92FF9254
:107040000F931F93CF93DF93809101078FB7F8942D
:10705000E09000078FBF8091010790E08E199109A1
:107060008F7099270497F4F01091010713501F7047
:1070700040E050E000E0F12C8DE4D82E1E1591F098
:10708000111101C010E11150D19EE0011124CE5F19
:10709000D84F602F7F2DCE0156DF402F5F2D0C2F54
:1070A000FD2EECCFDF91CF911F910F91FF90EF90CC
:1070B000DF9008954F925F926F927F92AF92BF924E
:1070C000CF92DF92EF92FF920F931F93CF93DF93B4
:1070D0008C01EB01009709F453C0FC0187A98111D1
:1070E0004FC046A057A060A471A4AEA0BFA0C8A482
:1070F000D9A49501A601C301B2010E94597287FF6C
:107100003FC0A3019201C301B2010E942E752B0161
:107110003C01F80182A993A9A4A9B5A9BC01CD019C
:1071200090589B01AC010E948071F80126A537A5FB
:1071300040A951A90E942E759B01AC01C301B20167
:107140000E947F710E949B757B018C019B01AC01A9
:10715000B501C6010E94597287FF02C07501860100
:107160009701A801B501C6010E945972882341F018
:10717000A701B8014EA35FA368A779A781E08EABF2
:10718000DF91CF911F910F91FF90EF90DF90CF9003
:10719000BF90AF907F906F905F904F900895EF9267
:1071A000FF920F931F93CF93DF93F090000700E0BF
:1071B00010E080E090E02DE4E22E20910107F2162D
:1071C00089F0EF9CE0011124CE5FD84FAE01B801E9
:1071D00071DF81E08F0D803109F480E0F82EC80165
:1071E0008E01EBCF40E050E0B801DF91CF911F91CD
:1071F0000F91FF90EF905ECF4F925F926F927F92D0
:107200008F929F92AF92BF92CF92DF92EF92FF92B6
:107210000F931F93CF93DF9390900007C0E0D0E0CF
:107220003DE4832E892D992787FD909520910107B4
:1072300030E082179307B9F1889E5001899EB00C07
:107240001124C5018E5F984F5C01209729F18EA90A
:10725000811104C0F50186A98823F1F0CAA0DBA042
:10726000ECA0FDA0A7019601F50166A177A180A57C
:1072700091A50E9460722B013C01A70196016EA1AD
:107280007FA188A599A50E946072AB01BC01930102
:107290008201CE0181DC1EAA9394F0E19F1201C00D
:1072A000912CE501BFCF2097E9F0CAA0DBA0ECA0AC
:1072B000FDA0A70196016DEC7CEC8CE49DE30E949F
:1072C00060724B015C01A70196016EA17FA188A5A8
:1072D00099A50E946072AB01BC0195018401CE01A9
:1072E0005BDC1EAADF91CF911F910F91FF90EF9071
:1072F000DF90CF90BF90AF909F908F907F906F90D6
:107300005F904F90089599DE4ADF76CF1092010783
:107310001092000780E1E7EEFBE0DF011D928A9505
:10732000E9F71092D70B1092D80B1092D90B10924C
:10733000DA0B1092DB0B1092DC0B1092DD0B10922B
:10734000DE0B1092DF0B1092E00B1092E10B10920B
:10735000E20B1092E30B1092E40B1092E50B1092EB
:10736000E60B1092D30B1092D40B1092D50B109207
:10737000D60B08954F925F926F927F928F929F9259
:10738000AF92BF92CF92DF92EF92FF920F931F9333
:10739000CF93DF938091D20B882309F4FCC060E087
:1073A0008091240D9091250D0E94E250C0902D02F5
:1073B000D0902E02E0902F02F090300220E030E0DA
:1073C00040E050E40E9480719601A7010E9459722A
:1073D00087FDE1C050900007612C712C00E010E0A7
:1073E0004DE4442E80910107581609F453C0852DB1
:1073F00090E0489EF001499EF00D1124EE5FF84F99
:107400004081518162817381452B462B472B81F44A
:107410004481558166817781452B462B472B41F46A
:107420004085518562857385452B462B472B69F135
:10743000489EE001499ED00D1124CE5FD84F6C8547
:107440007D858E859F850E94FB724B015C0168895A
:1074500079898A899B890E94F9729B01AC01C501D7
:10746000B4010E9460722AA13BA14CA15DA10E94BF
:107470002E755B01D82FC92F9301A8010E945C745F
:1074800018161CF435010D2F1C2F5394852D8F7069
:10749000582EA8CF2091290230912A0240912B0228
:1074A00050912C02B301C8010E942E759B01AC01C2
:1074B000B601C7010E9480718B01D82FC92F960198
:1074C000A7010E94597287FD03C06801ED2EFC2EB2
:1074D0000091310210913202D0913302C0913402F6
:1074E00098014D2F5C2FB601C7010E945C741816DD
:1074F0001CF08601DE2DCF2D8090FB069090FC06BF
:10750000A090FD06B090FE0698014D2F5C2FC5019E
:10751000B4010E945C741816D4F420E037ED43EAFD
:107520005CE3B8018D2F9C2F0E942E756B017C01AE
:1075300028E431EE4AE75FE3C501B4010E942E75ED
:10754000A70196010E9480718B01D82FC92FC80115
:10755000AD2FBC2F8093FB069093FC06A093FD06F5
:10756000B093FE06B8018D2F9C2F0E94C872DC01DB
:10757000CB0160E00E94EE4F9093250D8093240D87
:10758000C801AD2FBC2F80931A0D90931B0DA093B3
:107590001C0DB0931D0DDF91CF911F910F91FF90A6
:1075A000EF90DF90CF90BF90AF909F908F907F90A3
:1075B0006F905F904F900895CF93909100078091C6
:1075C0000107981701F1209100078DE4289FF00131
:1075D0001124E65BF84FC08130E04DE48091010753
:1075E0002817D9F0429FF0011124E65BF84F808103
:1075F0009181A281B381892B8A2B8B2B09F03F5F6C
:107600002F5F2F70EBCF6091BD05662321F070E0F6
:1076100088E00E94AE6EC0E030E08091BD0581112F
:1076200007C0311105C060E070E088E00E94AE6ED6
:107630008091BD05882339F0CC2329F06C2F70E0B0
:1076400088E00E94AE6ECF9195CE2F923F924F92DE
:107650005F926F927F928F929F92AF92BF92CF92E2
:10766000DF92EF92FF920F931F93CF93DF93CDB7EB
:10767000DEB7C856D1090FB6F894DEBF0FBECDBF36
:107680002C015B014A0139012196EFAE2197F8AE3A
:10769000D8A6CFA2209101072F5F25962FAF25975F
:1076A000203119F425961FAE259725963FAD2597D5
:1076B000E32EFF24E7FCF0948091000790E08E1504
:1076C0009F0529F40E94B6510E94931FF5CF209187
:1076D000330C3091340C4091350C5091360CD20162
:1076E0006D917D918D919C910E942E750E94FE74EA
:1076F00065966CAF7DAF8EAF9FAF65972091370CCD
:107700003091380C4091390C50913A0CF501608160
:107710007181828193810E942E750E94FE74699608
:107720006CAF7DAF8EAF9FAF699720913B0C3091CE
:107730003C0C40913D0C50913E0CD4016D917D91DB
:107740008D919C910E942E750E94FE746D966CAF77
:107750007DAF8EAF9FAF6D9720913F0C3091400C65
:107760004091410C5091420CF30160817181828102
:1077700093810E942E750E94FE746CAF7DAF8EAF18
:107780009FAF8091F30B9091F40BA091F50BB0910A
:10779000F60B2CAD3DAD4EAD5FAD281739074A074E
:1077A0005B0789F16091BE05E62FF0E0EE0FFF1F49
:1077B000E05EF24F808191810E94E25020E030E053
:1077C00040EF52E40E94597287FF1DC08091FF066E
:1077D000811119C00C9469449091C00095FFFCCFB1
:1077E0008093C600319684918111F6CFE3EDF7E0E6
:1077F000849181110C9479448091C00085FFFCCF65
:107800008AE08093C6008091F30B9091F40BA091D5
:10781000F50BB091F60B2CAD3DAD4EAD5FAD281B19
:10782000390B4A0B5B0BCA01B90157FF07C0909592
:107830008095709561957F4F8F4F9F4F0E94FB728F
:107840006B017C0120E030E043EC53E460913F0C9D
:107850007091400C8091410C9091420C0E942E75C9
:107860009B01AC01C701B6010E945C7418166CF54F
:107870004CAD5DAD6EAD7FAD4093F30B5093F40B0B
:107880006093F50B7093F60BEDEEF7E0849188238F
:1078900041F09091C00095FFFCCF8093C6003196D7
:1078A000F5CFE5EBF7E08491882341F09091C0009B
:1078B00095FFFCCF8093C6003196F5CF8091C00034
:1078C00085FFFCCF8AE08093C600809101075DE4CC
:1078D000859F10011124B1016E5F784F1B01FB01E0
:1078E000E45BFF4F10828091E70B9091E80BA09131
:1078F000E90BB091EA0B8BA39CA3ADA3BEA3659645
:107900004CAC5DAC6EAC7FAC6597481A590A6A0AFC
:107910007B0A77FE08C07094609450944094411C98
:10792000511C611C711CD1014D925D926D927C9233
:1079300013972091EB0B3091EC0B4091ED0B509194
:10794000EE0B2AA73BA74CA75DA769968CAC9DAC14
:10795000AEACBFAC6997821A930AA40AB50AB7FE07
:1079600008C0B094A09490948094811C911CA11C98
:10797000B11CD10114968D929D92AD92BC92179735
:107980002091EF0B3091F00B4091F10B5091F20BE5
:107990002EA73FA748AB59AB6D96CCACDDACEEAC97
:1079A000FFAC6D97C21AD30AE40AF50AF7FE08C0C5
:1079B000F094E094D094C094C11CD11CE11CF11C43
:1079C000D1011896CD92DD92ED92FC921B972091F9
:1079D000F30B3091F40B4091F50B5091F60B2CAB5F
:1079E0003DAB4EAB5FABA0911502B09116022CAD32
:1079F0003DAD4EAD5FAD6CA97DA98EA99FA9261B9B
:107A0000370B480B590B57FF07C0509540953095E1
:107A100021953F4F4F4F5F4F0E94647624E630E040
:107A200040E050E00E943876D1011C962D933D93A2
:107A30004D935C931F97C814D904EA04FB0414F413
:107A400075016401C216D306E406F50614F4690153
:107A50007A01D301C2014C145D046E047F0414F456
:107A6000D701C601F101808B918BA28BB38B069756
:107A7000A105B10508F446C7E85BFF4F8091BD053D
:107A800090E0A0E0B0E080839183A283B383659609
:107A90002CAD3DAD4EAD5FAD65976BA17CA18DA1C9
:107AA0009EA1261737074807590724F0D101909661
:107AB0001C9203C081E0F10180A369962CAD3DAD1D
:107AC0004EAD5FAD69976AA57BA58CA59DA52617D0
:107AD0003707480759073CF4D10190968C9190974D
:107AE000826090968C936D962CAD3DAD4EAD5FADA2
:107AF0006D976EA57FA588A999A92617370748070E
:107B000059073CF4D10190968C919097846090969F
:107B10008C932CAD3DAD4EAD5FAD6CA97DA98EA90A
:107B20009FA926173707480759073CF4D1019096BB
:107B30008C919097886090968C93EFA1F8A58081A6
:107B4000D10191968C9345284628472809F017982B
:107B5000F10184819581A681B781892B8A2B8B2B9A
:107B600009F01698F10180859185A285B385892B4E
:107B70008A2B8B2B09F01598F10184859585A685B4
:107B8000B785892B8A2B8B2B09F01498D1011C9671
:107B90002D913D914D915C911F9729962CAF3DAF52
:107BA0004EAF5FAF2997232B242B252B11F5B091D6
:107BB000070CBBA3E091080CEFA3F091090CFAAB02
:107BC00020910A0C29A72B2F3E2F4F2F59A5219624
:107BD0006FAD219778ADC8010E94597287FD1AC018
:107BE00021963FAD21973BA348AD4FA30AAB19A700
:107BF00011C050911F0C5BA36091200C6FA370917A
:107C0000210C7AAB8091220C89A7252F362F472F84
:107C1000582FDDCF8091E70B9091E80BA091E90BF5
:107C2000B091EA0B65962CAD3DAD4EAD5FAD65975D
:107C3000281B390B4A0B5B0BCA01B9010E94FB726E
:107C40002091330C3091340C4091350C5091360C0E
:107C50000E9460722B013C01698B7A8B8B8B9C8B11
:107C600069966CAD7DAD8EAD9FAD69972AA53BA59C
:107C70004CA55DA5621B730B840B950B0E94FB72D8
:107C80002091370C3091380C4091390C50913A0CBE
:107C90000E9460724B015C016D8B7E8B8F8B988F85
:107CA0006D966CAD7DAD8EAD9FAD6D972EA53FA54C
:107CB00048A959A9621B730B840B950B0E94FB7298
:107CC00020913B0C30913C0C40913D0C50913E0C6E
:107CD0000E9460726B017C01698F7A8F8B8F9C8F01
:107CE00000911502109116026CAD7DAD8EAD9FAD69
:107CF0002CA93DA94EA95FA9621B730B840B950BA0
:107D00000E94FB7220913F0C3091400C4091410C3D
:107D10005091420C0E9460726AA77BA78CA79DA716
:107D2000B801882777FD8095982F0E94FB729B01F0
:107D3000AC016AA57BA58CA59DA50E942E7520E0AF
:107D400030E048EC52E40E9460726D8F7E8F8F8F1E
:107D500098A3D1012D913D914D915C9113972CAB3E
:107D60003DAB4EAB5FAB2630310541055105FCF410
:107D700014960D911D912D913C9117970630110588
:107D800021053105A4F418960D911D912D913C917A
:107D90001B9706301105210531054CF4DC01CB01A0
:107DA000BF77F10186A797A7A0ABB1AB25C0C301F0
:107DB000B2010E94D9752B013C01C501B4010E949A
:107DC000D9759B01AC01C301B2010E9480714B01C6
:107DD0005C01C701B6010E94D9759B01AC01C501C8
:107DE000B4010E9480710E949B75D1019E966D9393
:107DF0007D938D939C93D197D1019E962D913D912A
:107E00004D915C91D19724962CAF3DAF4EAF5FAFB3
:107E1000249760E070E080E89FE30E9460729B011D
:107E2000AC016BA17FA18AA999A50E942E752B0197
:107E30003C019091010780910007E92FF0E0E81BD9
:107E4000F109EF70FF27FBABEAABA301920160E001
:107E500074E284E799E40E9460720E94FE746B01F0
:107E60007C012AA93BA9223031050CF442C049010A
:107E7000AA2497FCA094BA2CC501B4010E94FB72FD
:107E800020E030E040E051E40E94597287FF31C0A9
:107E90008091530C9091540CA091550CB091560CBC
:107EA000C816D906EA06FB0620F5BC01CD016C19FF
:107EB0007D098E099F09660F771F881F991FA501ED
:107EC00094010E941676CA01B9010E94F9720E94BB
:107ED000FE746C0D7D1D8E1D9F1D0E94F9729B010D
:107EE000AC0160E074E284E799E40E9460722B01C7
:107EF0003C01A301920124966CAD7DAD8EAD9FAD8A
:107F000024970E942E7568AF79AF8AAF9BAFD101DD
:107F100092966D937D938D939C93959750966D91CA
:107F20007D918D919C9153970E94F9726BA37CA3D4
:107F30008DA39EA3A30192010E942E750E944672FA
:107F40000E94CD726B017C01F10160AF71AF82AF15
:107F500093AF8E010F5E1F4F23E43CE061963FAF6D
:107F60002EAF6197AE014F5D5F4F5AA349A3BE018B
:107F70006F5F7F4F2F967FAF6EAF2F971FA219A60F
:107F800070E87AA78FE38EA7D8016D917D918D91CE
:107F90009D918D01A30192010E942E752F96EEAD49
:107FA000FFAD2F9761937193819391932F96FFAFBC
:107FB000EEAF2F979B01AC015F772D962CAF3DAFB5
:107FC0004EAF5FAF2D976196AEADBFAD61978D900F
:107FD0009D90AD90BD906196BFAFAEAF6197A5018A
:107FE00094012D966CAD7DAD8EAD9FAD2D970E9409
:107FF0005C741816F4F42D962CAD3DAD4EAD5FAD0E
:108000002D97C501B4010E946072B62EA72E982E3E
:10801000892E262F372F482F592F6FA179A58AA592
:108020009EA50E94597287FD04C0BFA2A9A69AA668
:108030008EA6E9A1FAA10E171F0709F0A5CF20E02F
:1080400030E040E85FE36FA179A58AA59EA50E9474
:10805000597287FF3DC05E01F1E1AF0EB11C8E0188
:108060000F5F1F4F2FA139A54AA55EA5D8016D91BD
:108070007D918D919C910E942E75F8016193719371
:10808000819391938F01EA15FB0561F72FA139A523
:108090004AA55EA568AD79AD8AAD9BAD0E942E75EF
:1080A000D10192966D937D938D939C939597C70183
:1080B000B6010E94F9722FA139A54AA55EA50E94BA
:1080C0002E750E94CD72F10160AF71AF82AF93AF98
:1080D00024962CAD3DAD4EAD5FAD24976BA17CA138
:1080E0008DA19EA10E9460726B017C012CA93DA90B
:1080F0004EA95FA9232B242B252B59F5F10184814F
:108100009581A681B781892B8A2B8B2B11F58085D0
:108110009185A285B385892B8A2B8B2BD1F4209155
:10812000170C3091180C4091190C50911A0CC70182
:10813000B6010E942E750E94467281010C5B1F4F92
:108140000E94CD72D8016D937D938D939C9313976C
:10815000F6C020911B0C30911C0C40911D0C5091CD
:108160001E0CC701B6010E942E750E9446720E9425
:10817000CD7281010C5B1F4FF80160837183828394
:1081800093834090F70B5090F80B6090F90B709030
:10819000FA0B0E94F9724B015C016CA97DA98EA9B2
:1081A0009FA90E94FB729B01AC01C501B4010E9412
:1081B0002E752BA13CA14DA15EA10E9460724B01C6
:1081C0005C01C301B2010E94F9729B01AC01C501BF
:1081D000B4010E945C74181634F4D8014D925D927B
:1081E0006D927C9213974090FB0B5090FC0B60902B
:1081F000FD0B7090FE0BF80160817181828193818B
:108200000E94F9724B015C01D10114966D917D9130
:108210008D919C9117970E94FB729B01AC01C50147
:10822000B4010E942E752BA13CA14DA15EA10E941C
:1082300060724B015C01C301B2010E94F9729B01A3
:10824000AC01C501B4010E945C7418162CF4F8014D
:1082500040825182628273824090030C5090040CE1
:108260006090050C7090060C81010C5B1F4FD801CB
:108270006D917D918D919C910E94F9724B015C01F1
:1082800029966CAD7DAD8EAD9FAD29970E94FB7296
:108290009B01AC01C501B4010E942E752BA13CA12C
:1082A0004DA15EA10E9460724B015C01C301B2014D
:1082B0000E94F9729B01AC01C501B4010E945C747B
:1082C00018162CF4F8014082518262827382409029
:1082D000FF0B5090000C6090010C7090020CD801C4
:1082E0006D917D918D919C910E94F9724B015C0181
:1082F000F10160857185828593850E94FB729B01E7
:10830000AC01C501B4010E942E752BA13CA14DA169
:108310005EA10E9460724B015C01C301B2010E9428
:10832000F9729B01AC01C501B4010E945C7418167E
:1083300034F4D8014D925D926D927C921397F101C5
:10834000EC5BFF4F60817181828193810E94F972A1
:108350004B015C01A70196010E946072A1966CAF6F
:108360007DAF8EAF9FAFA197F10162AB73AB84ABD2
:1083700095AB2DEB37E346E051E4C501B4010E9413
:108380002E750E94C872D1015C966D937D938D937A
:108390009C935F97C090130CD090140CE090150C38
:1083A000F090160C20E030E040E05FE3C701B6013A
:1083B0000E942E756BA37FA38C0129853A854B857E
:1083C0005C85A5962CAF3DAF4EAF5FAFA5974091B2
:1083D0000F0C5091100C6091110C7091120C48AF61
:1083E00059AF6AAF7BAF20E030E040E05FE368ADBB
:1083F00079AD8AAD9BAD0E942E75B62EA72E982E14
:10840000892EA5966CAD7DAD8EAD9FADA5979F775E
:108410002B2D3A2D492D582D0E945C7418167CF492
:108420002B2D3A2D492D582D6BA17FA1C8010E94FB
:10843000597287FD04C0BBA2AFA2092D182D6D850E
:108440007E858F859889A9966CAF7DAF8EAF9FAFE3
:10845000A99780910B0C90910C0CA0910D0CB091F0
:108460000E0C29968CAF9DAFAEAFBFAF299720E021
:1084700030E040E05FE3BC01CD010E942E75B62ED6
:10848000A72E982E892EA9966CAD7DAD8EAD9FAD91
:10849000A9979F772B2D3A2D492D582D0E945C745A
:1084A00018167CF42B2D3A2D492D582D6BA17FA148
:1084B000C8010E94597287FD04C0BBA2AFA2092D5A
:1084C000182DD1019296BC91B9A7F101F3A1FAA799
:1084D000D1019496BC91BEA7F101F5A1FCAB29A5F1
:1084E0003AA54B2F5F2F6BA17FA1C8010E94597243
:1084F00087FD06C029A52BA33AA53FA30EA51CA95D
:108500004AA95BA9423051050CF40BC15091D30B21
:108510005AAB6091D40B2A966FAF2A977091D50B06
:108520002E967FAF2E978091D60B60968FAF609777
:1085300027E137EB41ED58E36AA92A967FAD2A97E8
:108540002E968FAD2E9760969FAD60970E945C74BB
:1085500018160CF0E6C02091D70B3091D80B409143
:10856000D90B5091DA0B69817A818B819C810E94B1
:108570007F712B013C012091DB0B3091DC0B409192
:10858000DD0B5091DE0B6D817E818F8198850E947D
:108590007F714B015C01A3019201C301B2010E94F2
:1085A0002E752B013C01A5019401C501B4010E9467
:1085B0002E759B01AC01C301B2010E9480710E9423
:1085C0009B754B015C01A70196010E945C74181613
:1085D0004CF4A5019401C701B6010E9460725B01D1
:1085E0004C0106C0A12CB12C50E8852E6FE3962ECD
:1085F0002091DF0B3091E00B4091E10B5091E20BA9
:10860000A5966CAD7DAD8EAD9FADA5970E947F7197
:108610006B017C01E894F7F828AD39AD4AAD5BAD4C
:10862000C701B6010E945C741816D4F4A701960124
:1086300068AD79AD8AAD9BAD0E946072F62EE72ED3
:10864000D82EC92E262F372F482F592FB501C401F8
:108650000E94597287FD04C0AF2CBE2C8D2C9C2C1F
:108660002091E30B3091E40B4091E50B5091E60B28
:10867000A9966CAD7DAD8EAD9FADA9970E947F711F
:108680006B017C01E894F7F829962CAD3DAD4EAD19
:108690005FAD2997C701B6010E945C741816E4F417
:1086A000A701960129966CAD7DAD8EAD9FAD299742
:1086B0000E946072F62EE72ED82EC92E262F372F55
:1086C000482F592FB501C4010E94597287FD04C07B
:1086D000AF2CBE2C8D2C9C2C9501A40169A57AA5EC
:1086E0008EA59CA90E942E754B015C019B01AC01DB
:1086F0006AA92A967FAD2A972E968FAD2E976096FF
:108700009FAD60970E94597287FF0EC08AA82A9673
:108710009FAC2A972E96AFAC2E976096BFAC609711
:1087200003C08BA09FA05801C401D501F10182A70D
:1087300093A7A4A7B5A7A1966CAD7DAD8EAD9FAD57
:10874000A19790589B01AC010E94807124962CAD9A
:108750003DAD4EAD5FAD24970E942E759B01AC01DF
:108760006BE077ED83E29BE30E947F710E949B7533
:108770007B01D82EC92E9B01482F592FB401C5016A
:108780000E94597287FD03C04701AD2CBC2CC40167
:10879000D501F10186A397A3A0A7B1A797014D2DFD
:1087A0005C2D69A57AA58EA59CA90E945972181600
:1087B0002CF081E0D101D7968C9302C0F10117AA69
:1087C00081E0D101D6968C9380E1FE013196A7ED30
:1087D000BBE001900D928A95E1F789A59AA5AEA517
:1087E000BCA98093D30B9093D40BA093D50BB093DB
:1087F000D60B9C01AD016BA17FA1C8010E946072E4
:108800006B017C0129A53AA54EA55CA9B401C5015F
:108810000E946072AB01BC0197018601C1010E94F8
:10882000CC352596BFAD2597B093010765962CAD45
:108830003DAD4EAD5FAD65972093E70B3093E80BF0
:108840004093E90B5093EA0B69964CAD5DAD6EAD6C
:108850007FAD69974093EB0B5093EC0B6093ED0B5E
:108860007093EE0B6D966CAD7DAD8EAD9FAD6D973B
:108870006093EF0B7093F00B8093F10B9093F20BDE
:108880008CAD9DADAEADBFAD8093F30B9093F40B6B
:10889000A093F50BB093F60B0E948339C859DF4FB4
:1088A0000FB6F894DEBF0FBECDBFDF91CF911F9101
:1088B0000F91FF90EF90DF90CF90BF90AF909F907F
:1088C0008F907F906F905F904F903F902F900C947F
:1088D0000E5D2CAD3DAD4EAD5FAD2093F30B3093EF
:1088E000F40B4093F50B5093F60BEDEEF7E00C9480
:1088F000F33B9091C00095FFFCCF8093C60031966A
:108900000C94F83BC859DF4F0FB6F894DEBF0FBE8A
:10891000CDBFDF91CF911F910F91FF90EF90DF902E
:10892000CF90BF90AF909F908F907F906F905F900F
:108930004F903F902F900895EF92FF920F931F93C7
:10894000CF93DF937B018A01E9012091330C3091B1
:10895000340C4091350C5091360CFC0160817181D2
:10896000828193810E942E750E94FE746093E70BB2
:108970007093E80B8093E90B9093EA0B2091370CEE
:108980003091380C4091390C50913A0CF7016081CC
:108990007181828193810E942E750E94FE74609382
:1089A000EB0B7093EC0B8093ED0B9093EE0B2091FF
:1089B0003B0C30913C0C40913D0C50913E0CF80129
:1089C00060817181828193810E942E750E94FE7464
:1089D0006093EF0B7093F00B8093F10B9093F20B7D
:1089E00020913F0C3091400C4091410C5091420C31
:1089F000688179818A819B810E942E750E94FE7414
:108A00006093F30B7093F40B8093F50B9093F60B3C
:108A100023EF3BE04FEE5BE06BEE7BE087EE9BE00D
:108A20000E945D641092D30B1092D40B1092D50B60
:108A30001092D60B1092D70B1092D80B1092D90B24
:108A40001092DA0B1092DB0B1092DC0B1092DD0B04
:108A50001092DE0B1092DF0B1092E00B1092E10BE4
:108A60001092E20B1092E30B1092E40B1092E50BC4
:108A70001092E60BDF91CF911F910F91FF90EF9035
:108A8000089520913F0C3091400C4091410C509141
:108A9000420CFC0160817181828193810E942E755C
:108AA0000E94FE746093F30B7093F40B8093F50BAC
:108AB0009093F60B83EF9BE00C9499648093FF06F0
:108AC0000895FC0114821782138212828AEB93E0CC
:108AD0009183808308950F931F93CF93DF93EC01CD
:108AE0008E96EFDFCE01815B9F4FEBDFCE01825987
:108AF0009F4FE7DFCE0183579F4FE3DFFE01E45531
:108B0000FF4F89E1818314823596178ACE01815304
:108B10009F4FD7DFFE01E251FF4F10821182128278
:108B200013823896108211821282138219821A825D
:108B300018828E010E501F4FF8011082118212828E
:108B40001382389681E080831DA61CA60E94B16F17
:108B500068577C4E8F4F9F4FF801608371838283EB
:108B60009383DF91CF911F910F910895FC0120E035
:108B70003EE2DB014C91403241F0283011F4308369
:108B80003196DB014C91408331962F5F6F5F7F4FB1
:108B90002B3079F7108208953F924F925F926F9237
:108BA0007F928F929F92AF92BF92CF92DF92EF927D
:108BB000FF920F931F93CF93DF93CDB7DEB7C758C4
:108BC000D1090FB6F894DEBF0FBECDBF8C016B018B
:108BD0007A01312C84E0E80EF11C2801E0E14E0E10
:108BE000511C5801FBEFAF0EB11C48018DEF880EF0
:108BF000911C80E4682E712C6C0E7D1EE4E06E0EDC
:108C0000711CA201BE016F5F7F4FC7010E944D0D15
:108C100018160CF019C12C85322F3871303109F03B
:108C20009EC0F501808191810197029708F497C059
:108C3000BE016F5F7F4FCE0187589F4F97DFA09691
:108C40001FAEA097F6018081811107C061E873E033
:108C5000CE01815A9F4F0E946879B601CE01815A98
:108C60009F4F0E946879BE0167587F4FCE01815A9D
:108C70009F4F0E94687961E873E0CE01815A9F4F4F
:108C80000E946879CE01805C9F4F1BDF21E0AE011E
:108C900047585F4FB701C3010E94E210811139C0EC
:108CA000F50180819181892BA1F5ECE1F9E08491B6
:108CB000882341F09091C00095FFFCCF8093C600BF
:108CC0003196F5CFE3E8F3E08191882339F0909174
:108CD000C00095FFFCCF8093C600F6CF8091C00006
:108CE00085FFFCCF8AE08093C600FE01E758FF4F66
:108CF0008191882339F09091C00095FFFCCF80933B
:108D0000C600F6CF8091C00085FFFCCF8AE080933B
:108D1000C6008BE1FE01EC5BFF4FDE0195960190F2
:108D20000D928A95E1F724968EAD9FAD24979CA372
:108D30008BA38AEB93E09AA389A3AE014F5D5F4FAB
:108D4000BE01615A7F4FC80127DFCE0181960E9484
:108D5000AD35CE01805C9F4F0E94AD3552CF8981E9
:108D6000882309F471C0853E09F44BCF8E3209F493
:108D700048CF8F3509F445CF23FD43CF81E0303113
:108D800009F080E0F80183A7811108C08985873444
:108D900009F037CF8A858E3709F433CF98012D5FDC
:108DA0003F4FBE016F5F7F4FC901CA57DF4F288316
:108DB000C658D040C957DF4F3883C758D040D6DE99
:108DC000F50180819181CA57DF4F2881C658D04074
:108DD000C957DF4F3881C758D0400097F1F4F601EA
:108DE0008191882339F09091C00095FFFCCF80934A
:108DF000C600F6CFF9018191882339F09091C00027
:108E000095FFFCCF8093C600F6CF8091C00085FF10
:108E1000FCCF8AE08093C600F4CE8130910539F40E
:108E2000F40180819181019691838083EACE02973B
:108E300009F0E7CE232D30E0F401808191812817DD
:108E4000390711F03394DDCEC957DF4F0FB6F894D0
:108E5000DEBF0FBECDBFDF91CF911F910F91FF906D
:108E6000EF90DF90CF90BF90AF909F908F907F90CA
:108E70006F905F904F903F900895EF92FF920F9305
:108E80001F93CF93DF93CDB7DEB76F970FB6F894EC
:108E9000DEBF0FBECDBF8C01FC01E550FF4F11823C
:108EA00010827C0182E3E80EF11C40E050E0BA0140
:108EB000C7010E94000E8BE1F701DE0115960190BB
:108EC0000D928A95E1F7F80180A991A99C838B8383
:108ED0008AEB93E09A838983AE014F5F5F4F66EE22
:108EE00073E0C80159DECE0101960E94AD356F9640
:108EF0000FB6F894DEBF0FBECDBFDF91CF911F91AB
:108F00000F91FF90EF9008952BE1FB013496DC0167
:108F1000149601900D922A95E1F7FB01228133818D
:108F2000FC01338322830895EF92FF920F931F93E6
:108F3000CF93DF93EC011A828DA9882321F0CE0113
:108F4000C2960E94E50E7E018CEAE80EF11C45E314
:108F500060E0C7010E94285B81111FC0ECE1F9E0CD
:108F60008491882341F09091C00095FFFCCF8093BD
:108F7000C6003196F5CFEFE0F9E08491882341F007
:108F80009091C00095FFFCCF8093C6003196F5CF3D
:108F90008091C00085FFFCCF76C08E010F541F4F1B
:108FA00041E0B701C8010E947A6A811126C040E001
:108FB000B701C8010E947A6A81111FC0E2E2F9E09C
:108FC0008491882341F09091C00095FFFCCF80935D
:108FD000C6003196F5CFECEFF8E08491882341F09C
:108FE0009091C00095FFFCCF8093C6003196F5CFDD
:108FF0008091C00085FFFCCF46C0B801CE01C2966B
:109000000E94EE0B81111FC0E2E2F9E084918823F7
:1090100041F09091C00095FFFCCF8093C60031963F
:10902000F5CFECEEF8E08491882341F09091C000F8
:1090300095FFFCCF8093C6003196F5CF8091C0009C
:1090400085FFFCCF20C081E08A83ECE1F9E08491C8
:10905000882341F09091C00095FFFCCF8093C6001B
:109060003196F5CFE1EEF8E08491882341F09091BC
:10907000C00095FFFCCF8093C6003196F5CF80915C
:10908000C00085FFFCCF8AE08093C6008E01025DA0
:109090001F4FB801CE01815B9F4F36DFC35BDF4FAF
:1090A00019830883DF91CF911F910F91FF90EF906B
:1090B0000895FC01118212820895FC01228122236D
:1090C00011F021E021830895FC01218121111182F9
:1090D00008952F923F924F925F926F927F928F925C
:1090E0009F92AF92BF92CF92DF92EF92FF920F9337
:1090F0001F93CF93DF93CDB7DEB7AD970FB6F8943C
:10910000DEBF0FBECDBF7C016B014DA7FC0182818C
:10911000882309F4A3C14701F3ED8F0E911CC4010C
:109120000E94E50EF7011182CE0101965C01C9DCB7
:1091300017019DE4290E311CC7018E96F101918320
:109140008083F60180818F3209F081C06FE270E088
:10915000C6010E9473798C010F5F1F4F0115110525
:1091600009F47BC06FE270E0C8010E9473792C01A2
:10917000009709F473C00817190708F06FC03C0185
:10918000601A710AA301B801CE0180960E949379FA
:10919000E0E2F0E0EC0FFD1FE60DF71D1082FE018E
:1091A000B0968191882339F09091C00095FFFCCF53
:1091B0008093C600F6CF8091C00085FFFCCFFAE017
:1091C000F093C600F101608171816115710519F09C
:1091D0006C5F7F4F02C060E070E021E0AE01405E56
:1091E0005F4FCE0105960E94E21081112BC0EDEC7D
:1091F000F8E08491882341F09091C00095FFFCCF66
:109200008093C6003196F5CFFE01B09681918823F8
:1092100039F09091C00095FFFCCF8093C600F6CF47
:10922000EBECF8E08491882341F09091C00095FF29
:10923000FCCF8093C6003196F5CF8091C00085FFAA
:10924000FCCF06C1F101B182A082820185CFC701A6
:10925000815B9F4FF101918380838601FDA5FF23F0
:1092600009F49BC0F101608171816115710519F0EC
:109270006C5F7F4F02C060E070E021E0A801C40194
:109280000E94E210882309F45EC0F401818992896A
:10929000A389B489F701E251FF4F80839183A283B0
:1092A000B383EEEBF8E08491D701A251BF4F88233E
:1092B00049F09091C00095FFFCCF8093C600319695
:1092C0008491F5CFF8018191882339F09091C00005
:1092D00095FFFCCF8093C600F6CFE7EBF8E08491D2
:1092E000882341F09091C00095FFFCCF8093C60089
:1092F0003196F5CF4D915D916D917C912AE030E0F2
:1093000087E59CE0A3D58091C00085FFFCCF8AE073
:109310008093C600F701EA50FF4F1082118212823B
:109320001382E9EAF8E08491882341F09091C0002B
:1093300095FFFCCF8093C6003196F5CF8091C00099
:1093400085FFFCCF85C0E5E9F8E08491882341F0F2
:109350009091C00095FFFCCF8093C6003196F5CF69
:10936000F8018191882339F09091C00095FFFCCFDE
:109370008093C600F6CFE3E9F8E08491882341F0BA
:109380009091C00095FFFCCF8093C6003196F5CF39
:109390008091C00085FFFCCF5BC0F10160817181CD
:1093A0006115710519F06C5F7F4F02C060E070E0DD
:1093B00026E5A801C4010E94E21081112AC0EFE74E
:1093C000F8E08491882341F09091C00095FFFCCF94
:1093D0008093C6003196F5CFF8018191882339F04A
:1093E0009091C00095FFFCCF8093C600F6CFEDE7CB
:1093F000F8E08491882341F09091C00095FFFCCF64
:109400008093C6003196F5CF8091C00085FFFCCFD8
:109410001FC081E0F7018083EBE6F8E084918823A8
:1094200041F09091C00095FFFCCF8093C60031962B
:10943000F5CFF6018191882339F09091C00095FF16
:10944000FCCF8093C600F6CF8091C00085FFFCCF93
:109450008AE08093C600C5010E94AD35AD960FB677
:10946000F894DEBF0FBECDBFDF91CF911F910F915A
:10947000FF90EF90DF90CF90BF90AF909F908F9034
:109480007F906F905F904F903F902F9008953F9204
:109490004F925F926F927F928F929F92AF92BF9204
:1094A000CF92DF92EF92FF920F931F93CF93DF93B0
:1094B000CDB7DEB7AC970FB6F894DEBF0FBECDBF09
:1094C0007C015B01FC018281882309F401C1C70191
:1094D0008D529F4F0E94E50EF7011182CE01019639
:1094E0006C01EFDA27019DE4490E511CC7018E96ED
:1094F000F20191838083F50180818F3209F084C06D
:109500006FE270E0C5010E9473798C010F5F1F4FFD
:109510009AE0392E0115110509F47CC06FE270E064
:10952000C8010E9473794C01009709F474C00817B0
:10953000190708F070C03C01601A710AA301B80154
:10954000CE0180960E949379E0E2F0E0EC0FFD1FDF
:10955000E60DF71D1082FE01B0968191882339F047
:109560009091C00095FFFCCF8093C600F6CF80910C
:10957000C00085FFFCCF3092C600F201608171818E
:109580006115710519F06C5F7F4F02C060E070E0FB
:1095900021E0AE01405E5F4FCE0105960E94E210D1
:1095A00081112BC0E7E5F8E08491882341F0909188
:1095B000C00095FFFCCF8093C6003196F5CFFE0129
:1095C000B0968191882339F09091C00095FFFCCF2F
:1095D0008093C600F6CFE5E5F8E08491882341F05A
:1095E0009091C00095FFFCCF8093C6003196F5CFD7
:1095F0008091C00085FFFCCF65C0F201D182C0829E
:1096000084010F5F1F4F86CFC701815B9F4FF2011F
:10961000918380838501F20180819181009711F00F
:10962000049602C080E090E0B8010E94B91188233E
:1096300001F1E7E4F8E08491882341F09091C000C3
:1096400095FFFCCF8093C6003196F5CFF80181914C
:10965000882339F09091C00095FFFCCF8093C6001D
:10966000F6CFF701EA50FF4F108211821282138267
:109670002CC0EFE2F8E08491882341F09091C00083
:1096800095FFFCCF8093C6003196F5CFF80181910C
:10969000882339F09091C00095FFFCCF8093C600DD
:1096A000F6CFEDE2F8E08491882341F09091C0007C
:1096B00095FFFCCF8093C6003196F5CF8091C00016
:1096C00085FFFCCF8AE08093C600C6010E94AD35BD
:1096D000AC960FB6F894DEBF0FBECDBFDF91CF9131
:1096E0001F910F91FF90EF90DF90CF90BF90AF90C0
:1096F0009F908F907F906F905F904F903F900895D4
:10970000CF93DF93EC018A818823B1F1EBE1F8E09C
:109710008491882341F09091C00095FFFCCF809305
:10972000C6003196F5CFFE01EA50FF4F40815181CE
:10973000628173812AE030E087E59CE087D3E9E12C
:10974000F8E08491882341F09091C00095FFFCCF10
:109750008093C6003196F5CFC251DF4F48815981C1
:109760006A817B812AE030E087E59CE06FD38091BD
:10977000C00085FFFCCF11C0E9E0F8E084918823A8
:1097800041F09091C00095FFFCCF8093C6003196C8
:10979000F5CF8091C00085FFFCCF8AE08093C600A2
:1097A000DF91CF910895AF92BF92CF92DF92EF9267
:1097B000FF920F931F93CF93DF935C01EB01FB01AB
:1097C00001900020E9F78F0101501109061B170BCA
:1097D0006C01F3EDCF0ED11CF60110826EE470E047
:1097E000CE010E9473797C01009729F4F80131972A
:1097F000EC0FFD1F0DC060E270E00E947379EC0178
:1098000021966AE270E0C7010E947379FC013197EA
:109810008DE081838AE082831382BE01C50181537A
:109820009F4F8FD1F6018081882309F1E2E2F9E0B0
:109830008491882341F09091C00095FFFCCF8093E4
:10984000C6003196F5CFE3EFF7E08491882341F02D
:109850009091C00095FFFCCF8093C6003196F5CF64
:109860008091C00085FFFCCF8AE08093C600DF9125
:10987000CF911F910F91FF90EF90DF90CF90BF900D
:10988000AF9008952F923F924F925F926F927F9286
:109890008F929F92AF92BF92CF92DF92EF92FF9200
:1098A0000F931F93CF93DF93CDB7DEB7CC55D1097C
:1098B0000FB6F894DEBF0FBECDBF8C0186509F4F10
:1098C0005C01662339F0F5011082F8018281811173
:1098D0001DC015C0FC018081882309F4ADC0F801CA
:1098E000EE50FF4FC080D180E280F3800E94B16FC4
:1098F000C616D706E806F90608F49EC0E4CFC801EC
:1099000013DBF8018281882309F496C0F80185A54C
:109910008F9384A58F9386E993E09F938F937E0125
:10992000FFE3EF0EF11CFF92EF920E94BC790F90C3
:109930000F900F900F900F900F90B12CF7010190A6
:109940000020E9F73197EE19FF09BE1684F467018C
:10995000CB0CD11CB7FCDA94F6018081992787FDE6
:1099600090950E943279F6018083B394E7CF480145
:10997000F2E38F0E911C40E050E0BA01C4010E9456
:10998000000E512CCE0101966C012FE9622E23E0CE
:10999000722E5E0191E2A90EB11C40E050E0B601CA
:1099A000C4010E944D0D1816DCF5412CF601019002
:1099B0000020E9F73197EC19FD094E1674F41601F1
:1099C000240C311C47FC3A94F101808190E00E9404
:1099D0003279F10180834394E9CF8A858E37E9F2A9
:1099E00045E050E0B701C6010E948579892BA9F6B0
:1099F000FF92EF927F926F92BF92AF920E94BC79DA
:109A0000C5010E940B1886EA93E00E940B180F9084
:109A10000F900F900F900F900F9055245394BDCF3F
:109A2000511004C08FEF9FEFF80104C0F80184A526
:109A300095A5019695A784A7C45ADF4F0FB6F89451
:109A4000DEBF0FBECDBFDF91CF911F910F91FF9071
:109A5000EF90DF90CF90BF90AF909F908F907F90CE
:109A60006F905F904F903F902F9008950F931F93AA
:109A7000CF93DF93EC018C010D521F4FC8010E9460
:109A80009A0EC8010E94E50E1882DF91CF911F91B6
:109A90000F910895CF93DF93EC010E9451640E94CF
:109AA000BE6419828AEA93E00E940B188091D20B5F
:109AB000882391F11092D20B6091BE05E62FF0E061
:109AC000EE0FFF1FEC5DF24F808191817BD32091DF
:109AD0002D0230912E0240912F02509130020E94AF
:109AE0005C741816CCF46091BE05C62FD0E080E0FF
:109AF00090E074D2FE01EE0FFF1FEC5DF24F9183F8
:109B00008083FE01EE0FFF1FEE0FFF1FE65EF24F98
:109B10001082118212821382DF91CF910895CF9328
:109B2000DF931F92CDB7DEB7698341E050E0BE01FD
:109B30006F5F7F4F04960E94E1110F90DF91CF91EC
:109B40000895FB0101900020E9F7AF014150510950
:109B5000461B570B04960C94E1111F920F920FB6FF
:109B60000F9211240BB60F922F933F934F935F9355
:109B70006F938F939F93EF93FF936091C600209113
:109B8000D80C3091D90CC90101968F779927409153
:109B9000DA0C5091DB0C8417950741F0F901E85A73
:109BA000F34F60839093D90C8093D80CFF91EF9181
:109BB0009F918F916F915F914F913F912F910F9056
:109BC0000BBE0F900FBE0F901F9018959A01AB011E
:109BD000211581EE38074105510549F182E0809356
:109BE000C00060E079E08DE390E00E94387621507B
:109BF000310941095109CA01B90122E030E040E0D0
:109C000050E00E9438763093C5002093C4008091C4
:109C1000C10080618093C1008091C1008860809301
:109C2000C1008091C10080688093C10008951092A6
:109C3000C00020E130E0E7CF2091DA0C3091DB0C5E
:109C40008091D80C9091D90C8217930771F0F9018B
:109C5000E85AF34F80812F5F3F4F2F7733273093A0
:109C6000DB0C2093DA0C90E008958FEF9FEF0895BE
:109C70008091DA0C9091DB0C9093D90C8093D80CE6
:109C800008954F925F926F927F928F929F92AF92C0
:109C9000BF92CF92DF92EF92FF920F931F93CF93D9
:109CA000DF93CDB7DEB7A0970FB6F894DEBF0FBE37
:109CB000CDBF5C014115510561057105E9F420E056
:109CC00030E040E350E060E070E0A0960FB6F8941A
:109CD000DEBF0FBECDBFDF91CF911F910F91FF90DF
:109CE000EF90DF90CF90BF90AF909F908F907F903C
:109CF0006F905F904F905BC08E010F5F1F4FC12C24
:109D0000D12C76014801422E512C612C712C8FEF01
:109D1000C81AD80AE80AF80ACB01BA01A3019201CD
:109D20000E941676CA01F80161938F01A901BC0156
:109D3000411551056105710551F7F1E0CF1AD108C0
:109D4000E108F108F401EC0DFD1D80818A3010F46A
:109D500040E301C047E3480F552747FD5095652F65
:109D6000752F20E030E0C50122D081E0C81AD1086B
:109D7000E108F108EFEFCE16DE06EE06FE0611F75B
:109D8000A0960FB6F894DEBF0FBECDBFDF91CF9186
:109D90001F910F91FF90EF90DF90CF90BF90AF9009
:109DA0009F908F907F906F905F904F9008952115B6
:109DB000310539F48091C00085FFFCCF4093C60087
:109DC00008952A30310509F41CC05BCFCF93DF938F
:109DD000EC0120E030E04DE050E060E070E0E7DFD3
:109DE00020E030E04AE050E060E070E0CE01DF913A
:109DF000CF91DDCF9A01AB01662757FD6095762F95
:109E0000D6CFCF92DF92EF92FF92CF93DF93EC0108
:109E10006A017B0177FF0FC020E030E04DE250E0A7
:109E200060E070E0C4DFF094E094D094C094C11C72
:109E3000D11CE11CF11C2AE0B701A601CE01DF9183
:109E4000CF91FF90EF90DF90CF901BCF2115310580
:109E500039F48091C00085FFFCCF4093C60008957F
:109E600010CF9A01462F50E060E070E0EFCFCF9323
:109E7000DF93EC019A01AB0160E070E0E7DFCE0117
:109E8000DF91CF91A3CF8F929F92AF92BF92CF924B
:109E9000DF92EF92FF921F93CF93DF93EC016A0161
:109EA0007B01122F20E030E0A901C701B6010E941A
:109EB000597287FF0CC020E030E04DE250E060E0D6
:109EC00070E0CE0174DFF7FAF094F7F8F094B12C5B
:109ED00060E070E080E09FE3B11641F020E030E008
:109EE00040E251E40E946072B394F6CF9B01AC0152
:109EF000C701B6010E9480716B017C010E94CD7286
:109F00004B015C010E94F9729B01AC01C701B601D3
:109F10000E947F716B017C012AE0B501A401CE0192
:109F2000B0DE112361F0EEEBF3E08191882339F08C
:109F30009091C00095FFFCCF8093C600F6CF11230F
:109F400019F120E030E040E251E4C701B6010E947F
:109F50002E756B017C010E94C8724B01AA2497FCEC
:109F6000A094BA2CB501A401CE014BDFC501B40108
:109F70000E94FB729B01AC01C701B6010E947F7178
:109F80006B017C011150DBCFDF91CF911F91FF90CE
:109F9000EF90DF90CF90BF90AF909F908F900895FB
:109FA00072CF20914202309143024091440250917D
:109FB000450260E070E08FE793E40E946072609376
:109FC000F50C7093F60C8093F70C9093F80C0895B1
:109FD0008D50934FFC01808190E00895EF92FF92A5
:109FE0000F931F93CF93DF93EC01662349F1EDEDBF
:109FF000FAE08491882341F09091C00095FFFCCF56
:10A000008093C6003196F5CF70E04AE050E087E5D6
:10A010009CE0F0DEEAEDF9E08491882341F0909134
:10A02000C00095FFFCCF8093C6003196F5CF80919C
:10A03000C00085FFFCCF8AE08093C6000E94661FA7
:10A040004AEE5AE021E030E0C9012733310509F436
:10A0500048C0FA01659174912F5F3F4FFA01349621
:10A060006C177D070CF03BC09C0121503109B901F0
:10A07000660F771F660F771F6C51754FFB010591B7
:10A080001491220F331F220F331F2A51354FF9012C
:10A09000A591B491FC01EE0FFF1FEE0FFF1FEC51D5
:10A0A000F54F85919491FB01E590F490FA0165914B
:10A0B0007491F90125913491CA1BDB0BAC014E1947
:10A0C0005F09C49FC001C59F900DD49F900D1124BE
:10A0D000621B730B0E940376600F711F06C0AF01F5
:10A0E000B3CFECEBFBE06591749180EF9FE3861BAF
:10A0F000970BDF91CF911F910F91FF90EF900895F3
:10A10000EF92FF920F931F93CF93DF934AEE5AE0A3
:10A1100021E030E0FA0165917491681779070CF03D
:10A120003AC0D9011197BD01660F771F660F771FDF
:10A130006C51754FFB01C591D491AA0FBB1FAA0F9B
:10A14000BB1FAA51B54FFD0105911491F901EE0F06
:10A15000FF1FEE0FFF1FEC51F54FE590F490FB0150
:10A1600025913491FA0165917491FD0145915491C5
:10A17000FC01E01BF10BE21AF30AEE9DC001EF9D1A
:10A18000900DFE9D900D1124641B750B0E940376AB
:10A190006C0F7D1F0CC02F5F3F4F4C5F5F4F27330D
:10A1A000310509F0B7CFECEBFBE06591749180EFDE
:10A1B0009FE3861B970BDF91CF911F910F91FF902B
:10A1C000EF9008954F925F926F927F928F929F923D
:10A1D000AF92BF92CF92DF92EF92FF920F931F93B5
:10A1E000CF93DF93EC01662349F1EDEDFAE0849122
:10A1F000882341F09091C00095FFFCCF8093C6006A
:10A200003196F5CF70E04AE050E087E59CE0F2DD62
:10A21000EDEBF9E08491882341F09091C00095FF27
:10A22000FCCF8093C6003196F5CF8091C00085FFAA
:10A23000FCCF8AE08093C6000E94661FB0EF4B2ED1
:10A24000BFE35B2E4C1A5D0A28EE3AE081E090E015
:10A25000DC018733910509F46EC0F90145915491F1
:10A260000196B9016C5F7F4F441655060CF061C032
:10A27000CD010197AC01440F551F440F551F4A51A2
:10A28000554FFA0165917491880F991F880F991F96
:10A290008C51954FFC0165907490FD01EE0FFF1FEE
:10A2A000EE0FFF1FEA51F54FA590B490FA0105910A
:10A2B0001491F901C591D491FC018590949088275F
:10A2C00077FD8095982F0E94FB726B017C01B20193
:10A2D00066197709882777FD8095982F0E94FB7271
:10A2E0002B013C01B501601B710B882777FD809520
:10A2F000982F0E94FB729B01AC01C301B2010E9426
:10A300002E752B013C01BE0168197909882777FD5C
:10A310008095982F0E94FB729B01AC01C301B20192
:10A320000E9460729B01AC01C701B6010E9480715E
:10A330000CC09B018DCFEEEBFBE0659174918827FB
:10A3400077FD8095982F0E94FB72DF91CF911F912E
:10A350000F91FF90EF90DF90CF90BF90AF909F90C4
:10A360008F907F906F905F904F9008952F923F92C3
:10A370004F925F926F927F928F929F92AF92BF9215
:10A38000CF92DF92EF92FF920F931F93CF93DF93C1
:10A3900000D01F92CDB7DEB78091190D882309F444
:10A3A00078C18FB7F8941092190D8FBF60E080913B
:10A3B000200D9091210D06DF6B017C019B01AC010A
:10A3C00060911A0D70911B0D80911C0D90911D0DC7
:10A3D0000E947F712B013C016093FD0C7093FE0C79
:10A3E0008093FF0C9093000D20E030E040E251E4B8
:10A3F0000E945C7418160CF4E9C020E030E040E2E2
:10A4000051ECC301B2010E94597287FDDBC08091FB
:10A41000F40C8111CCC0209146023091470240914A
:10A42000480250914902C301B2010E942E754B01AE
:10A430005C016093090D70930A0D80930B0D90934E
:10A440000C0D2091110D3091120D4091130D509172
:10A45000140DC301B2010E9480712B013C010091D7
:10A46000F90C1091FA0C2090FB0C3090FC0C980128
:10A47000A1010E94597287FD98C00091F50C1091BE
:10A48000F60C2090F70C3090F80C9801A101B20165
:10A49000C3010E945C7418160CF487C08201C801C5
:10A4A000D3018093110D9093120DA093130DB093CF
:10A4B000140D209142023091430240914402509188
:10A4C0004502B801C3010E942E7569837A838B838C
:10A4D0009C836093050D7093060D8093070D9093F8
:10A4E000080D20910D0D30910E0D40910F0D5091E2
:10A4F000100DC701B6010E947F7120913E0230917C
:10A500003F0240914002509141020E942E7520ED81
:10A510003CEC4CE45DE30E942E752B013C0123E3EF
:10A5200033E343E75FE36091010D7091020D809189
:10A53000030D9091040D0E942E759B01AC01C30187
:10A54000B2010E9480712B013C016093010D709358
:10A55000020D8093030D9093040DC0920D0DD092C7
:10A560000E0DE0920F0DF092100D29813A814B8172
:10A570005C81C501B4010E948071A30192010E9417
:10A580007F716B017C0120E030E0A9010E945972CB
:10A5900087FD26C020E030E04FE753E4C701B60155
:10A5A0000E945C741816FCF414C0310178CF10922C
:10A5B000110D1092120D1092130D1092140D109295
:10A5C000F40C29CF81E08093F40C0AC081E08093E1
:10A5D000F40CC12CD12C0FE7E02E03E4F02E03C0C5
:10A5E000C12CD12C76018091200D9091210D2091CC
:10A5F000F10C3091F20C281739071CF01092F30C73
:10A600000FC0209138023091390282179307B4F7B6
:10A61000C701B6010E94C872759567956093F30CE7
:10A620000E94B16F0091150D1091160D2091170D1C
:10A630003091180D601B710B820B930B68387341BE
:10A640008105910530F10E94B16F6093150D7093F3
:10A65000160D8093170D9093180D80911E0D9091FB
:10A660001F0D2091EF0C3091F00C2817390784F45E
:10A670002091360230913702821793074CF42091D3
:10A68000220D3091230D8217930714F4759A01C09F
:10A6900075980F900F900F900F90DF91CF911F91B1
:10A6A0000F91FF90EF90DF90CF90BF90AF909F9071
:10A6B0008F907F906F905F904F903F902F90089574
:10A6C0004F925F926F927F928F929F92AF92BF92C2
:10A6D000CF92DF92EF92FF920F931F93CF93DF936E
:10A6E000D0EF4D2EDFE35D2E481A590A28EE3AE0EE
:10A6F00081E090E0F90145915491441655060CF023
:10A7000062C0AC0141505109DA01AA0FBB1FAA0F68
:10A71000BB1FAA51B54FFD0165917491440F551FA0
:10A72000440F551F4C51554FFA0165907490FC0130
:10A73000EE0FFF1FEE0FFF1FEA51F54FA590B490EB
:10A74000FD0105911491F901C591D491FA0185900B
:10A750009490882777FD8095982F0E94FB726B015B
:10A760007C01B20166197709882777FD8095982FBB
:10A770000E94FB722B013C01B501601B710B882705
:10A7800077FD8095982F0E94FB729B01AC01C3015D
:10A79000B2010E942E752B013C01BE016819790996
:10A7A000882777FD8095982F0E94FB729B01AC0152
:10A7B000C301B2010E9460729B01AC01C701B601E6
:10A7C0000E94807111C001962C5F3F4F8733910525
:10A7D00009F090CFEEEBFBE065917491882777FD4F
:10A7E0008095982F0E94FB72DF91CF911F910F915E
:10A7F000FF90EF90DF90CF90BF90AF909F908F90A1
:10A800007F906F905F904F9008951092F90C109286
:10A81000FA0C1092FB0C1092FC0C20914202309129
:10A820004302409144025091450260E070E08FE79E
:10A8300093E40E9460726093F50C7093F60C809321
:10A84000F70C9093F80CE1E0F1E080818064808364
:10A850008081806180836D9A80818062808387EDB2
:10A8600080937A00EEE7F0E0108210927D00808104
:10A870008160808380818260808380818460808326
:10A8800080E888BDEEE6F0E08081846080836AEF36
:10A8900070E080E090E00E94E06F60E085E090E092
:10A8A0009DDB9093F20C8093F10C60E08AEF90E0D6
:10A8B00095DB909339028093380285E090E020DCAC
:10A8C0009093F00C8093EF0C86E990E019DC909364
:10A8D0003702809336020895089560E080E090E0AA
:10A8E0007DDB9093250D8093240D10921A0D10920C
:10A8F0001B0D10921C0D10921D0D80E090E000DCED
:10A900009093230D8093220D1092250D1092240D0B
:10A910001092F30C9FB7F894E2E0F1E080818F7B16
:10A9200080839FBF1092270D1092260D1092F40C79
:10A930009FB7F89480818F7E80839FBF1092230DF4
:10A940001092220D759808952F923F924F925F9228
:10A950006F927F928F929F92AF92BF92CF92DF922F
:10A96000EF92FF920F931F93CF93DF93CDB7DEB794
:10A97000A6970FB6F894DEBF0FBECDBF6EA37B8B3C
:10A980008C8B292E0E94B16F6D8B7E8B8F8B988F55
:10A99000E0ECF3E08191882339F09091C00095FFBD
:10A9A000FCCF8093C600F6CF8091C00085FFFCCF1E
:10A9B0008AE08093C60091DF8FE78093F30C2D89A6
:10A9C0003E894F89588D2F87388B498B5A8B2B871F
:10A9D0003C874D875E878FE790E0A0E0B0E08983F9
:10A9E0009A83AB83BC836FE7462E512C612C712C6C
:10A9F00091E09D831A8619868091190D882309F4A8
:10AA0000CBC08FB7F8941092190D8FBF60E0809182
:10AA1000200D9091210DD6DB362E072F182F9DA3E8
:10AA2000262F372F482F592F698D7A8D8B8D9C8D2E
:10AA30000E945C7418162CF0398E0A8F1B8FADA102
:10AA4000AC8F232D302F412F5DA16D8D7E8D8F8D8D
:10AA500098A10E94597287FD05C03D8E0E8F1F8FF1
:10AA6000BDA1B8A3ED81EE2309F448C02EA13B8916
:10AA70004C89522D632D702F812F9DA10E945C74F3
:10AA800018160CF089C00E94B16F2F85388949894A
:10AA90005A89621B730B840B950B693873418105CE
:10AAA000910508F479C0D301C20129813A814B8113
:10AAB0005C81821B930BA40BB50BB595A79597955D
:10AAC00087958093F30C0E94B16F6B877C878D878D
:10AAD0009E87DC01CB012F85388949895A89821BE1
:10AAE000930BA40BB50B89A39AA3ABA3BCA33EA164
:10AAF000398F4B894A8F5C895B8F2C8E2EA13B89C5
:10AB00004C89522D632D702F812F9DA10E94597267
:10AB100087FFCDC20E94B16F2B853C854D855E8538
:10AB2000621B730B840B950B69387341810591058A
:10AB300008F4BDC20E94B16F6F87788B898B9A8BA6
:10AB4000DC01CB012B853C854D855E85821B930BFB
:10AB5000A40BB50B49855A85452B09F0F6C08981B0
:10AB60009A81AB81BC81840D951DA61DB71DB5953D
:10AB7000A795979587958093F30C29853A852F5F44
:10AB80003F4F3A8729873EA13D8F4B894E8F5C8985
:10AB90005F8F28A281E08D8320E030E040EA51E41D
:10ABA0006EA17B898C89922D0E9480719B01AC01E2
:10ABB000632D702F812F9DA10E945C74181694F450
:10ABC000EEE6FAE08491882341F09091C00095FF71
:10ABD000FCCF8093C6003196F5CF8091C00085FFF1
:10ABE000FCCF97C00E94B16F2D893E894F89588D47
:10ABF000621B730B840B950B613D774081059105BA
:10AC000008F43CC00E94B16F6D8B7E8B8F8B988F48
:10AC1000E8E6FAE08491882341F09091C00095FF26
:10AC2000FCCF8093C6003196F5CF60E08091200D77
:10AC30009091210DC7DAAB01BC0122E030E087E53D
:10AC40009CE0AED9E4E6FAE08491882341F090914B
:10AC5000C00095FFFCCF8093C6003196F5CF609180
:10AC6000F30C70E04AE050E087E59CE0C3D88091A7
:10AC7000C00085FFFCCF8AE08093C6000E94B16FC0
:10AC80006B017C010E94B16F8B849C84AD84BE8477
:10AC90002F85388949895A89820E931EA41EB51EB4
:10ACA000C818D908EA08FB08C60ED71EE81EF91E08
:10ACB00031E8C3163FE4D30632E1E306F10490F035
:10ACC000E7E4FAE08491882341F09091C00095FF79
:10ACD000FCCF8093C6003196F5CF8091C00085FFF0
:10ACE000FCCF17C049855A85463051050CF484CEF7
:10ACF000E6EFF9E08491882341F09091C00095FF40
:10AD0000FCCF8093C6003196F5CF8091C00085FFBF
:10AD1000FCCF8AE08093C600A6960FB6F894DEBFFB
:10AD20000FBECDBFDF91CF911F910F91FF90EF909C
:10AD3000DF90CF90BF90AF909F908F907F906F905B
:10AD40005F904F903F902F90089589A09AA0ABA05C
:10AD5000BCA0880E991EAA1EBB1E29A13AA14BA118
:10AD60005CA1281B390B4A0B5B0BCA01B901298175
:10AD70003A814B815C810E94F475A50194010E9487
:10AD80003876240D351D461D571D243131054105EA
:10AD9000510504F129013A013CEE431651046104C6
:10ADA00071042CF04BEE442E512C612C712C40E898
:10ADB0004416510461047104DCF08EEF90E0A0E0D1
:10ADC000B0E084199509A609B70989839A83AB83F2
:10ADD000BC8312C034E1432E512C612C712C24E130
:10ADE00030E040E050E029833A834B835C8304C029
:10ADF00049825A826B827C82E5EDFAE08491882355
:10AE000041F09091C00095FFFCCF8093C600319631
:10AE1000F5CF2AE030E0B301A20187E59CE00E9473
:10AE2000D74EE0EDFAE08491882341F09091C00084
:10AE300095FFFCCF8093C6003196F5CF2AE030E035
:10AE400049815A816B817C8187E59CE00E94D74EC5
:10AE5000E9ECFAE08491882341F09091C00095FFDD
:10AE6000FCCF8093C6003196F5CF22E030E04D8DC7
:10AE70005E8D6F8D78A187E59CE092D8E2ECFAE0D8
:10AE80008491882341F09091C00095FFFCCF80937E
:10AE9000C6003196F5CF22E030E0498D5A8D6B8D9A
:10AEA0007C8D87E59CE07CD88091C00085FFFCCF3D
:10AEB0008AE08093C60029853A85233031050CF459
:10AEC0004ECE69817A818B819C810E94FB7220E049
:10AED00030E040E850E40E942E756B017C012D8D1E
:10AEE0003E8D4F8D58A1698D7A8D8B8D9C8D0E94E2
:10AEF0007F7120ED3FE049E450E40E942E7520E090
:10AF000030E040E05FE30E942E759B01AC01C70179
:10AF1000B6010E9460726B017C01C501B4010E9400
:10AF2000FB7220E030E04AE754E40E9460724B017B
:10AF30005C01ECEBFAE08491882341F09091C00031
:10AF400095FFFCCF8093C6003196F5CF22E030E02C
:10AF5000B701A60187E59CE023D8E6EBFAE08491EF
:10AF6000882341F09091C00095FFFCCF8093C600EC
:10AF70003196F5CF22E030E0B501A40187E59CE0F1
:10AF80000FD88091C00085FFFCCF8AE08093C60077
:10AF90002AE939E949E15FE3C701B6010E942E754C
:10AFA0006B017C019B01AC010E948071A5019401A1
:10AFB0000E9460726D837E838F839887A5019401C0
:10AFC000C701B6010E942E7520E030E040E05EE34C
:10AFD0000E942E754B015C01E9EAFAE08491882316
:10AFE00041F09091C00095FFFCCF8093C600319650
:10AFF000F5CF8091C00085FFFCCF8AE08093C6002A
:10B00000E3EAFAE08491882341F09091C00095FF33
:10B01000FCCF8093C6003196F5CF22E030E0B70137
:10B02000A60187E59CE00E94D04F8091C00085FF7B
:10B03000FCCF8AE08093C600EDE9FAE08491882392
:10B0400041F09091C00095FFFCCF8093C6003196EF
:10B05000F5CF22E030E04D815E816F81788587E514
:10B060009CE00E94D04F8091C00085FFFCCF8AE019
:10B070008093C600E7E9FAE08491882341F090913B
:10B08000C00095FFFCCF8093C6003196F5CF22E03B
:10B0900030E0B501A40187E59CE00E94D04F80918B
:10B0A000C00085FFFCCF8AE08093C60058CD1D828A
:10B0B00073CDCF93C82F11DC0E942E20811130C098
:10B0C000EDEDFAE09491992341F08091C00085FF65
:10B0D000FCCF9093C6003196F5CF6C2F70E04AE01C
:10B0E00050E087E59CE00E94FA4E8091C00085FF09
:10B0F000FCCF8AE08093C600E0E9F9E084918823E0
:10B1000041F09091C00095FFFCCF8093C60031962E
:10B11000F5CF8091C00085FFFCCF8AE08093C60008
:10B12000CF910895CF93C82FD8DB0E942E20811194
:10B1300030C0EDEDFAE09491992341F08091C00088
:10B1400085FFFCCF9093C6003196F5CF6C2F70E051
:10B150004AE050E087E59CE00E94FA4E8091C000F2
:10B1600085FFFCCF8AE08093C600E3E6F9E0849196
:10B17000882341F09091C00095FFFCCF8093C600DA
:10B180003196F5CF8091C00085FFFCCF8AE0809397
:10B19000C600CF91089575980E942E20811121C07C
:10B1A000EDEDFAE08491882341F09091C00095FF85
:10B1B000FCCF8093C6003196F5CFE9E2F9E08491A7
:10B1C000882341F09091C00095FFFCCF8093C6008A
:10B1D0003196F5CF8091C00085FFFCCF8AE0809347
:10B1E000C60008951F920F920FB60F9211240BB64E
:10B1F0000F922F933F934F935F936F937F938F9310
:10B200009F93AF93BF93EF93FF938091350281118A
:10B210000EC08091F30C8093EE0C882341F09FB711
:10B22000F894809102018064809302019FBF909105
:10B23000EE0C80913502891740F09FB7F894809109
:10B2400002018F7B809302019FBF809135028F5F47
:10B250008F77809335028091ED0C90E088309105D6
:10B2600008F080C0FC01EE58FF4F0C945476109209
:10B270007B0080E480937C0080917A0080648093DE
:10B280007A0081E019C02091780030917900809196
:10B29000E90C9091EA0CA091EB0CB091EC0C820FB0
:10B2A000931FA11DB11D8093E90C9093EA0CA0930C
:10B2B000EB0CB093EC0C82E08093ED0C53C082E475
:10B2C00080937C0080917A00806480937A0083E090
:10B2D000F3CF20917800309179008091E50C909126
:10B2E000E60CA091E70CB091E80C820F931FA11D12
:10B2F000B11D8093E50C9093E60CA093E70CB093FE
:10B30000E80C84E0D9CF10927B0081E480937C002C
:10B3100080917A00806480937A0085E0CDCF20917F
:10B320007800309179008091E10C9091E20CA0912D
:10B33000E30CB091E40C820F931FA11DB11D80930B
:10B34000E10C9093E20CA093E30CB093E40C86E044
:10B35000B3CF87E0B1CF1092ED0C8091E00C8F5FFE
:10B360008093E00C8091E00C803108F471C02FEFE5
:10B370003FE38091E90C9091EA0CA901481B590B1D
:10B38000CA015093210D4093200D4091E50C50913E
:10B39000E60C241B350B30931F0D20931E0D21E06E
:10B3A0002093190D1092E00C1092E90C1092EA0C07
:10B3B0001092EB0C1092EC0C1092E10C1092E20C3B
:10B3C0001092E30C1092E40C1092DC0C1092DD0C45
:10B3D0001092DE0C1092DF0C1092E50C1092E60C2D
:10B3E0001092E70C1092E80C20913802309139024B
:10B3F0008217930744F01092250D1092240D80E0DF
:10B4000058DE0E94F31F2091200D3091210D809174
:10B41000F10C9091F20C8217930744F01092250DD5
:10B420001092240D80E07EDE0E94F31F20911E0DFD
:10B4300030911F0D809136029091370228173907FD
:10B440003CF01092230D1092220DA5DE0E94F31FF6
:10B45000FF91EF91BF91AF919F918F917F916F91EC
:10B460005F914F913F912F910F900BBE0F900FBEA8
:10B470000F901F9018958FEF8EBD0DB407FEFDCF76
:10B480008EB508958EBD0DB407FEFDCF089561E021
:10B49000FC0180810C94EE70FC012281322F306A15
:10B4A00036953CBD20FD06C031E0263009F430E081
:10B4B000232F01C020E02DBD60E0FC0180810C94B1
:10B4C000EE70CF92DF92EF92FF920F931F93CF9384
:10B4D000DF93EC018B017A010E94B16F6B01CBDF2E
:10B4E0008B838F3F49F40E94B16F6C197D096D32D7
:10B4F0007140A8F381E103C08E3F31F08FE0898372
:10B50000CE01C5DF80E024C0E114F104E1F081E068
:10B51000E81AF1088FEF8EBDF8012FEFCF01801BE5
:10B52000910B8E159F0538F40DB407FEFDCF8EB537
:10B5300081932EBDF3CF0DB407FEFDCF8EB5F8017C
:10B54000EE0DFF1D808397DF96DFCE01A0DF81E047
:10B55000DF91CF911F910F91FF90EF90DF90CF90EF
:10B5600008950F931F93CF93DF93EB010E94B16F68
:10B570008B0181DF8F3F49F00E94B16F601B710B1F
:10B580006C177D07B0F380E001C081E0DF91CF91BF
:10B590001F910F910895CF92DF92FF920F931F9307
:10B5A000CF93DF9300D01F92CDB7DEB76C01F62E9C
:10B5B00029833A834B835C836FDF6CE271E0C601C1
:10B5C000D0DF8F2D80645EDF08E110E05C814B816D
:10B5D0003A812981DA01C901002E04C0B695A795E8
:10B5E000979587950A94D2F729833A834B835C8396
:10B5F00049DF0850110929813A814B815C81083F5C
:10B600008FEF180739F7FF2029F0E8E0FE1621F048
:10B610008FEF03C085E901C087E834DFFCE0FF124B
:10B6200001C029DF10E027DFF601838387FF04C014
:10B630001F3F11F01F5FF7CF0F900F900F900F90EB
:10B64000DF91CF911F910F91FF90DF90CF900895E0
:10B65000BF92CF92DF92EF92FF920F931F93CF93FF
:10B66000DF93EC01B62E1C82198248830E94B16FD1
:10B670008B0161E088810E94B570CE0108DF60E037
:10B6800082E30E94B57061E083E30E94B57061E0DF
:10B6900084E30E94B57061E085E30E94B57061E0CB
:10B6A00085E30E94EE7085E08A8382E58CBD1DBC37
:10B6B0002AE0F22E8FEFE6DEFA94E1F720E030E0A8
:10B6C000A90160E0CE0167DFF82E8B8381E0F816D8
:10B6D00049F00E94B16F601B710B613D774070F3C0
:10B6E00081E046C02AEA31E040E050E068E0CE0167
:10B6F00052DF82FF02C0FC820CC094E0F92EBBDE58
:10B700008B83FA94E1F78A3A11F082E031C082E04B
:10B710008C838C81823031F4C12CD12CE12C80E4DB
:10B72000F82E03C0C12CD12C760120E030E0A90115
:10B7300067E3CE0130DFA701960169E2CE012BDF7E
:10B740008B83882349F00E94B16F601B710B613DB0
:10B75000774058F38AE00CC08C818230B1F420E04D
:10B7600030E0A9016AE3CE0116DF882329F088E0E2
:10B770008983CE018CDE14C07EDE807C803C11F497
:10B7800083E08C8378DE77DE76DECE0180DE86E0B5
:10B790008B1518F488E1898303C0BA8281E001C067
:10B7A00080E0DF91CF911F910F91FF90EF90DF909C
:10B7B000CF90BF9008950F931F93CF93DF93EC0129
:10B7C00089018C81833039F039E0440F551F661FA1
:10B7D000771F3A95D1F79A01AB0161E1CE01DBDE2B
:10B7E000811109C040E052E0B801CE01DF91CF9154
:10B7F0001F910F9166CE84E08983CE0148DE80E000
:10B80000DF91CF911F910F910895CF93DF93EC01BA
:10B810006EBD20E030E00DB407FEFDCFFA01E20F6F
:10B82000F31F80818EBD0DB407FEFDCF81818EBDDB
:10B830002E5F3F4F211582E0380769F70DB407FEF0
:10B84000FDCF8FEF1FDE8FEF1DDE15DE8B838F7137
:10B85000853031F083E18983CE0119DE80E001C0BB
:10B8600081E0DF91CF9108950F931F93CF93DF93E2
:10B87000EC0189018C81833039F089E0440F551F38
:10B88000661F771F8A95D1F79A01AB0168E1CE0157
:10B8900082DE882311F086E01EC0A8016EEFCE0183
:10B8A000B4DF8823C9F068E572E0CE015ADE182FB4
:10B8B000811102C087E10FC020E030E0A9016DE0F6
:10B8C000CE0169DE811106C0D6DD811103C0CE0133
:10B8D000DEDD05C086E18983CE01D9DD10E0812F50
:10B8E000DF91CF911F910F91089580913E0D8111AD
:10B8F00009C080913D0D811105C080913C0D8111E1
:10B9000001C00895EFEFF3E18491882341F0909115
:10B91000C00095FFFCCF8093C6003196F5CFE0EFD5
:10B92000FBE08491882341F09091C00095FFFCCF0B
:10B930008093C6003196F5CF80913E0D8823D1F0DB
:10B9400060913F0D7091400D8091410D9091420D9D
:10B950000E94FB722091330C3091340C4091350CD5
:10B960005091360C0E946072AB01BC018CEE9BE0E2
:10B970000E94F71480913D0D8823D1F06091430D12
:10B980007091440D8091450D9091460D0E94FB727F
:10B990002091370C3091380C4091390C50913A0C71
:10B9A0000E946072AB01BC0188EE9BE00E94F7141C
:10B9B00080913C0D8823D1F06091470D7091480D26
:10B9C0008091490D90914A0D0E94FB7220913B0C91
:10B9D00030913C0C40913D0C50913E0C0E946072A5
:10B9E000AB01BC0184EE9BE00E94F7148091C00083
:10B9F00085FFFCCF8AE08093C60010923E0D109226
:10BA00003D0D10923C0D089510923E0D10923D0D8B
:10BA100010923C0D089580934E020895EFE6F0E0F9
:10BA200080818260808308951F920F920FB60F92DB
:10BA300011240BB60F920F931F932F933F934F93A5
:10BA40005F936F937F938F939F93AF93BF93EF9386
:10BA5000FF9380916D0D90916E0D892B09F07DC142
:10BA60009091010780910007981771F0E09100070D
:10BA70008DE4E89FF0011124EE5FF84FDF01A45B35
:10BA8000BF4F81E08C9302C0E0E0F0E0F0936E0DD8
:10BA9000E0936D0D309709F45AC1DF01A45BBF4FED
:10BAA00081E08C931092500D1092510D1092520D16
:10BAB0001092530D60AD71AD61349CE9790728F4A3
:10BAC00061329EE4790748F002C060E47CE9769533
:10BAD00067957695679584E007C0613197E27907AD
:10BAE00030F07695679582E080934D0D07C0809386
:10BAF0004D0D6032710510F460E270E06052710922
:10BB0000611588E07807D0F0872F9927880F991F53
:10BB1000880F991F8150904FFC01329645915491A6
:10BB2000AA27659F9001649F210D3A1F06942A1F42
:10BB30003A1F1124FC01859194911DC0CB0196956B
:10BB400087958C7F8150944FFC01459154910296CA
:10BB5000FC0185919491FB01E770FF278E9F900176
:10BB60008F9F300D9E9F300D1124E3E03695279571
:10BB7000EA95E1F7CA01821B930B84369105A0F484
:10BB8000E3EDF3E08191882339F09091C00095FFB7
:10BB9000FCCF8093C600F6CF4AE050E087E59CE0FA
:10BBA0000E94374F84E690E090934C0D80934B0DAC
:10BBB000E0916D0DF0916E0D64AD75AD70934F0D0C
:10BBC00060934E0D61349CE9790728F461328EE46C
:10BBD000780748F002C060E47CE976956795769531
:10BBE000679584E007C0613197E2790730F0769578
:10BBF000679582E080934D0D08C081E080934D0DE4
:10BC00006032710510F460E270E0605271096115F4
:10BC100088E07807E0F0872F9927880F991F880F11
:10BC2000991F8150904FFC01329625913491AA279B
:10BC3000639FA001629F410D5A1F06944A1F5A1F1D
:10BC40001124FC0125913491241B350B1EC0CB011E
:10BC5000969587958C7F8150944FFC012591349166
:10BC60000296FC0145915491FB01E770FF274E9F1E
:10BC7000C0014F9F900D5E9F900D1124F3E09695AB
:10BC80008795FA95E1F7281B390B24363105A0F486
:10BC9000E3EDF3E08191882339F09091C00095FFA6
:10BCA000FCCF8093C600F6CF4AE050E087E59CE0E9
:10BCB0000E94374F24E630E0C901A0E0B0E0809355
:10BCC000540D9093550DA093560DB093570D30938E
:10BCD000890020938800E0916D0DF0916E0D8089B0
:10BCE0009189A289B389B695A79597958795B095BF
:10BCF000A095909581959F4FAF4FBF4F8093680D52
:10BD00009093690DA0936A0DB0936B0D8093640DB1
:10BD10009093650DA093660DB093670D8093600DB1
:10BD20009093610DA093620DB093630D80935C0DB1
:10BD300090935D0DA0935E0DB0935F0D1092580D22
:10BD40001092590D10925A0D10925B0D06C080EDA5
:10BD500097E09093890080938800E0916D0DF091B9
:10BD60006E0D309709F488C580A180936C0D9FB744
:10BD700080FF48C0F89480910B018D7F80930B0168
:10BD80009FBF8FEF80934A0280914E02882309F46F
:10BD90007EC023B131E026FB222720F9232779F149
:10BDA00080913B0D882359F1E0916D0DF0916E0D5E
:10BDB00080819181A281B381181619061A061B068B
:10BDC000F4F48091260D9091270DA091280DB0914B
:10BDD000290D80933F0D9093400DA093410DB0939A
:10BDE000420D30933E0D80899189A289B389809359
:10BDF000580D9093590DA0935A0DB0935B0D20935D
:10BE00003B0D45C0F89480910B01826080930B013B
:10BE10009FBF31E030934A0280914E028823B9F1EE
:10BE200020B122FB222720F9232779F180913A0DB6
:10BE3000882359F1E0916D0DF0916E0D8081918113
:10BE4000A281B381181619061A061B06F4F4809114
:10BE5000260D9091270DA091280DB091290D80936A
:10BE60003F0D9093400DA093410DB093420D309340
:10BE70003E0D80899189A289B3898093580D909352
:10BE8000590DA0935A0DB0935B0D20933A0D8091FC
:10BE90006C0D9FB781FF48C0F89480910B018160C1
:10BEA00080930B019FBF8FEF80934B0280914E02D6
:10BEB000882309F47DC023B131E025FB222720F936
:10BEC000232779F18091390D882359F1E0916D0D87
:10BED000F0916E0D84819581A681B781181619069F
:10BEE0001A061B06F4F480912A0D90912B0DA09157
:10BEF0002C0DB0912D0D8093430D9093440DA09384
:10BF0000450DB093460D30933D0D80899189A289EE
:10BF1000B3898093580D9093590DA0935A0DB09307
:10BF20005B0D2093390D44C0F89480910B018E7FF6
:10BF300080930B019FBF31E030934B0280914E0202
:10BF40008823B1F120B126952170232779F18091C2
:10BF5000380D882359F1E0916D0DF0916E0D8481BB
:10BF60009581A681B781181619061A061B06F4F4E6
:10BF700080912A0D90912B0DA0912C0DB0912D0D3B
:10BF80008093430D9093440DA093450DB093460DBF
:10BF900030933D0D80899189A289B3898093580D92
:10BFA0009093590DA0935A0DB0935B0D2093380DCB
:10BFB00080916C0D9FB782FF47C0F89480910B0170
:10BFC0008B7F80930B019FBF8FEF80934C028091FA
:10BFD0004E02882309F47DC023B131E022952170FF
:10BFE000232779F18091370D882359F1E0916D0D68
:10BFF000F0916E0D80859185A285B385181619067E
:10C000001A061B06F4F480912E0D90912F0DA0912D
:10C01000300DB091310D8093470D9093480DA09352
:10C02000490DB0934A0D30933C0D80899189A289C6
:10C03000B3898093580D9093590DA0935A0DB093E6
:10C040005B0D2093370D45C0F89480910B018460FF
:10C0500080930B019FBF31E030934C0280914E02E0
:10C060008823B9F126B12095221F2227221F79F1BA
:10C070008091360D882359F1E0916D0DF0916E0D90
:10C0800080859185A285B385181619061A061B06A8
:10C09000F4F480912E0D90912F0DA091300DB09160
:10C0A000310D8093470D9093480DA093490DB093A7
:10C0B0004A0D30933C0D80899189A289B389809380
:10C0C000580D9093590DA0935A0DB0935B0D20938A
:10C0D000360D80916C0D9FB783FF09C0F894809155
:10C0E0000B01806480930B019FBF8FEF08C0F89411
:10C0F00080910B018F7B80930B019FBF81E0809328
:10C100004D0220E080914D0D28170CF0ADC18091BB
:10C11000C00087FF19C03091C6004091D80C5091E3
:10C12000D90CCA0101968F7799276091DA0C70912A
:10C13000DB0C8617970741F0FA01E85AF34F30837A
:10C140009093D90C8093D80CE0916D0DF0916E0D09
:10C150008091680D9091690DA0916A0DB0916B0D61
:10C160004081518162817381840F951FA61FB71F83
:10C170008093680D9093690DA0936A0DB0936B0D39
:10C18000181619061A061B06CCF5409AE0916D0D9B
:10C19000F0916E0D8091680D9091690DA0916A0DDE
:10C1A000B0916B0D4089518962897389841B950B0D
:10C1B000A60BB70B8093680D9093690DA0936A0D41
:10C1C000B0936B0D40914A028091260D9091270DFE
:10C1D000A091280DB091290D552747FD5095652F49
:10C1E000752F840F951FA61FB71F8093260D909360
:10C1F000270DA093280DB093290D4098E0916D0D67
:10C20000F0916E0D8091640D9091650DA091660D79
:10C21000B091670D4481558166817781840F951FA8
:10C22000A61FB71F8093640D9093650DA093660DB4
:10C23000B093670D181619061A061B06CCF5419A1D
:10C24000E0916D0DF0916E0D8091640D9091650DF2
:10C25000A091660DB091670D4089518962897389FB
:10C26000841B950BA60BB70B8093640D9093650D03
:10C27000A093660DB093670D40914B0280912A0DFB
:10C2800090912B0DA0912C0DB0912D0D552747FDB0
:10C290005095652F752F840F951FA61FB71F80938C
:10C2A0002A0D90932B0DA0932C0DB0932D0D41983A
:10C2B000E0916D0DF0916E0D8091600D9091610D8A
:10C2C000A091620DB091630D4085518562857385A3
:10C2D000840F951FA61FB71F8093600D9093610D6B
:10C2E000A093620DB093630D181619061A061B066B
:10C2F000CCF5429AE0916D0DF0916E0D8091600D3C
:10C300009091610DA091620DB091630D40895189AA
:10C3100062897389841B950BA60BB70B8093600D04
:10C320009093610DA093620DB093630D40914C0208
:10C3300080912E0D90912F0DA091300DB091310D67
:10C34000552747FD5095652F752F840F951FA61F04
:10C35000B71F80932E0D90932F0DA093300DB093A7
:10C36000310D4298E0916D0DF0916E0D80915C0D54
:10C3700090915D0DA0915E0DB0915F0D4485558546
:10C3800066857785840F951FA61FB71F80935C0D68
:10C3900090935D0DA0935E0DB0935F0D1816190676
:10C3A0001A061B06CCF5439AE0916D0DF0916E0DC7
:10C3B00080915C0D90915D0DA0915E0DB0915F0D2F
:10C3C0004089518962897389841B950BA60BB70B31
:10C3D00080935C0D90935D0DA0935E0DB0935F0D07
:10C3E00040914D028091320D9091330DA091340D0A
:10C3F000B091350D552747FD5095652F752F840F4A
:10C40000951FA61FB71F8093320D9093330DA093F5
:10C41000340DB093350D43988091580D9091590D7E
:10C42000A0915A0DB0915B0D0196A11DB11D809395
:10C43000580D9093590DA0935A0DB0935B0D4091F8
:10C44000580D5091590D60915A0D70915B0DE0910E
:10C450006D0DF0916E0D80899189A289B38948177D
:10C4600059076A077B07B0F04091580D5091590D5C
:10C4700060915A0D70915B0DE0916D0DF0916E0D14
:10C4800084899589A689B78984179507A607B70770
:10C4900018F4DAC02F5F36CE4091540D5091550DEF
:10C4A0006091560D7091570D048D158D268D378D29
:10C4B000AA27419FB12D529FC001629F900D619F9D
:10C4C000800D911D429FB00D811D9A1F519FB00D8F
:10C4D000811D9A1F609FB00D811D9A1F509FB10D45
:10C4E0008A1F9A1FB6958A1F9A1F112444AD55AD15
:10C4F000480F591F50934F0D40934E0D80AD91AD95
:10C50000A2ADB3AD60E070E084179507A607B7074A
:10C5100020F490934F0D80934E0D60914E0D7091CD
:10C520004F0D61349CE9790728F461328EE4780775
:10C5300048F002C060E47CE976956795769567954A
:10C5400084E007C0613197E2790730F0769567950E
:10C5500082E080934D0D08C081E080934D0D6032E4
:10C56000710510F460E270E060527109611588E0B5
:10C570007807E0F0872F9927880F991F880F991F58
:10C580008150904FFC01329625913491AA27639FE8
:10C59000A001629F410D5A1F06944A1F5A1F112481
:10C5A000FC0125913491241B350B1EC0CB019695BF
:10C5B00087958C7F8150944FFC0125913491029690
:10C5C000FC0145915491FB01E770FF274E9FC0018C
:10C5D0004F9F900D5E9F900D112413E096958795C7
:10C5E0001A95E1F7281B390B24363105A0F4E3ED49
:10C5F000F3E08191882339F09091C00095FFFCCF42
:10C600008093C600F6CF4AE050E087E59CE00E94A8
:10C61000374F24E630E030938900209388008091E2
:10C62000540D9091550DA091560DB091570D820F5C
:10C63000931FA11DB11D8093540D9093550DA09390
:10C64000560DB093570DF3C04091580D5091590DB0
:10C6500060915A0D70915B0D808D918DA28DB38D7F
:10C6600084179507A607B70708F0D9C04091500D69
:10C670005091510D6091520D7091530D048D158D97
:10C68000268D378DAA27419FB12D529FC001629FF1
:10C69000900D619F800D911D429FB00D811D9A1FCD
:10C6A000519FB00D811D9A1F609FB00D811D9A1F73
:10C6B000509FB10D8A1F9A1FB6958A1F9A1F112489
:10C6C00020914E0D30914F0DE05CFF4F2817390738
:10C6D00018F42081318102C0281B390B808191819F
:10C6E000A281B381A90160E070E0481759076A0789
:10C6F0007B0708F49C0121349CE9390728F4213296
:10C700008EE4380748F002C020E43CE936952795CE
:10C710003695279584E007C0213197E2390730F03C
:10C720003695279582E080934D0D08C081E0809377
:10C730004D0D2032310510F420E230E0B901605295
:10C740007109611588E07807E0F0872F9927880F35
:10C75000991F880F991F8150904FFC0132962591A7
:10C760003491AA27639FA001629F410D5A1F06942E
:10C770004A1F5A1F1124FC0125913491241B350BAB
:10C780001EC0CB01969587958C7F8150944FFC01FC
:10C79000259134910296FC0145915491FB01E7707B
:10C7A000FF274E9FC0014F9F900D5E9F900D11245B
:10C7B00043E0969587954A95E1F7281B390B243677
:10C7C0003105A0F4E3EDF3E08191882339F09091F5
:10C7D000C00095FFFCCF8093C600F6CF4AE050E042
:10C7E00087E59CE00E94374F24E630E030938900D3
:10C7F000209388008091500D9091510DA091520D81
:10C80000B091530D820F931FA11DB11D8093500D48
:10C810009093510DA093520DB093530D08C0809189
:10C820004B0D90914C0D909389008093880040911E
:10C83000580D5091590D60915A0D70915B0DE0911A
:10C840006D0DF0916E0D80899189A289B389481789
:10C8500059076A077B0780F010926E0D10926D0DDC
:10C860009091010780910007981731F0809100079F
:10C870008F5F8F7080930007FF91EF91BF91AF9111
:10C880009F918F917F916F915F914F913F912F91E8
:10C890001F910F910F900BBE0F900FBE0F901F9026
:10C8A00018959091010780910007981729F00E9430
:10C8B000B6510E94931FF5CF0895CF93DF93EFB742
:10C8C000F894EC0188819981AA81BB818093260D1F
:10C8D0009093270DA093280DB093290DEB0188812B
:10C8E0009981AA81BB8180932A0D90932B0DA093EF
:10C8F0002C0DB0932D0DEA0188819981AA81BB810D
:10C9000080932E0D90932F0DA093300DB093310D89
:10C91000E90188819981AA81BB818093320D90932E
:10C92000330DA093340DB093350DEFBFDF91CF9150
:10C9300008952FB7F894FC0180819181A281B38181
:10C940008093320D9093330DA093340DB093350D39
:10C950002FBF08952FB7F89494E0899FF001112418
:10C96000EA5DF24F60817181828193812FBF0895CA
:10C9700098DF179A169A159A149A089580916F0065
:10C980008D7F80936F00909101078091000798132D
:10C990000AC010926E0D10926D0D80916F00826032
:10C9A00080936F0008959091010780910007981778
:10C9B00051F3809100078F5F8F7080930007E3CF62
:10C9C000CF93DF93D82FC62F60E086E20E94EE70EF
:10C9D000DEBD0DB407FEFDCF8EB5CEBD0DB407FE96
:10C9E000FDCF8EB561E086E20E94EE70DF91CF91BF
:10C9F0000895CF93DF9300D01F921F92CDB7DEB77B
:10CA000095E0EFE7F2E0DE01119601900D929A9524
:10CA1000E1F7E1E0F0E0EC0FFD1FE80FF11D808190
:10CA200090E00F900F900F900F900F90DF91CF91AB
:10CA3000C7CFFF920F931F93CF93DF9300D01F9226
:10CA40001F92CDB7DEB785E0E4E8F2E0DE01119693
:10CA500001900D928A95E1F70E949C6E61E086E25A
:10CA60000E94B5708E010F5F1F4FF12CF80161918C
:10CA70008F0170E08F2DBDDFF394F5E0FF12F6CF4C
:10CA80000F900F900F900F900F90DF91CF911F910B
:10CA90000F91FF900895CF93C42F67FD2BC0823074
:10CAA000B9F028F4882341F0813061F023C083304D
:10CAB000A9F08430C9F01EC088E20E94EE70C7FF62
:10CAC00028C038C085E40E94EE70C7FF25C032C080
:10CAD00084E40E94EE70C7FF22C02CC081E40E9453
:10CAE000EE70C7FF1FC026C08FE30E94EE70C7FF25
:10CAF0001CC020C0C7FD1EC0823089F028F48823E6
:10CB000041F0813049F016C0833061F0843069F023
:10CB100011C06C2F89E20BC06C2F87E208C06C2F0C
:10CB200083E405C06C2F82E402C06C2F80E4CF91B7
:10CB30000C94EE70CF910895643079F028F4613050
:10CB400041F0623041F00895683051F0603141F0B9
:10CB5000089540E003C040E004C041E060E002C04E
:10CB600041E061E098CFFF920F931F93CF93DF9343
:10CB700000D01F921F92CDB7DEB785E0E9E8F2E062
:10CB8000DE01119601900D928A95E1F761E089E24C
:10CB90000E94B57061E087E20E94B57061E083E4B5
:10CBA0000E94B57061E082E40E94B57061E080E4AB
:10CBB0000E94B5708E010F5F1F4FF12CF80161913B
:10CBC0008F018F2DB9DFF394F5E0FF12F7CF0F90AF
:10CBD0000F900F900F900F90DF91CF911F910F91B9
:10CBE000FF90089526DFBFDFEAE0F1E080818260F8
:10CBF0008083808181608083808184608083808164
:10CC0000806480838081806880830F9A179A0E9A4F
:10CC1000169A0D9A159A0C9A149A0B9A139A2698AA
:10CC20002E9A25982D9A24982C9A0A98129A099847
:10CC3000119A3F98479A389A4098179A399A41988A
:10CC4000169A3A9A4298159A3B9A4398149A3C9AA3
:10CC50004498139AA1E8B0E08C918F7E8C938C91CC
:10CC600088608C93E0E8F0E080818D7F8083808114
:10CC70008E7F808380818F73808380818F7C80838F
:10CC80008C91887F82608C9380E090E490938900FF
:10CC9000809388001092850010928400EFE6F0E007
:10CCA00080818260808381E080934E027894089531
:10CCB000E6EDFBE08491882341F09091C00095FF60
:10CCC000FCCF8093C6003196F5CFE2EDFBE0849176
:10CCD000882341F09091C00095FFFCCF8093C6005F
:10CCE0003196F5CF88E20E9423714AE050E0BC0102
:10CCF00087E59CE00E94FA4E89E20E9423714AE097
:10CD000050E0BC0187E59CE00E94FA4E8091C00093
:10CD100085FFFCCF8AE08093C600EEECFBE08491B7
:10CD2000882341F09091C00095FFFCCF8093C6000E
:10CD30003196F5CF85E40E9423714AE050E0BC01B2
:10CD400087E59CE00E94FA4E87E20E9423714AE048
:10CD500050E0BC0187E59CE00E94FA4E8091C00043
:10CD600085FFFCCF8AE08093C600EAECFBE084916B
:10CD7000882341F09091C00095FFFCCF8093C600BE
:10CD80003196F5CF84E40E9423714AE050E0BC0163
:10CD900087E59CE00E94FA4E83E40E9423714AE0FA
:10CDA00050E0BC0187E59CE00E94FA4E8091C000F3
:10CDB00085FFFCCF8AE08093C600E5ECFBE0849120
:10CDC000882341F09091C00095FFFCCF8093C6006E
:10CDD0003196F5CF81E40E9423714AE050E0BC0116
:10CDE00087E59CE00E94FA4E82E40E9423714AE0AB
:10CDF00050E0BC0187E59CE00E94FA4E8091C000A3
:10CE000085FFFCCF8AE08093C600E0ECFBE08491D4
:10CE1000882341F09091C00095FFFCCF8093C6001D
:10CE20003196F5CF8FE30E9423714AE050E0BC01B8
:10CE300087E59CE00E94FA4E80E40E9423714AE05C
:10CE400050E0BC0187E59CE00E94FA4E8091C00052
:10CE500085FFFCCF8AE08093C6000895CF93809130
:10CE6000730D8823B9F14091760F5091770F60913F
:10CE7000780F7091790F26E73DE08091740D9091C5
:10CE8000750D0E94345CC82F811102C0C0E023C020
:10CE900040916F0D5091700D6091710D7091720DF8
:10CEA000411551056105710591F026E73DE080913E
:10CEB000740D9091750D0E94345C882339F31092A3
:10CEC0006F0D1092700D1092710D1092720D1092E4
:10CED000730D01C0C1E08C2FCF910895CF92DF92E6
:10CEE000EF92FF92CF936B017C01C42F8091760F5C
:10CEF0009091770FA091780FB091790F8C159D05C7
:10CF0000AE05BF05C9F0AADF811102C080E018C0DC
:10CF100026E73DE0B701A6018091740D9091750D53
:10CF20000E94DB5B882391F3C092760FD092770F3B
:10CF3000E092780FF092790F81E0C1118093730D28
:10CF4000CF91FF90EF90DF90CF9008958F929F92B6
:10CF5000AF92BF92CF92DF92EF92FF920F931F9307
:10CF6000CF93DF93EC016A017B01890189859A8562
:10CF7000AB85BC850196A11DB11D84179507A60739
:10CF8000B70710F480E054C08F89803129F49927C5
:10CF9000872F762F652F0BC08032A1F7CB01BA0106
:10CFA00027E096958795779567952A95D1F78B8891
:10CFB0009C88AD88BE88680D791D8A1D9B1D809058
:10CFC000760F9090770FA090780FB090790F68153A
:10CFD00079058A059B0581F48F89803191F4DD24E0
:10CFE000EE24FF24F601EE0FFF1FEA58F24F808176
:10CFF0009181A0E0B0E016C040E070DF8111ECCF7D
:10D00000C1CFE894C7F8DD24EE24FF24F601EE0F2B
:10D01000FF1FEE0FFF1FEA58F24F80819181A2811E
:10D02000B381BF70F80180839183A283B38381E0D1
:10D03000DF91CF911F910F91FF90EF90DF90CF90F4
:10D04000BF90AF909F908F9008954F925F926F9294
:10D050007F92AF92BF92CF92DF92EF92FF920F93A7
:10D060001F93CF93DF9300D01F92CDB7DEB78C0113
:10D0700049835A836B837C835901C12CD12C76015F
:10D08000412C42E0542E612C712C49815A816B81D4
:10D090007C819E012F5F3F4FC80158DF882341F1FB
:10D0A000D301C201F801058404C0880F991FAA1F8B
:10D0B000BB1F0A94D2F7C80ED91EEA1EFB1E498177
:10D0C0005A816B817C818789803139F481E0483FC6
:10D0D0005F4F6105710538F4D8CF81E0483F5F4F5D
:10D0E0006F4F7F4090F2F501C082D182E282F382DD
:10D0F0000F900F900F900F90DF91CF911F910F9194
:10D10000FF90EF90DF90CF90BF90AF907F906F90A7
:10D110005F904F9008954F925F926F927F928F929F
:10D120009F92AF92BF92CF92DF92EF92FF920F93B6
:10D130001F93CF93DF93EC014A015B012801390172
:10D14000423051056105710508F462C049855A8570
:10D150006B857C854F5F5F4F6F4F7F4F481559053B
:10D160006A057B0508F454C08F89803129F4FF24B7
:10D17000EB2CDA2CC92C0CC0803209F049C07501A7
:10D18000640177E0F694E794D794C7947A95D1F741
:10D190004B895C896D897E89C40ED51EE61EF71EFB
:10D1A00041E0C701B6019ADE882391F19F89903151
:10D1B00059F49924AA24BB24F401EE0FFF1FEA5866
:10D1C000F24F5182408210C0E89487F89924AA2433
:10D1D000BB24F401EE0FFF1FEE0FFF1FEA58F24FC2
:10D1E00040825182628273829A89923090F04D819E
:10D1F0005E816F8178854C0D5D1D6E1D7F1D409396
:10D200006F0D5093700D6093710D7093720D01C08E
:10D2100080E0DF91CF911F910F91FF90EF90DF9011
:10D22000CF90BF90AF909F908F907F906F905F90C6
:10D230004F9008952F923F924F925F926F927F92FC
:10D240008F929F92AF92BF92CF92DF92EF92FF9216
:10D250000F931F93CF93DF93CDB7DEB72F970FB602
:10D26000F894DEBF0FBECDBF1C014C875D876E8773
:10D270007F873B872A87DC0119960D911D912D919F
:10D280003C911C970F5F1F4F2F4F3F4F0D831E8305
:10D290002F833887EA85FB8580809180A280B380C8
:10D2A00081149104A104B10431F0FFEF8F1A9F0A99
:10D2B000AF0ABF0A10C0DC018D909D90AD90BC906C
:10D2C000B1E0B9870C851D852E853F85013011059C
:10D2D0002105310509F0198675016401412C512C95
:10D2E0003201F10181859285A385B48548165906DE
:10D2F0006A067B0608F04EC00D811E812F8138859D
:10D300000C151D052E053F0550F4F2E0CF2ED12C53
:10D31000E12CF12CA2E08A2E912CA12CB12C9E01A3
:10D320002F5F3F4FB701A601C10110DE882391F1A5
:10D3300049815A816B817C81D701C6010196A11D6B
:10D34000B11D452B462B472B19F04C015D010FC039
:10D35000AC01BD01481959096A097B090C851D8575
:10D360002E853F85401751076207730741F01FEF75
:10D37000411A510A610A710A6C017D01B2CF0FEFA7
:10D380001FEF2FEF3FE0B701A601C101C4DE8D837F
:10D39000811113C01D823DC02601370121E0421AD0
:10D3A00051086108710897018601B301A201C1010A
:10D3B000B2DE882379F3730162018C149D04AE04FC
:10D3C000BF0450F3AA85BB854D915D916D917C9111
:10D3D0004115510561057105A9F4EA85FB85808237
:10D3E0009182A282B382F985FF2399F00FEF801A10
:10D3F000900AA00AB00AD1018D929D92AD92BC9282
:10D40000139707C095018401C10185DE8111E5CF25
:10D41000C1CF8D812F960FB6F894DEBF0FBECDBF62
:10D42000DF91CF911F910F91FF90EF90DF90CF9000
:10D43000BF90AF909F908F907F906F905F904F9034
:10D440003F902F900895AF92BF92CF92DF92EF92CC
:10D45000FF920F931F93CF93DF9300D01F92CDB70E
:10D46000DEB75C016A017B0182E090E0A0E0B0E001
:10D47000F50180839183A283B3839E012F5F3F4F89
:10D48000B701A601C50162DD811102C080E023C0A1
:10D4900000E010E09801B701A601C5013CDE882339
:10D4A000A9F3C980DA80EB80FC80F501878980319F
:10D4B00049F481E0F8EFCF16FFEFDF06E104F10455
:10D4C00050F4DBCF81E098EFC9169FEFD906E9064B
:10D4D0009FE0F90690F20F900F900F900F90DF9160
:10D4E000CF911F910F91FF90EF90DF90CF90BF9061
:10D4F000AF9008957F928F929F92AF92BF92CF92FA
:10D50000DF92EF92FF920F931F93CF93DF93EC0183
:10D51000142F7093750D6093740D1F8A82E090E054
:10D52000A0E0B0E088839983AA83BB831092730D37
:10D5300010926F0D1092700D1092710D1092720D6D
:10D540008FEF9FEFDC018093760F9093770FA0937E
:10D55000780FB093790F442349F1453008F0DEC0CD
:10D5600040E060E070E0CB01B9DC882309F4D6C06C
:10D5700020E1129FF0011124EC5DF04F80818F7744
:10D5800009F0CCC084859585A685B785843691053C
:10D59000A105B10508F4C2C0C084D184E284F3843B
:10D5A000C114D104E104F10421F4B8C0C12CD12C80
:10D5B000760140E0C701B60191DC782E882309F49A
:10D5C000ADC08091810D9091820D8115924009F03E
:10D5D000A5C03091860D332309F4A0C08091840D3D
:10D5E0009091850D892B09F499C02091830D2223F8
:10D5F00009F494C03A8B2C831D8630E041E050E062
:10D600006D85062FCA01062E02C0880F991F0A9445
:10D61000E2F72817390731F081E0860F8D876830EF
:10D6200078F37CC020918C0D30918D0D2115310542
:10D6300019F040E050E008C020919A0D30919B0D08
:10D6400040919C0D50919D0D2D833E834F835887B3
:10D650008091840D9091850D46015701880E991E89
:10D66000A11CB11C8B8A9C8AAD8ABE8AE091870D71
:10D67000F091880DF98FE88FA091860DB0E00E949F
:10D680005A76680D791D8A1D9B1D6A8F7B8F8C8F42
:10D690009D8FB5E0EE0FFF1FBA95E1F7E150FE4F09
:10D6A000EF2FFF27E695DC01CB018E0F9F1FA11DF9
:10D6B000B11D8E879F87A88BB98B8090890D909024
:10D6C0008A0D8114910419F0A12CB12C08C080900E
:10D6D000960D9090970DA090980DB090990DA70180
:10D6E0009601281B390B4A0B5B0BDA01C901880D27
:10D6F000991DAA1DBB1D04C0B695A7959795879542
:10D700000A95D2F789879A87AB87BC87853F3FE028
:10D710009307A105B10520F48CE08F8B712C15C007
:10D72000853F9F4FA105B10510F480E10DC08091A8
:10D73000A20D9091A30DA091A40DB091A50D8A8F7B
:10D740009B8FAC8FBD8F80E28F8B872DDF91CF9128
:10D750001F910F91FF90EF90DF90CF90BF90AF900F
:10D760009F908F907F9008952F923F924F925F925B
:10D770006F927F928F929F92AF92BF92CF92DF92E1
:10D78000EF92FF920F931F93CF93DF93CDB7DEB746
:10D79000C454D1090FB6F894DEBF0FBECDBF3C0113
:10D7A0001B014A012FA309A7EBA62196ACAEBDAE83
:10D7B000CEAEDFAE219734E0239F20011124440D2B
:10D7C000551D5AAB49ABDA01CD90DD90ED90FC9040
:10D7D000FC01E40DF51D2081318142815381C70197
:10D7E000B6018ED56BAB7CAB8DAB9EABB4E00B9F23
:10D7F00080011124F401E00FF11FF8AFEFAB80803E
:10D800009180A280B380F301E00FF11F208131816C
:10D8100042815381C501B40173D569AF7AAF8BAF33
:10D820009CAF2BA5F4E02F9FC0011124F301E80F5A
:10D83000F91F2081318142815381298F3A8F4B8F8B
:10D840005C8FF101E80FF91F608171818281938102
:10D8500056D56F8F78A389A39AA3D1011C968D9179
:10D860009D910D90BC91A02D8DA79EA7AFA7B8ABA1
:10D87000D3011C962D913D914D915C911F972BA347
:10D880003CA34DA35EA3A701960150582D8B3E8B60
:10D890004F8B588FD501C401B058898B9A8BAB8BB5
:10D8A000BC8BF101E40DF51D2BA93CA94DA95EA986
:10D8B000608171818281938122D56B017C01F101AC
:10D8C000E00FF11F29AD3AAD4BAD5CAD60817181C8
:10D8D0008281938114D54B015C01A70196016D896A
:10D8E0007E898F89988D0E942E752B013C01A501A0
:10D8F000940169897A898B899C890E942E759B0184
:10D90000AC01C301B201FCD42B013C01A50194017F
:10D910006D897E898F89988D0E942E754B015C01DF
:10D92000A701960169897A898B899C890E942E7545
:10D930009B01AC01C501B401E2D4A301920153D50E
:10D940006B017C0120E030E0A901B3D587FF09C05D
:10D950002BED3FE049EC50E4C701B601D1D46B0197
:10D960007C016F968FAD6F97882349F02BED3FE0D8
:10D9700049EC50E4C701B601C2D46B017C016E963C
:10D980002CAD3DAD4EAD5FAD6E97C701B6010E94A7
:10D990002E752F8D38A149A15AA15F779AD74B01D7
:10D9A0005C012FE632E143E85AE383D587FDAAC143
:10D9B000C501B4015BD6F1D57E8F6D8FDB01AB2B3A
:10D9C00021F4E1E0F0E0FE8FED8F2D8D3E8DB90169
:10D9D00080E090E00ED64B015C019B01AC01C701D9
:10D9E000B6016ED52B013C01A50194016F8D78A184
:10D9F00089A19AA165D525966CAF7DAF8EAF9FAFFB
:10DA000025972BA13CA14DA15EA16DA57EA58FA55B
:10DA100098A975D4A501940153D56DA77EA78FA7AA
:10DA200098AB20E030E040E05FE3C301B2010E9428
:10DA30002E75A30192010E942E759B01AC0160E03E
:10DA400070E080E89FE35BD46F8F78A389A39AA3EB
:10DA5000CE010196FC014BA534E0439FE00DF11D82
:10DA60001124298D3A8D4B8D5C8D20833183428327
:10DA700053832BA13CA14DA15EA12D873E874F87EB
:10DA8000588BB12C41E050E05A8F498F81E090E0F3
:10DA90008C0F9D1FBFA1A4E0BA9F800D911D112482
:10DAA0009CA78BA721E030E02C0F3D1F59A544E037
:10DAB000549F200D311D11243AA729A7F8A7EFA3E1
:10DAC000498D5A8D8D8D9E8D4817590708F004C1D8
:10DAD00088E18B150CF43EC02F8D38A149A15AA1C5
:10DAE00069897A898B899C89B9D76B017C01A301EB
:10DAF00092016D897E898F89988DB0D7A701960193
:10DB0000FFD3A62E172F982E892E2F8D38A149A12D
:10DB10005AA16D897E898F89988DA0D76B017C0170
:10DB2000A301920169897A898B899C8997D79B0186
:10DB3000AC01C701B601E3D36D8B7E8B8F8B988FC1
:10DB4000B3948A2D912FA92DB82D898B9A8BAB8BED
:10DB5000BC8B60C0A98DBA8DBD0180E090E049D535
:10DB6000A30192017BD76B017C01A7D4698B7A8BCF
:10DB70008B8B9C8BC701B601D4D74B015C01E9A903
:10DB8000FAA9C080D180E280F380F7FAF094F7F828
:10DB9000F094AFA9B8AD2D913D914D915C912BA31F
:10DBA0003CA34DA35EA329893A894B895C89C701AF
:10DBB000B60154D76D8B7E8B8F8B988FA501940106
:10DBC0006BA17CA18DA19EA149D79B01AC016D8960
:10DBD0007E898F89988D94D36D8B7E8B8F8B988F58
:10DBE000A5019401C701B60139D76B017C012989D0
:10DBF0003A894B895C896BA17CA18DA19EA12ED70E
:10DC00009B01AC01C701B6017AD3698B7A8B8B8BF0
:10DC10009C8BB12C2D893E894F89588D6BA97CA98D
:10DC20008DA99EA96DD3EBA5FCA56083718382832A
:10DC3000938329893A894B895C8969AD7AAD8BAD2B
:10DC40009CAD5ED3A9A5BAA56D937D938D939C934E
:10DC5000139725962CAD3DAD4EAD5FAD2597EFA149
:10DC6000F8A560817181828193814AD3AFA1B8A563
:10DC70006D937D938D939C9313972DA53EA54FA5F2
:10DC800058A96D857E858F8598893AD36D877E8763
:10DC90008F87988BCE0101960E94631DFE01E15A89
:10DCA000FF4F6F012196ECACFDAC0EAD1FAD21977F
:10DCB0009E01235F3F4FAE01475F5F4FBE016B5F29
:10DCC0007F4FCE0101960E94253B298D3A8D2F5F13
:10DCD0003F4F3A8F298FF4CE9101245F3F4FA1012E
:10DCE000485F5F4FB1016C5F7F4FDE01A15ABF4FAC
:10DCF0006D012196ECACFDAC0EAD1FAD2197C101BD
:10DD00000E94253BCC5BDF4F0FB6F894DEBF0FBE01
:10DD1000CDBFDF91CF911F910F91FF90EF90DF90DA
:10DD2000CF90BF90AF909F908F907F906F905F90BB
:10DD30004F903F902F90089561E085E34FD261E0CE
:10DD400085E313D28CB580618CBD8CB580648CBDAD
:10DD500061E084E30AD261E083E307C21F93CF93BB
:10DD6000DF93182FEB0161E000D2209711F460E0FF
:10DD700004C0CF3FD10531F461E0812FDF91CF9115
:10DD80001F912CC2E12FF0E0EB5FFB4E449150E07D
:10DD9000FA013197E131F10508F090C0E658FF4FE4
:10DDA00083C784B5806884BDC7BD8DC084B58062DB
:10DDB00084BDC8BD88C08091800080688093800049
:10DDC000D0938900C09388007EC0809180008062DB
:10DDD00080938000D0938B00C0938A0074C08091A0
:10DDE000B00080688093B000C093B3006CC0809195
:10DDF000B00080628093B000C093B40064C0809192
:10DE00009000806880939000D0939900C093980010
:10DE10005AC080919000806280939000D0939B00C4
:10DE2000C0939A0050C080919000886080939000C9
:10DE3000D0939D00C0939C0046C08091A000806854
:10DE40008093A0008091A0008F7B8093A000D0934E
:10DE5000A900C093A80037C08091A0008062809381
:10DE6000A000D093AB00C093AA002DC08091A00069
:10DE700088608093A000D093AD00C093AC0023C015
:10DE800080912001806880932001D0932901C09364
:10DE9000280119C080912001806280932001D093D5
:10DEA0002B01C0932A010FC08091200188608093CC
:10DEB0002001D0932D01C0932C0105C0C038D1059D
:10DEC0000CF05ACF54CFDF91CF911F9108951F923C
:10DED0000F920FB60F9211242F933F938F939F931E
:10DEE000AF93BF9380917B0F90917C0FA0917D0F9A
:10DEF000B0917E0F30917A0F23E0230F2D3720F45D
:10DF00000196A11DB11D05C026E8230F0296A11D93
:10DF1000B11D20937A0F80937B0F90937C0FA09379
:10DF20007D0FB0937E0F80917F0F9091800FA09115
:10DF3000810FB091820F0196A11DB11D80937F0FBB
:10DF40009093800FA093810FB093820FBF91AF91F8
:10DF50009F918F913F912F910F900FBE0F901F9027
:10DF600018952FB7F89460917B0F70917C0F80917A
:10DF70007D0F90917E0F2FBF08953FB7F894809149
:10DF80007F0F9091800FA091810FB091820F26B5E5
:10DF9000A89B05C02F3F19F00196A11DB11D3FBFE1
:10DFA0006627782F892F9A2F620F711D811D911D71
:10DFB00042E0660F771F881F991F4A95D1F7089591
:10DFC000CF92DF92EF92FF92CF93DF936B017C01B0
:10DFD000D4DFEB01C114D104E104F10471F0CDDF11
:10DFE0006C1B7D0B683E7340A8F381E0C81AD10812
:10DFF000E108F108C851DC4FEDCFDF91CF91FF90E0
:10E00000EF90DF90CF900895789484B5826084BDBE
:10E0100084B5816084BD85B5826085BD85B581602C
:10E0200085BDEEE6F0E0808181608083E1E8F0E08C
:10E030001082808182608083808181608083E0E8BB
:10E04000F0E0808181608083E1EBF0E0808184609A
:10E050008083E0EBF0E0808181608083E1E9F0E0A3
:10E06000808182608083808181608083E0E9F0E04C
:10E07000808181608083E1EAF0E08081826080833A
:10E08000808181608083E0EAF0E08081816080832C
:10E09000E1E2F1E080818260808380818160808321
:10E0A000E0E2F1E0808181608083EAE7F0E0808156
:10E0B00084608083808182608083808181608083AE
:10E0C0008081806880831092C100089590E0FC01F7
:10E0D0003197E131F10508F047C0E557FF4FE4C53E
:10E0E000809180008F7703C0809180008F7D809326
:10E0F0008000089584B58F7702C084B58F7D84BD7C
:10E1000008958091B0008F7703C08091B0008F7D1B
:10E110008093B0000895809190008F7707C0809120
:10E1200090008F7D03C080919000877F8093900046
:10E1300008958091A0008F7707C08091A0008F7D07
:10E1400003C08091A000877F8093A00008958091F4
:10E1500020018F7707C0809120018F7D03C08091BF
:10E160002001877F809320010895CF93DF9390E073
:10E17000FC01E55BFB4E2491FC01EF56FB4E8491C4
:10E18000882349F190E0880F991FFC01E55FFA4E62
:10E19000A591B4918F509B4EFC01C591D4919FB72E
:10E1A000611108C0F8948C91209582238C9388810A
:10E1B00082230AC0623051F4F8948C91322F30954A
:10E1C00083238C938881822B888304C0F8948C915C
:10E1D000822B8C939FBFDF91CF9108950F931F9354
:10E1E000CF93DF931F92CDB7DEB7282F30E0F90130
:10E1F000EB5FFB4E8491F901E55BFB4E1491F90155
:10E20000EF56FB4E04910023C1F0882319F0698377
:10E210005DDF6981E02FF0E0EE0FFF1FEF50FB4E56
:10E22000A591B4919FB7F8948C91611103C010959A
:10E23000812301C0812B8C939FBF0F90DF91CF91E1
:10E240001F910F910895CF93DF93282F30E0F901AC
:10E25000EB5FFB4E8491F901E55BFB4ED491F90134
:10E26000EF56FB4EC491CC2389F081112FDFEC2FA8
:10E27000F0E0EE0FFF1FE952FB4EA591B4912C91F7
:10E280002D2381E090E021F480E002C080E090E066
:10E29000DF91CF910895CF92DF92EF92FF920F938B
:10E2A0001F93CF93DF936C017A01EB01E60EF71E0B
:10E2B00000E010E0CE15DF0561F06991D601ED9127
:10E2C000FC910190F081E02DC6011995080F191FEE
:10E2D000F1CFC801DF91CF911F910F91FF90EF9087
:10E2E000DF90CF90089590DE0E94FB23C0E0D0E045
:10E2F0000E942F352097E1F30E940000F9CF50587B
:10E30000BB27AA270ED076C23FD230F044D220F0ED
:10E3100031F49F3F11F41EF40FC20EF4E095E7FBB9
:10E32000DCC1E92F89D280F3BA176207730784072B
:10E33000950718F071F49EF5B8C20EF4E0950B2E17
:10E34000BA2FA02D0B01B90190010C01CA01A00147
:10E350001124FF27591B99F0593F50F4503E68F1A2
:10E360001A16F040A22F232F342F4427585FF3CFE3
:10E37000469537952795A795F0405395C9F77EF4B4
:10E380001F16BA0B620B730B840BBAF09150A1F0FD
:10E39000FF0FBB1F661F771F881FC2F70EC0BA0F83
:10E3A000621F731F841F48F4879577956795B7950B
:10E3B000F7959E3F08F0B3CF9395880F08F0992703
:10E3C000EE0F979587950895DFD158F080E891E09A
:10E3D00009F49EEFE0D128F040E851E059F45EEFF7
:10E3E00009C0AAC162C2E92FE07826D268F3092EDB
:10E3F000052AC1F3261737074807590738F00E2EAC
:10E4000007F8E02569F0E025E0640AC0EF6307F84B
:10E41000009407FADB01B9019D01DC01CA01AD01DD
:10E42000EF935DD0E7D10AD05F91552331F02BED0A
:10E430003FE049E450FD49EC63CF0895DF93DD27C9
:10E44000B92FBF7740E85FE31616170648075B074A
:10E4500010F4D92F96D29F938F937F936F93A9D364
:10E46000E8E3F1E06CD1C6D12F913F914F915F91DC
:10E4700001D3DD2349F09058A2EA2AED3FE049ECB0
:10E480005FE3D0785D274DDFDF91B4C1F7D180F035
:10E490009F3740F491110EF409C260E070E080E80B
:10E4A0009FE3089526F01B16611D711D811D1BC180
:10E4B00035C1EFD008F481E0089575D1E395ABC183
:10E4C0000CD098C168D140F05FD130F021F45F3FAB
:10E4D00019F003C15111EAC12FC1AED198F39923AC
:10E4E000C9F35523B1F3951B550BBB27AA27621718
:10E4F0007307840738F09F5F5F4F220F331F441F5D
:10E50000AA1FA9F333D00E2E3AF0E0E830D0915094
:10E510005040E695001CCAF729D0FE2F27D0660F81
:10E52000771F881FBB1F261737074807AB07B0E8C0
:10E5300009F0BB0B802DBF01FF2793585F4F2AF0D6
:10E540009E3F510568F0C9C0B1C15F3FECF3983EF2
:10E55000DCF3869577956795B795F7959F5FC9F733
:10E56000880F911D9695879597F90895E1E0660FBC
:10E57000771F881FBB1F621773078407BA0720F035
:10E58000621B730B840BBA0BEE1F88F7E09508959E
:10E5900004D06894B1118AC1089556D188F09F576C
:10E5A00090F0B92F9927B751A0F0D1F0660F771FDF
:10E5B000881F991F1AF0BA95C9F712C0B13081F0BF
:10E5C00074D1B1E0089571C1672F782F8827B85FA3
:10E5D00039F0B93FCCF3869577956795B395D9F720
:10E5E0003EF490958095709561957F4F8F4F9F4F2A
:10E5F0000895E89409C097FB3EF490958095709536
:10E6000061957F4F8F4F9F4F9923A9F0F92F96E97E
:10E61000BB279395F695879577956795B795F111F3
:10E62000F8CFFAF4BB0F11F460FF1BC06F5F7F4F90
:10E630008F4F9F4F16C0882311F096E911C07723A2
:10E6400021F09EE8872F762F05C0662371F096E8AB
:10E65000862F70E060E02AF09A95660F771F881F7A
:10E66000DAF7880F9695879597F9089507D180F086
:10E670009F3740F491110EF019C160E070E080E81E
:10E680009FEB089526F41B16611D711D811D2BC083
:10E6900045C0990F0008550FAA0BE0E8FEEF1616CB
:10E6A0001706E807F907C0F012161306E407F50786
:10E6B00098F0621B730B840B950B39F40A2661F0FA
:10E6C000232B242B252B21F408950A2609F4A1409D
:10E6D000A6958FEF811D811D089597F99F6780E8AA
:10E6E00070E060E00895882371F4772321F098505A
:10E6F000872B762F07C0662311F499270DC0905100
:10E70000862B70E060E02AF09A95660F771F881FCD
:10E71000DAF7880F9695879597F908959F3F31F01E
:10E72000915020F4879577956795B795880F911D3F
:10E730009695879597F908959FEF80EC0895DF935C
:10E74000CF931F930F93FF92EF92DF927B018C0187
:10E75000689405C0DA2EEF018DD1FE01E894A591F1
:10E760002591359145915591AEF3EF01DADDFE012A
:10E770009701A801DA9479F7DF90EF90FF900F915D
:10E780001F91CF91DF91089500240A941616170661
:10E7900018060906089500240A9412161306140692
:10E7A00005060895C9CF50D0E8F3E894E0E0BB2710
:10E7B0009F57F0F02AED3FE049EC06C0EE0FBB0F8B
:10E7C000661F771F881F28F0B23A62077307840715
:10E7D00028F0B25A620B730B840BE3959A9572F78B
:10E7E000803830F49A95BB0F661F771F881FD2F7C9
:10E7F000904896CF092E0394000C11F4882352F010
:10E80000BB0F40F4BF2B11F460FF04C06F5F7F4F5C
:10E810008F4F9F4F0895EF93E0FF06C0A2EA2AEDC5
:10E820003FE049EC5FEB7DDDE5DF0F90039401FCF9
:10E830009058E5E6F1E0C7C157FD9058440F551FC9
:10E8400059F05F3F71F04795880F97FB991F61F072
:10E850009F3F79F087950895121613061406551FE9
:10E86000F2CF4695F1DF08C0161617061806991F55
:10E87000F1CF86957105610508940895E5DFA0F054
:10E88000BEE7B91788F4BB279F3860F41616B11D90
:10E89000672F782F8827985FF7CF869577956795AC
:10E8A000B11D93959639C8F30895E894BB27662760
:10E8B0007727CB0197F90895ECDE08F48FEF0895E0
:10E8C00063DF19F068DF09F037CF07CFB901CA015C
:10E8D00025CF9F775F77B0DF98F39923B9F355235E
:10E8E000B9F3FF27951758F4E52FE91BED3070F7C2
:10E8F0005E3B10F0F1E41CC09034E0F40AC0E92F54
:10E90000E51BED3028F79E3B10F0F1E411C05034C8
:10E9100088F4F9EA88232AF09A95660F771F881FF2
:10E92000DAF744232AF05A95220F331F441FDAF7EF
:10E930009F1B5F1BFF931F930F93FF92EF92790131
:10E940008A01BB27AB2F9B01AC0196D09701A80190
:10E95000BF937B018C01AA27BA2FB901CA018CD0C1
:10E96000AF919701A801EF90FF900F911F91D9DC13
:10E9700041DFE1D04F9140FF0895552747FD509565
:10E9800009C09B01AC0160E070E080E89FE398CD96
:10E99000A4CEC4CE59DFE8F39923D9F3940F511DC7
:10E9A000BBF39150504094F059F0882332F0660F39
:10E9B000771F881F91505040C1F79E3F510544F783
:10E9C000880F911D9695879597F908955F3FACF054
:10E9D000983E9CF0BB27869577956795B79508F488
:10E9E000B1609395C1F7BB0F58F711F460FFE8CF02
:10E9F0006F5F7F4F8F4F9F4FE3CF58CF25DF58F189
:10EA00009E5758F19851A0F0E9F0983020F5092E62
:10EA10009927660F771F881F991F0A94D1F712C094
:10EA2000062E672F782F8827985F11F4000C07C0F7
:10EA3000993FB4F38695779567959395D9F7611DBE
:10EA4000711D811D3EF490958095709561957F4F65
:10EA50008F4F9F4F0895689429CF27CF0BD0CACEF0
:10EA600093DE28F098DE18F0952309F036CE64CEB8
:10EA700011241CCFE1DEA0F3959FD1F3950F50E058
:10EA8000551F629FF001729FBB27F00DB11D639F60
:10EA9000AA27F00DB11DAA1F649F6627B00DA11D06
:10EAA000661F829F2227B00DA11D621F739FB00DAC
:10EAB000A11D621F839FA00D611D221F749F33271C
:10EAC000A00D611D231F849F600D211D822F762FB5
:10EAD0006A2F11249F5750408AF0E1F088234AF0B2
:10EAE000EE0FFF1FBB1F661F771F881F91505040FE
:10EAF000A9F79E3F510570F0F0CDD8CE5F3FECF303
:10EB0000983EDCF3869577956795B795F795E795E9
:10EB10009F5FC1F7FE2B880F911D9695879597F9FA
:10EB200008959F9340DE0F9007FCEE5F74CE11F4C2
:10EB30000EF402CEF3CD88DED0F39923D9F3CEF3D1
:10EB40009F57550B87FF38D00024A0E640EA90017C
:10EB500080585695979528F4805C660F771F881F1C
:10EB600020F026173707480730F4621B730B840B1D
:10EB7000202931294A2BA695179407942025312561
:10EB80004A2758F7660F771F881F20F02617370788
:10EB9000480730F4620B730B840B200D311D411DAF
:10EBA000A09581F7B901842F9158880F9695879584
:10EBB00008959B01AC0152CF91505040660F771FD2
:10EBC000881FD2F708959F938F937F936F93FF933E
:10EBD000EF939B01AC0142DFEF91FF91B0DD2F91EC
:10EBE0003F914F915F913ACFDB018F939F9362D01A
:10EBF000BF91AF91A29F800D911DA39F900DB29FD9
:10EC0000900D1124089597FB072E16F4009406D05A
:10EC100077FD08D063D007FC05D03EF49095819530
:10EC20009F4F0895709561957F4F0895A1E21A2E28
:10EC3000AA1BBB1BFD010DC0AA1FBB1FEE1FFF1FA0
:10EC4000A217B307E407F50720F0A21BB30BE40BF0
:10EC5000F50B661F771F881F991F1A9469F7609537
:10EC60007095809590959B01AC01BD01CF010895F1
:10EC7000052E97FB16F400940FD057FD05D0D6DF74
:10EC800007FC02D046F408C0509540953095219578
:10EC90003F4F4F4F5F4F08959095809570956195C8
:10ECA0007F4F8F4F9F4F0895EE0FFF1F0590F491F8
:10ECB000E02D199427D0A59F900DB49F900DA49F8F
:10ECC000800D911D11240895B7FFF4CFF3DF821B4F
:10ECD000930B08950790F691E02D1994AA1BBB1B86
:10ECE00051E107C0AA1FBB1FA617B70710F0A61B4C
:10ECF000B70B881F991F5A95A9F780959095BC016D
:10ED0000CD010895A29FB001B39FC001A39F700DD4
:10ED1000811D1124911DB29F700D811D1124911D23
:10ED200008958F929F92AF92BF92CF92DF92EF920F
:10ED3000FF920F931F93CF93DF938B0161157105A2
:10ED400021F0DB018C9311969C93EC015E01BFEFE7
:10ED5000AB1ABB0A7501C8808C2D90E07BD2892B41
:10ED600011F0E501F3CFEDE2CE1208C07E01F2E032
:10ED7000EF0EF11CC980DD24D39409C02BE2C2122E
:10ED800005C07E0142E0E40EF11CC980D12CE701F0
:10ED9000219743E050E06DE275E1CE016BD2892B03
:10EDA000B9F4239645E050E068E275E1CE0162D205
:10EDB000892B09F425960115110519F0D801CD9379
:10EDC000DC93D11000C160E070E080E89FE704C1EF
:10EDD00043E050E065E275E1CE014CD2892B59F455
:10EDE0000115110509F4F4C0B2E0EB0EF11CF801B5
:10EDF000F182E082EDC0F70160E070E0CB01C0E09D
:10EE0000D0E07F01A0EDAA2EAC0C29E02A1528F154
:10EE10004D2D4260B42E2D2D2870D2FE04C021113C
:10EE200024C0219622C021112197A5E0B0E09B01CA
:10EE3000AC0140DF660F771F881F991F6A0D711D97
:10EE4000811D911D6839A9E97A078A07A9E19A0706
:10EE500060F0BD2DB660BB2E08C02EEFA2120AC016
:10EE6000D3FC50C04D2D4860B42E3196D701CC90C4
:10EE7000DB2CC7CF2C2D2F7D253409F043C0A0817A
:10EE8000AD3241F4BD2DB061DB2E7F0122E0E20EF8
:10EE9000F11C0CC07F01AB3231F04FEFE41AF40AE1
:10EEA00021E030E006C0A2E0EA0EF11CA18122E0E0
:10EEB00030E0A053AA3018F0E21AF30A23C0F70199
:10EEC00020E030E02038BCE03B075CF4A901440FAF
:10EED000551F440F551F240F351F220F331F2A0FB4
:10EEE000311DAF014F5F5F4F7A01A081A053AA305F
:10EEF00010F4FA01E7CFD4FE03C031952195310912
:10EF0000C20FD31FD1FE09C00115110531F0E1E098
:10EF1000EE1AF108D801ED92FC926BDB2D2D2370D7
:10EF2000233019F04B015C0106C04B015C01B7FABC
:10EF3000B094B7F8B09420E030E0A901C501B40165
:10EF4000B8DA882309F43CC0D7FF06C0D195C19533
:10EF5000D10904E415E102C00CE515E16801B8E14E
:10EF6000CB1AD10890E2E92EF12CCE15DF056CF01A
:10EF7000F8012591359145915491C501B4016EDD9B
:10EF80004B015C01CE19DF09F0CF04501109F59453
:10EF9000E7940C151D0549F78A2D880F8B2D881FC6
:10EFA0008F3F41F020E030E0A901C501B40181DAD2
:10EFB000811106C082E290E09093880F8093870FC2
:10EFC000C501B40109C060E070E080E89FEF04C0B3
:10EFD00060E070E080EC9FE7DF91CF911F910F918F
:10EFE000FF90EF90DF90CF90BF90AF909F908F9069
:10EFF00008952F923F925F926F927F928F929F928D
:10F00000AF92BF92CF92DF92EF92FF920F931F9336
:10F01000CF93DF938B01EA016115710521F0DB01CC
:10F020008C9311969C93209739F09E0122503109C0
:10F030002332310508F0F8C07C016701BFEFCB1A1D
:10F04000DB0A5601F7016080862D90E003D1892B01
:10F0500011F07601F2CFFDE26F120AC0570182E093
:10F06000A80EB11CD70111966C90772473940BC035
:10F07000BBE26B1207C05701E2E0AE0EB11CD70134
:10F0800011966C90712CCE018F7E892B89F4B0E3A0
:10F090006B1222C0F50180818F7D883541F561803A
:10F0A000F2E0AF0EB11C872D8260782EC0E1D0E077
:10F0B000C830D105F1F04CF4C230D10511F5C12CA6
:10F0C000D12CE12CB0E4FB2E2EC0CA30D10531F09A
:10F0D000C031D10519F115C0209751F7CAE0D0E031
:10F0E000ACECCA2EDC2CEC2CACE0FA2E1CC0209729
:10F0F000F9F6C8E0D0E0C12CD12CE12CF0E1FF2ED4
:10F1000012C060E070E080E090E89E01442737FD87
:10F110004095542F8BDD69017A0105C0C12CD12C9B
:10F12000E12CE8E0FE2EF50160E020E030E0A901EE
:10F130004E01AA2497FCA094BA2C1F0170ED572E03
:10F14000560CA9E0A51570F48FEB860D8A3118F4E2
:10F1500099EC592E06C08FE9860D8A3128F589EA87
:10F16000582E560C852D90E08C179D07ECF467FD0A
:10F1700017C0C216D306E406F50678F0C501B4013F
:10F1800033DD9B01AC01250D311D411D511D213089
:10F1900031054105B0E85B0710F06FEF01C061E099
:10F1A0003196D1016C90C9CF872D81700115110561
:10F1B00071F0662329F03197D801ED93FC9307C0D5
:10F1C00071FE19C03297D801ED93FC9314C067FF0C
:10F1D00012C0882329F020E030E040E050E804C06D
:10F1E0002FEF3FEF4FEF5FE782E290E09093880FC1
:10F1F0008093870F16C0882341F050954095309535
:10F2000021953F4F4F4F5F4F0CC057FF0AC082E21E
:10F2100090E09093880F8093870F2FEF3FEF4FEF91
:10F220005FE7B901CA0104C060E070E080E090E0EF
:10F23000DF91CF911F910F91FF90EF90DF90CF90D2
:10F24000BF90AF909F908F907F906F905F903F9016
:10F250002F9008959111C2C2803219F089508550C3
:10F26000D0F708959111089581548A5108F4805E71
:10F27000855A0895FB01DC014150504088F08D9182
:10F2800081341CF08B350CF4805E659161341CF088
:10F290006B350CF4605E861B611171F3990B089558
:10F2A000881BFCCFFB01DC0104C08D91019080190B
:10F2B00021F441505040C8F7881B990B0895FB0179
:10F2C000DC0102C001900D9241505040D8F70895E2
:10F2D000FB01DC010D900020E9F7119701900D92E0
:10F2E0000020E1F70895FC018191861721F0882321
:10F2F000D9F7992708953197CF010895FB01DC01D3
:10F3000001900D920020E1F70895FB01DC014150CE
:10F31000504030F08D910190801919F40020B9F718
:10F32000881B990B0895FB01DC014150504048F0C7
:10F3300001900D920020C9F701C01D92415050402C
:10F34000E0F70895FB0151915523A9F0BF01DC01BD
:10F350004D9145174111E1F759F4CD01019000207D
:10F3600049F04D9140154111C9F3FB014111EFCF17
:10F3700081E090E0019708950F931F93CF93DF935F
:10F38000CDB7DEB72E970FB6F894DEBF0FBECDBF58
:10F390000E891F8986E08C831A8309838FEF9FE78C
:10F3A0009E838D83AE01465E5F4F688D798DCE0161
:10F3B000019610D0EF81F885E00FF11F10822E9694
:10F3C0000FB6F894DEBF0FBECDBFDF91CF911F9176
:10F3D0000F9108952F923F924F925F926F927F927A
:10F3E0008F929F92AF92BF92CF92DF92EF92FF9255
:10F3F0000F931F93CF93DF93CDB7DEB72C970FB644
:10F40000F894DEBF0FBECDBF7C016B018A01FC0109
:10F4100017821682838181FFB0C1CE0101964C0113
:10F42000F7019381F60193FD859193FF81916F011F
:10F43000882309F49EC1853239F493FD859193FFA9
:10F4400081916F01853221F4B70190E0E0D1E8CFDE
:10F45000512C312C20E02032A0F48B3269F030F4B2
:10F46000803259F0833269F420612CC08D3239F03A
:10F47000803339F4216026C02260246023C02860D4
:10F4800021C027FD27C030ED380F3A3078F426FF31
:10F4900006C0FAE05F9E300D1124532E13C08AE09F
:10F4A000389E300D1124332E20620CC08E3221F490
:10F4B00026FD5FC1206406C08C3611F4206802C0AE
:10F4C000883641F4F60193FD859193FF81916F0198
:10F4D0008111C1CF982F9F7D9554933028F40C5FF4
:10F4E0001F4FFFE3F9830DC0833631F0833771F08E
:10F4F000833509F057C021C0F801808189830E5FF0
:10F500001F4F44244394512C540114C03801F2E09D
:10F510006F0E711CF801A080B18026FF03C0652D1D
:10F5200070E002C06FEF7FEFC5012C8765D12C0121
:10F5300083012C852F77222E16C03801F2E06F0E42
:10F54000711CF801A080B18026FF03C0652D70E01A
:10F5500002C06FEF7FEFC5012C8743D12C012C85B2
:10F560002068222E830123FC19C0832D90E04816C9
:10F570005906A0F4B70180E290E049D13A94F5CF62
:10F58000F50127FC859127FE81915F01B70190E08D
:10F590003ED131103A94F1E04F1A51084114510410
:10F5A00079F7DEC0843611F0893631F5F80127FF8E
:10F5B00007C060817181828193810C5F1F4F08C0F9
:10F5C00060817181882777FD8095982F0E5F1F4F8E
:10F5D0002F76B22E97FF09C0909580957095619512
:10F5E0007F4F8F4F9F4F2068B22E2AE030E0A4015A
:10F5F00040D1A82EA81843C0853729F42F7EB22EFB
:10F600002AE030E025C0F22FF97FBF2E8F36C1F0FF
:10F6100018F4883579F0ADC0803719F0883721F0BB
:10F62000A8C02F2F2061B22EB4FE0DC08B2D846098
:10F63000B82E09C024FF0AC09F2F9660B92E06C0BD
:10F6400028E030E005C020E130E002C020E132E0F7
:10F65000F801B7FE07C060817181828193810C5FE0
:10F660001F4F06C06081718180E090E00E5F1F4FE8
:10F67000A401FFD0A82EA818FB2DFF77BF2EB6FE41
:10F680000BC02B2D2E7FA51450F4B4FE0AC0B2FC83
:10F6900008C02B2D2E7E05C07A2C2B2D03C07A2C72
:10F6A00001C0752C24FF0DC0FE01EA0DF11D808103
:10F6B000803311F4297E09C022FF06C0739473942D
:10F6C00004C0822F867809F0739423FD12C020FFB6
:10F6D00006C05A2C731418F4530C5718732C731457
:10F6E00060F4B70180E290E02C8791D073942C8570
:10F6F000F6CF731410F4371801C0312C24FF11C059
:10F70000B70180E390E02C8782D02C8522FF16C0C1
:10F7100021FF03C088E590E002C088E790E0B701D0
:10F720000CC0822F867851F021FD02C080E201C01A
:10F730008BE227FD8DE2B70190E069D0A51430F48B
:10F74000B70180E390E063D05A94F8CFAA94F40113
:10F75000EA0DF11D8081B70190E059D0A110F6CFDC
:10F76000332009F45DCEB70180E290E050D03A94A6
:10F77000F7CFF7018681978102C08FEF9FEF2C961C
:10F780000FB6F894DEBF0FBECDBFDF91CF911F91B2
:10F790000F91FF90EF90DF90CF90BF90AF909F9030
:10F7A0008F907F906F905F904F903F902F90089533
:10F7B000F999FECF92BD81BDF89A992780B5089539
:10F7C000262FF999FECF1FBA92BD81BD20BD0FB67D
:10F7D000F894FA9AF99A0FBE019608959927882706
:10F7E0000895FC010590615070400110D8F7809594
:10F7F00090958E0F9F1F0895FC01615070400190FD
:10F800000110D8F7809590958E0F9F1F08950F9344
:10F810001F93CF93DF93182F092FEB018B8181FD6D
:10F8200003C08FEF9FEF20C082FF10C04E815F8129
:10F830002C813D81421753077CF4E881F9819F01B7
:10F840002F5F3F4F39832883108306C0E885F985F1
:10F85000812F1995892B29F72E813F812F5F3F4FEB
:10F860003F832E83812F902FDF91CF911F910F9196
:10F870000895FA01AA27283051F1203181F1E89446
:10F880006F936E7F6E5F7F4F8F4F9F4FAF4FB1E093
:10F890003ED0B4E03CD0670F781F891F9A1FA11D8E
:10F8A000680F791F8A1F911DA11D6A0F711D811D8F
:10F8B000911DA11D20D009F468943F912AE0269F54
:10F8C00011243019305D3193DEF6CF010895462FB3
:10F8D0004770405D4193B3E00FD0C9F7F6CF462F94
:10F8E0004F70405D4A3318F0495D31FD40524193FD
:10F8F00002D0A9F7EACFB4E0A695979587957795BA
:10F900006795BA95C9F700976105710508959B0140
:10F91000AC010A2E06945795479537952795BA95C9
:10F92000C9F7620F731F841F951FA01D089515E16D
:10F93000C2E6D5E100E005C022970109FE010BBF38
:10F94000C9D9C436D10780E00807B1F7F894FFCFD2
:10F9500060EA00000080BB440100003E4300004814
:10F96000430000C8426400640000803B4500803BC7
:10F97000450000704300000000CDCCCC3D0000529B
:10F980004300007A4301FF3FFF3F0000803F1070BB
:10F99000594485F4103E9A99B141010101010100D9
:10F9A0000049420000494200003D440000CC4300B1
:10F9B00000FA430000FA430000A04000003442284F
:10F9C000230000282300006400000010270000042A
:10F9D000050300018787AA878708080808084D31B2
:10F9E0003130002569206D696E2C202569207365F2
:10F9F00063005573696E672044656661756C742099
:10FA000073657474696E67733A004820004C200077
:10FA10004D31303420496E76616C696420657874AC
:10FA2000727564657220004D31303520496E766103
:10FA30006C696420657874727564657220004D315C
:10FA4000303920496E76616C69642065787472750E
:10FA500064657220003F006F6B0020703A002069DF
:10FA60003A0020643A0020633A005400496E7661FF
:10FA70006C696420657874727564657200416374A2
:10FA80006976652045787472756465723A20004D18
:10FA900032390000000100250030001D000C001864
:10FAA00000240031001C000B00170023002F001B56
:10FAB000000A001E000D0004000300080022002BB5
:10FAC000001A00090000000100FFFF020058595A07
:10FAD000452F0043616E6E6F74206F70656E2073EA
:10FAE0007562646972006175746F25692E67004DD7
:10FAF0003233202573004D3234004D3834205820E5
:10FB000059205A204500000000008F4D4B712E00F7
:10FB1000504944204175746F74756E65207374612B
:10FB2000727400537465707261746520746F20681C
:08FB3000696768203A2000001B
:00000001FF
